:100000000C94B80B0C94AB9F0C94DC9F0C940DA03B
:100010000C943EA00C946FA00C94A0A00C94D1A0C2
:100020000C9402A10C94E90B0C94E90B0C94E90BD1
:100030000C94E90B0C94E90B0C94E90B0C94E90B70
:100040000C94E90B0C94290F0C94E90B0C94E90B1C
:100050000C94E90B0C94E90B0C94877D0C94DBA2B7
:100060000C94E90B0C94CB7E0C94E90B0C94E90BEB
:100070000C94E90B0C94E90B0C94E90B0C94E90B30
:100080000C94E90B0C94E90B0C94E90B0C94E90B20
:100090000C94E90B0C94E90B0C94E90B0C94E90B10
:1000A0000C94E90B0C94E90B0C94E90B0C94E90B00
:1000B0000C94E90B0C94E90B0C94E90B0C94E90BF0
:1000C0000C94E90B0C94E90B0C94E90B0C94E90BE0
:1000D0000C94E90B0C94E90B0C94E90B0C94E90BD0
:1000E0000C94E90B084AD73B3BCE016E84BCBFFDA4
:1000F000C12F3D6C74319ABD56833DDA3D00C77FF8
:1001000011BED9E4BB4C3E916BAAAABE0000008090
:100110003F05A84CCDB2D44EB93836A9020C50B91F
:10012000918688083CA6AAAA2ABE000000803F65E6
:1001300063686F3A00656E6473746F7073206869EA
:10014000743A200020583A0020593A00205A3A00C8
:1001500024F404D9201BC40C5C0E9804C4095F026B
:1001600065077101F405F900FB04B300480487003A
:10017000C10369005803550003034500BE023A005D
:100180008402310053022A002902250004022000C3
:10019000E4011C00C8011900AF0117009801140008
:1001A00084011300710110006101100051010E0063
:1001B00043010D0036010B002B010B0020010B0049
:1001C000150109000C01090003010800FB000800EB
:1001D000F3000800EB000700E4000600DE00060064
:1001E000D8000600D2000600CC000500C7000500BC
:1001F000C2000500BD000400B9000400B500040001
:10020000B1000400AD000400A9000400A500030033
:10021000A20003009F0004009B000300980003005D
:100220009500020093000300900003008D0002007F
:100230008B00030088000200860002008400030097
:10024000810002007F0002007D0002007B000200AE
:1002500079000200770001007600020074000200BD
:1002600072000100710002006F0002006D000100C9
:100270006C0002006A0001006900020067000100D2
:1002800066000100650001006400020062000100D8
:1002900061000100600001005F0002005D000100DC
:1002A0005C0001005B0001005A00010059000100E0
:1002B00058000100570001005600010055000100E0
:1002C00054000100530000005300010052000100DF
:1002D00051000100500001004F0001004E000000DD
:1002E0004E0001004D0001004C0001004B000000D9
:1002F0004B0001004A0001004900010048000000D5
:1003000048000100470001004600000046000100CF
:1003100045000000450001004400010043000000CA
:1003200043000100420000004200010041000000C3
:1003300041000100400001003F0000003F000100BB
:100340003E0000003E0001003D0000003D000100B5
:100350003C0000003C0000003C0001003B000000AD
:100360003B0001003A0000003A00010039000000A3
:10037000390001003800000038000000380001009A
:100380003700000037000100360000003600000092
:100390003600010035000000350000003500010086
:1003A000340000003400000034000100330000007D
:1003B0003300000033000100320000003200000072
:1003C0003200010031000000310000003100010066
:1003D0003000000030000000300001002F0000005D
:1003E0002F0000002F0000002F0001002E00000051
:1003F0002E0000002E0001002D0000002D00000046
:100400002D0000002D0001002C0000002C00000039
:100410002C0000002C0001002B0000002B0000002D
:100420002B0000002B0001002A0000002A00000021
:100430002A0000002A000100290000002900000015
:100440002900000029000000290001002800000008
:1004500028000000280000002800000028000100FB
:1004600027000000270000002700000027000000F0
:1004700027000100260000002600000026000000E2
:1004800026000000260001002500000025000000D5
:1004900025000000250000002500000025000100C7
:1004A00024000000240000002400000024000000BC
:1004B00024000100230000002300000023000000AE
:1004C000230000002300000023000000230001009F
:1004D0002200000022000000220000002200000094
:1004E0002200000022000100210000002100000085
:1004F0002100000021000000210000002100000078
:100500002100010020000000200000002000000069
:10051000200000002000000020000000200000005B
:10052000200001001F0000001F0000001F0000004D
:100530001F0000001F0000001F0000001F0001003E
:100540001E0000001E0000001E0000001E00000033
:1005500024F4D43050C38E20C2A24017828B701175
:10056000127A910D816CD90AA861E108C758660713
:10057000615143061E4B5D05C145A7041A41110494
:10058000093D9803713931034036DB02653391022E
:10059000D4305402802E1D02632CEE01752AC50151
:1005A000B028A001102781018F2564012B244B0165
:1005B000E0223401AC211F018D200D01801FFC00C1
:1005C000841EED00971DDF00B81CD200E61BC6009C
:1005D000201BBC00641AB200B219A8000A19A000BE
:1005E0006A189900D117910040178B00B516840046
:1005F00031167E00B31579003A157300C7146F00E9
:1006000058146A00EE1366008813630025135E0019
:10061000C7125B006C12570015125400C111510033
:1006200070114F0021114B00D61049008D1047006A
:100630004610440002104200C00F4000800F3E00F0
:10064000420F3C00060F3B00CB0E3800930E3700E4
:100650005C0E3500270E3400F30D3200C10D310061
:10066000900D3000600D2E00320D2D00050D2C0078
:10067000D90C2B00AE0C2900850C29005C0C27003E
:10068000350C27000E0C2600E80B2400C40B2400B8
:10069000A00B23007D0B23005A0B2100390B2100F6
:1006A000180B2000F80A1F00D90A1E00BB0A1E0002
:1006B0009D0A1D00800A1D00630A1C00470A1B00DA
:1006C0002C0A1B00110A1A00F7091A00DD0919008B
:1006D000C4091900AB091900920917007B09180019
:1006E000630917004C091600360916002009160088
:1006F0000A091500F5081500E0081400CC081400DC
:10070000B8081400A4081400900813007D08120013
:100710006B08130058081200460812003408110034
:10072000230811001208110001081100F007100041
:10073000E0071000D0071000C0071000B0070F003E
:10074000A107100091070E0083070F0074070F0028
:1007500065070E0057070E0049070E003B070D0006
:100760002E070E0020070D0013070D0006070D00D1
:10077000F9060C00ED060D00E0060C00D4060C0096
:10078000C8060C00BC060C00B0060C00A4060B004A
:1007900099060C008D060B0082060B0077060B00F5
:1007A0006C060B0061060A0057060B004C060A0097
:1007B00042060A0038060A002E060A0024060A002D
:1007C0001A060A001006090007060A00FD050900BE
:1007D000F4050900EB050900E2050900D905090047
:1007E000D0050900C7050900BE050900B5050800C8
:1007F000AD050800A50509009C0508009405080042
:100800008C050800840508007C05080074050800B4
:100810006C050700650508005D0507005605080022
:100820004E0507004705070040050800380507008A
:10083000310507002A050700230507001C050600EF
:10084000160507000F05070008050600020507004A
:10085000FB040600F5040700EE040600E8040600A9
:10086000E2040700DB040600D5040600CF040600FE
:10087000C9040600C3040600BD040600B704060050
:10088000B1040500AC040600A6040600A00405009F
:100890009B04060095040500900406008A040500E8
:1008A00085040500800406007A040500750405002F
:1008B000700405006B040500660405006104050072
:1008C0005C04050057040500520405004D040500B2
:1008D00048040500430405003E0404003A040500F2
:1008E00035040500300404002C040500270404002E
:1008F000230405001E0404001A0404001604050065
:10090000110404000D04040009040500040404009B
:1009100000040400FC030400F8030400F4030400D2
:10092000F0030400EC030400E8030400E403040003
:10093000E0030400DC030400D8030400D403040033
:10094000D0030400CC030400C8030300C503030064
:1009500052656C65617365642E007C3C3E5E2B3D88
:100960003F2F5B5D3B2C2A225C006563686F3A0079
:10097000656E717565696E6720220022007374616F
:10098000727400506F7765725570002045787465F9
:10099000726E616C205265736574002042726F77CD
:1009A0006E206F75742052657365740020576174F2
:1009B0006368646F672052657365740020536F66C7
:1009C0007477617265205265736574004D61726C55
:1009D000696E2000312E302E302052433200204CE0
:1009E00061737420557064617465643A20004D61D0
:1009F000726C696E2D4D6F6E2C203131204A756EF0
:100A000020323031322031373A33333A3432202BEE
:100A100030323030202D20623637646163646338B1
:100A20006631626434383965303538653136643959
:100A3000326261323963333634623261386535008F
:100A4000207C20417574686F723A20004275696C91
:100A5000642D4D652D4D61726C696E002046726586
:100A600065204D656D6F72793A20002020506C61D1
:100A70006E6E657242756666657242797465733A28
:100A8000200053746F7265642073657474696E67B7
:100A900073207265747265697665643A0053746593
:100AA00070732070657220756E69743A0020204D55
:100AB0003932205800205900205A002045004D614D
:100AC00078696D756D206665656472617465732003
:100AD000286D6D2F73293A0020204D323033205875
:100AE00000205900205A002045004D6178696D753D
:100AF0006D20416363656C65726174696F6E202857
:100B00006D6D2F7332293A0020204D32303120583C
:100B100000205900205A00204500416363656C6540
:100B2000726174696F6E3A20533D616363656C65F1
:100B3000726174696F6E2C20543D726574726163CA
:100B40007420616363656C65726174696F6E002007
:100B5000204D323034205300205400416476616EC1
:100B6000636564207661726961626C65733A2053D3
:100B70003D4D696E20666565647261746520286DFF
:100B80006D2F73292C20543D4D696E20747261764F
:100B9000656C20666565647261746520286D6D2FD3
:100BA00073292C20423D6D696E696D756D207365EA
:100BB000676D656E742074696D6520286D73292CCE
:100BC00020583D6D6178696D756D207859206A6592
:100BD000726B20286D6D2F73292C20205A3D6D617A
:100BE00078696D756D205A206A65726B20286D6D6D
:100BF0002F73290020204D3230352053002054001F
:100C0000204200205800205A00204500504944202E
:100C100073657474696E67733A002020204D333019
:100C2000312050002049002044006F6B00446F6E5B
:100C30006520736176696E672066696C652E004574
:100C400072726F723A004C696E65204E756D626506
:100C500072206973206E6F74204C617374204C692C
:100C60006E65204E756D6265722B312C204C617360
:100C700074204C696E653A00636865636B73756DCB
:100C8000206D69736D617463682C204C61737420EE
:100C90004C696E653A004E6F20436865636B7375EF
:100CA0006D2077697468206C696E65206E756D6261
:100CB00065722C204C617374204C696E653A004E4D
:100CC0006F204C696E65204E756D62657220776984
:100CD000746820636865636B73756D2C204C617359
:100CE00074204C696E653A006F6B005072696E74C7
:100CF00065722073746F707065642064657520740C
:100D00006F206572726F72732E2046697820746846
:100D100065206572726F7220616E64207573652044
:100D20004D39393920746F20726573746172742182
:100D30002E202854656D7065726174757265206926
:100D4000732072657365742E205365742069742056
:100D50006265666F72652072657374617274696E24
:100D600067290053544F505045442E2000446F6E65
:100D700065207072696E74696E672066696C6500C3
:100D8000536C6565702E2E2E005761697420666F56
:100D90007220757365722E2E2E004E6F206D6F7649
:100DA000652E00426567696E2066696C65206C6916
:100DB000737400456E642066696C65206C69737499
:100DC000006F6B20543A00202F0020423A00202F61
:100DD0000020403A0048656174696E672E2E2E002F
:100DE000543A0020453A0020573A0048656174693A
:100DF0006E6720646F6E652E0042656420486561F1
:100E000074696E672E00543A0020453A0020423A39
:100E10000042656420646F6E652E005061727469D3
:100E2000616C2052656C65617365004649524D578F
:100E30004152455F4E414D453A4D61726C696E209D
:100E400056313B20537072696E7465722F677262FF
:100E50006C206D617368757020666F722067656EB7
:100E600036204649524D574152455F55524C3A68DB
:100E70007474703A2F2F6669726D776172652E7582
:100E80006C74696D616B65722E636F6D2050524F8B
:100E9000544F434F4C5F56455253494F4E3A312EB3
:100EA00030204D414348494E455F545950453A55CD
:100EB0006C74696D616B6572204558545255444598
:100EC000525F434F554E543A310A00583A00593A4E
:100ED000005A3A00453A0020436F756E7420583A24
:100EE00000593A005A3A00785F6D696E3A00785FAF
:100EF0006D61783A00795F6D696E3A00795F6D6176
:100F0000783A007A5F6D696E3A007A5F6D61783A7F
:100F100000556E6B6E6F776E20636F6D6D616E64E2
:100F20003A2200220053657474696E67732053740B
:100F30006F72656400526573656E643A006F6B0092
:100F40005072696E7465722068616C7465642E20DD
:100F50006B696C6C28292063616C6C6564202121AD
:100F6000004B494C4C45442E20005072696E74650C
:100F7000722073746F707065642064657520746F7F
:100F8000206572726F72732E2046697820746865CE
:100F9000206572726F7220616E6420757365204DDA
:100FA00039393920746F2072657374617274212E1F
:100FB000202854656D70657261747572652069735F
:100FC0002072657365742E205365742069742062E5
:100FD00065666F72652072657374617274696E679D
:100FE000290053544F505045442E2000556C7469CD
:100FF0006D616B65722052656164792E00022D2D42
:101000002D2F2D2D2D0120006820006D005A3A0053
:1010100025200025534400204D61696E20030020E7
:101020004175746F737461727400204469736162F6
:101030006C6520537465707065727300204175741F
:101040006F20486F6D650020536574204F7269678B
:10105000696E00205072656865617420504C4100D3
:101060002050726568656174204142530020436FCF
:101070006F6C646F776E00204D6F766520417869E4
:10108000732020202020207E002050726570617225
:101090006520030020583A0020593A00205A3A00AF
:1010A000204578747275646500204D61696E200377
:1010B000002053706565643A0020024E6F7A7A6CA6
:1010C000653A0020024265643A002046616E207352
:1010D000706565643A0020466C6F773A0020436F74
:1010E0006E74726F6C20030020024E6F7A7A6C650A
:1010F0003A002046616E2073706565643A002050A6
:1011000049442D503A2000205049442D493A2000AE
:10111000205049442D443A2000205049442D433A60
:10112000200020436F6E74726F6C200300204163B7
:10113000633A00303000303000205678792D6A65EF
:10114000726B3A200020566D61782000783A007961
:101150003A007A3A00653A0020566D696E3A0020EE
:101160005654726176206D696E3A0020416D617847
:101170002000783A00793A007A3A00653A00303037
:101180000030300020412D726574726163743A0042
:10119000303000303000205873746570732F6D6DDF
:1011A0003A00205973746570732F6D6D3A00205AA0
:1011B00073746570732F6D6D3A002045737465709C
:1011C000732F6D6D3A00204D61696E202020202024
:1011D00020202003002054656D7065726174757263
:1011E00065207E00204D6F74696F6E2020202020C6
:1011F000207E002053746F7265206D656D6F72796B
:1012000000204C6F6164206D656D6F727900205213
:101210006573746F7265204661696C736166650001
:10122000204D61696E200300045265667265736823
:1012300000200020576174636820202003002050A4
:10124000726570617265207E002054756E65202085
:1012500020207E0020436F6E74726F6C207E002011
:1012600053746F70205072696E742020207E0020AD
:1012700043617264204D656E75202020207E002021
:101280004E6F204361726400536F6D657468696EC0
:10129000672069732077726F6E6720696E207468AB
:1012A00065204D656E755374727563747572652E25
:1012B000004361726420696E7365727465640043F3
:1012C0006172642072656D6F766564002062696189
:1012D000733A200020643A2000206D696E3A2000A5
:1012E000206D61783A2000204B753A20002054751B
:1012F0003A200020436C6173696320504944200008
:10130000204B703A2000204B693A2000204B643A71
:101310002000504944204175746F74756E652066D5
:1013200061696C6564212054656D706572617475C6
:10133000726520746F2068696768006F6B20543A8B
:101340000020403A00504944204175746F74756E16
:1013500065206661696C6564212074696D656F75CF
:101360007400504944204175746F74756E65206631
:10137000696E6973686564202120506C6163652023
:10138000746865204B702C204B6920616E64204B83
:101390006420636F6E7374616E747320696E207461
:1013A000686520636F6E66696775726174696F6ED8
:1013B0002E68004572726F723A00202D20496E76B9
:1013C000616C6964206578747275646572206E75ED
:1013D0006D6265722100202D20496E76616C696412
:1013E000206578747275646572206E756D626572C1
:1013F0002021003A204578747275646572207377F5
:10140000697463686564206F66662E204D41585488
:10141000454D5020747269676765726564202100CC
:101420003A204578747275646572207377697463C5
:10143000686564206F66662E204D494E54454D50B8
:101440002074726967676572656420210054656D58
:101450007065726174757265206865617465642079
:10146000626564207377697463686564206F66667B
:101470002E204D415854454D502074726967676560
:10148000726564202121006563686F3A005344202F
:10149000696E6974206661696C004572726F723A98
:1014A00000766F6C756D652E696E69742066616972
:1014B0006C6564006F70656E526F6F742066616951
:1014C0006C65640053442063617264206F6B006F2D
:1014D00070656E206661696C65642C2046696C6578
:1014E0003A20002E0046696C65206F70656E656459
:1014F0003A002053697A653A0046696C6520736545
:101500006C6563746564006F70656E206661696CFC
:1015100065642C2046696C653A20002E006F70656A
:101520006E206661696C65642C2046696C653A20A2
:10153000002E0057726974696E6720746F206669A7
:101540006C653A20006F70656E206661696C656439
:101550002C2046696C653A20002E0046696C652097
:1015600064656C657465643A0044656C6574696FA4
:101570006E206661696C65642C2046696C653A2052
:10158000002E005344207072696E74696E67206289
:1015900079746520002F004E6F74205344207072C0
:1015A000696E74696E67006572726F722077726916
:1015B00074696E6720746F2066696C650043616EA4
:1015C0006E6F7420656E74657220737562646972E3
:1015D0003A006563686F3A0020636F6C6420657839
:1015E00074727573696F6E2070726576656E74655E
:1015F000640020746F6F206C6F6E67206578747262
:101600007573696F6E2070726576656E74656400BF
:101610000000090A02080B0C0D0706030401000074
:1016200000000000000000000000000000000000BA
:1016300000000000000000000000000011100F007A
:10164000000000000000000000000000000000009A
:1016500000000000000001021020200808102040B7
:101660001020408002010201080402010102040866
:1016700010204080804020100804020180040201F4
:10168000804020100804020108040201010204083D
:101690001020408001020408102040800505050547
:1016A000070508080808020202020A0A08080404DA
:1016B0000404010101010101010103030303030308
:1016C0000303040707070C0C0C0C0C0C0C0C020297
:1016D000020206060606060606060B0B0B0B0B0B94
:1016E0000B0B000020002300260029002C002F00F7
:1016F0003200000100000301060109010000220080
:10170000250028002B002E003100340002010000CB
:10171000050108010B0100002100240027002A0018
:101720002D003000330001010000040107010A010F
:10173000494E46494E4954594E414E000020410001
:1017400000C84200401C4620BCBE4CCA1B0E5AAE0C
:10175000C59D74CDCCCC3D0AD7233C17B7D1387783
:10176000CC2B329595E6241FB14F0A00F974FE7414
:1017700011241FBECFEFD1E2DEBFCDBF00E00CBF12
:1017800014E0A0E0B2E0EEE4F3E601E00BBF02C03B
:1017900007900D92AC38B107D9F710E1ACE8B4E08E
:1017A00001C01D92AA35B107E1F717E1CEE6D7E1F6
:1017B00000E006C022970109FE010BBF0E9451AB59
:1017C000CC36D10780E00807A9F70E94F6A30C9455
:1017D00095B10C940000282F30E0A901559547954C
:1017E00040654CBD80FD03C091E0863009F490E077
:1017F0009DBD08958FEF8EBD0DB407FEFDCF8EB554
:1018000008958EBD0DB407FEFDCF0895FC018081C3
:1018100061E00E94A4A20895CF93DF93EC018A8136
:101820000E94EB0B888160E00E94A4A2DF91CF911F
:101830000895CF92DF92EF92FF920F931F93CF9371
:10184000DF93EC016B018A010E9425A3DC01CB012F
:101850007C010AC00E9425A36E197F0981E06D32C8
:10186000780710F081E108C00E94FA0B8B838F3F4C
:1018700089F38E3F39F08FE08983CE010E94060CF8
:1018800080E027C098012150304001151105C9F0B2
:101890008FEF8EBDF60180E090E04FEF07C00DB4F2
:1018A00007FEFDCF5EB551934EBD0196821793079B
:1018B000B0F30DB407FEFDCF8EB52C0D3D1DF90123
:1018C00080830E94FA0B0E94FA0BCE010E94060C44
:1018D00081E0DF91CF911F910F91FF90EF90DF900A
:1018E000CF9008950F931F93CF93DF93EB010E9446
:1018F00025A38B019C0107C00E9425A3601B710BCF
:101900006C177D0730F40E94FA0B8F3FA9F781E036
:1019100001C080E0DF91CF911F910F9108958F92C8
:101920009F92AF92BF92EF92FF920F931F93CF932C
:101930007C01C62F49015A010E940C0CC7016CE2C0
:1019400071E00E94720C8C2F80640E94010C08E1EF
:1019500010E0D501C401002E04C0B695A795979557
:1019600087950A94D2F70E94010C085010408FEF1F
:10197000083F180771F7CC2321F0C83021F08FEF12
:1019800003C085E901C087E80E94010CCC3011F446
:101990000E94FA0BC0E00E94FA0BF701838387FFD5
:1019A00004C0CF3F11F0CF5FF6CFCF911F910F91C1
:1019B000FF90EF90BF90AF909F908F900895CF923F
:1019C000DF92EF92FF920F931F93CF93DF93EC017F
:1019D0006A017B0189018C81833039F0A9E0CC0C4C
:1019E000DD1CEE1CFF1CAA95D1F7CE0161E1A70119
:1019F00096010E948F0C882339F084E08983CE0100
:101A00000E94060C80E006C0CE01B80140E052E022
:101A10000E94190CDF91CF911F910F91FF90EF90D1
:101A2000DF90CF900895AF92BF92CF92DF92EF9266
:101A3000FF920F931F93CF93DF93EC01162F1C821D
:101A4000198248830E9425A3DC01CB015C018881B7
:101A500061E00E9483A2CE010E94060C82E360E056
:101A60000E9483A283E361E00E9483A284E361E099
:101A70000E9483A285E361E00E9483A285E361E086
:101A80000E94A4A285E08A830E94EB0B0AE08FEFFC
:101A90000E94010C0150D9F70AC00E9425A36A19BF
:101AA0007B0987E0613D780710F081E05AC0CE01E4
:101AB00060E020E030E040E050E00E948F0C082F12
:101AC0008B83813051F7CE0168E02AEA31E040E0B3
:101AD00050E00E948F0C82FF02C00C830CC004E017
:101AE0000E94FA0B8B830150D9F78A3A11F082E0F9
:101AF00038C082E08C838C81823031F4C12CD12CAF
:101B0000E12CB0E4FB2E0EC0CC24DD2476010AC00B
:101B10000E9425A36A197B0987E0613D780710F0D0
:101B20008AE01FC0CE0167E320E030E040E050E0F3
:101B30000E948F0CCE0169E2A70196010E948F0CD2
:101B40008B83882329F78C818230E9F4CE016AE304
:101B500020E030E040E050E00E948F0C882331F01C
:101B600088E08983CE010E94060C18C00E94FA0BFF
:101B7000807C803C11F483E08C830E94FA0B0E94ED
:101B8000FA0B0E94FA0BCE010E94060C173018F0D7
:101B900088E1898303C01A8381E001C080E0DF917E
:101BA000CF911F910F91FF90EF90DF90CF90BF905A
:101BB000AF900895CF93DF93EC016EBDFA0180E002
:101BC00090E00DB407FEFDCF20812EBD0DB407FEC1
:101BD000FDCF21812EBD0296329622E08030920701
:101BE00081F70DB407FEFDCF8FEF0E94010C8FEF40
:101BF0000E94010C0E94FA0B8B838F71853039F0A3
:101C000083E18983CE010E94060C80E001C081E05F
:101C1000DF91CF910895CF92DF92EF92FF920F93D1
:101C20001F93CF93DF93EC016A017B0189018C81C3
:101C3000833039F089E0CC0CDD1CEE1CFF1C8A954A
:101C4000D1F7CE0168E1A70196010E948F0C88238D
:101C500011F086E01FC0CE016EEFA8010E94DA0DE0
:101C60008823C9F0CE0168E572E00E94720C8823D7
:101C700011F487E10FC0CE016DE020E030E040E0DC
:101C800050E00E948F0C882321F40E94FA0B8823D5
:101C900079F086E18983CE010E94060C80E0DF9115
:101CA000CF911F910F91FF90EF90DF90CF9008950B
:101CB000CE010E94060C81E0F2CF80919E04882321
:101CC00049F480919D04882329F480919C04882301
:101CD00009F4AEC0EFE2F1E007C09091C00095FFBB
:101CE000FCCF8093C600319684918823B1F7E5E359
:101CF000F1E007C09091C00095FFFCCF8093C60033
:101D0000319684918823B1F780919E04882349F10C
:101D1000E4E4F1E007C09091C00095FFFCCF809310
:101D2000C600319684918823B1F760919F04709129
:101D3000A0048091A1049091A2040E94D5A72091B3
:101D400003103091041040910510509106100E942C
:101D50003AA7AB01BC018FE59AE022E030E00E9497
:101D60002B8180919D04882349F1E8E4F1E007C0CC
:101D70009091C00095FFFCCF8093C600319684916E
:101D80008823B1F76091A3047091A4048091A50405
:101D90009091A6040E94D5A72091071030910810B9
:101DA0004091091050910A100E943AA7AB01BC0162
:101DB0008FE59AE022E030E00E942B8180919C0424
:101DC000882349F1ECE4F1E007C09091C00095FF51
:101DD000FCCF8093C600319684918823B1F760913F
:101DE000A7047091A8048091A9049091AA040E946C
:101DF000D5A720910B1030910C1040910D105091EF
:101E00000E100E943AA7AB01BC018FE59AE022E0D8
:101E100030E00E942B818091C00085FFFCCF8AE0DA
:101E20008093C60010929E0410929D0410929C0410
:101E3000089510929E0410929D0410929C0408959F
:101E4000809307040895EFE6F0E08081826080834C
:101E500008951F920F920FB60F920BB60F92112496
:101E60000F931F932F933F934F935F936F937F93A2
:101E70008F939F93AF93BF93CF93DF93EF93FF9392
:101E80008091AF049091B004009709F086C19091C1
:101E9000E60A8091E50A9817A1F02091E50A30E062
:101EA0008DE490E0289FF001299FF00D389FF00D00
:101EB0001124E951F54FDF01A45BBF4F81E08C9302
:101EC00002C0E0E0F0E0F093B004E093AF0430979C
:101ED00009F45DC1DF01A45BBF4F81E08C931092D8
:101EE000B1041092B2041092B3041092B40460AD25
:101EF00071AD2CE96134720728F49EE461327907F0
:101F000048F002C060E47CE9769567957695679520
:101F100084E007C0E7E261317E0730F0769567958F
:101F200082E08093B50407C08093B50460327105E8
:101F300010F460E270E060527040F8E060307F07BB
:101F4000E0F0272F30E0220F331F220F331F205BDA
:101F50003E4FF901329685919491AA27699FE0013D
:101F6000689FC10DDA1F0694CA1FDA1F1124F901F8
:101F7000459154914C1B5D0B1FC0CB0196958795E5
:101F80008C7F805B9A4FFC01459154910296FC0135
:101F9000A591B491862F90E087709070A89F9001D2
:101FA000A99F300DB89F300D1124D3E036952795A9
:101FB000DA95E1F7421B530B44365105A0F4E0E0FB
:101FC000F2E006C09091C00095FFFCCF8093C60060
:101FD00081918823B9F78FE59AE04AE050E00E94AA
:101FE000508044E650E05093B7044093B604E0912B
:101FF000AF04F091B00464AD75AD7093B904609313
:10200000B8042CE96134720728F48EE46132780751
:1020100048F002C060E47CE976956795769567950F
:1020200084E007C097E26131790730F076956795D3
:1020300082E08093B50408C081E08093B5046032EB
:10204000710510F460E270E060527040E8E06030CA
:102050007E07E0F0272F30E0220F331F220F331FBF
:10206000205B3E4FF901329685919491AA27699F92
:10207000E001689FC10DDA1F0694CA1FDA1F112400
:10208000F901459154914C1B5D0B1FC0CB019695F6
:1020900087958C7F805B9A4FFC0145915491029605
:1020A000FC01A591B491862F90E087709070A89F55
:1020B0009001A99F300DB89F300D1124E3E03695B3
:1020C0002795EA95E1F7421B530B44365105A0F4DE
:1020D000E0E0F2E006C09091C00095FFFCCF809355
:1020E000C60081918823B9F78FE59AE04AE050E075
:1020F0000E94508044E650E0CA01A0E0B0E0809326
:10210000BA049093BB04A093BC04B093BD04509355
:10211000890040938800E091AF04F091B004808979
:102120009189A289B389B695A79597958795B0951A
:10213000A095909581959F4FAF4FBF4F8093BE0460
:102140009093BF04A093C004B093C1048093C204D1
:102150009093C304A093C404B093C5048093C604B1
:102160009093C704A093C804B093C9048093CA0491
:102170009093CB04A093CC04B093CD041092AB0405
:102180001092AC041092AD041092AE0406C080ED23
:1021900097E09093890080938800E091AF04F091DC
:1021A000B004309709F435C580A18093CE0480FF38
:1021B0003CC0119A8FEF8093030480910704882319
:1021C00009F46DC020B1217031E0232759F18091CD
:1021D000CF04882339F180819181A281B3811816BF
:1021E00019061A061B06F4F480918C0490918D0454
:1021F000A0918E04B0918F0480939F049093A004CB
:10220000A093A104B093A20430939E048089918985
:10221000A289B3898093AB049093AC04A093AD04DE
:10222000B093AE042093CF043AC0119881E080931C
:10223000030480910704882391F121E0029B02C0EE
:1022400020E02BC08091D004882339F180819181D6
:10225000A281B381181619061A061B06F4F48091A0
:102260008C0490918D04A0918E04B0918F04809382
:102270009F049093A004A093A104B093A204209380
:102280009E0480899189A289B3898093AB0490933D
:10229000AC04A093AD04B093AE042093D00480911D
:1022A000CE0481FF40C044988FEF80930404809156
:1022B0000704882309F475C021E0049B02C020E0D4
:1022C0002FC08091D104882359F1E091AF04F0919F
:1022D000B00484819581A681B781181619061A0663
:1022E0001B06F4F48091900490919104A0919204C3
:1022F000B09193048093A3049093A404A093A504A5
:10230000B093A60420939D0480899189A289B38902
:102310008093AB049093AC04A093AD04B093AE044F
:102320002093D1043EC0449A81E0809304048091BC
:1023300007048823B1F121E0069B02C020E02FC0F2
:102340008091D204882359F1E091AF04F091B00458
:1023500084819581A681B781181619061A061B0675
:10236000F4F48091900490919104A0919204B09122
:1023700093048093A3049093A404A093A504B09322
:10238000A60420939D0480899189A289B3898093B2
:10239000AB049093AC04A093AD04B093AE0420932F
:1023A000D2048091CE0482FF42C0A29A8FEF809324
:1023B000050480910704882309F477C026B120958D
:1023C000221F2227221F81F18091D304882361F1EB
:1023D000E091AF04F091B00480859185A285B3852A
:1023E000181619061A061B06FCF4809194049091A5
:1023F0009504A0919604B09197048093A7049093BC
:10240000A804A093A904B093AA0481E080939C043B
:1024100080899189A289B3898093AB049093AC049D
:10242000A093AD04B093AE042093D3043EC0A29811
:1024300081E080930504809107048823B1F121E0B5
:10244000359B02C020E02FC08091D404882359F12D
:10245000E091AF04F091B00480859185A285B385A9
:10246000181619061A061B06F4F48091940490912C
:102470009504A0919604B09197048093A70490933B
:10248000A804A093A904B093AA0420939C04808973
:102490009189A289B3898093AB049093AC04A093F3
:1024A000AD04B093AE042093D4048091CE049FB7C2
:1024B000F89483FF08C080910B018F7E80930B01FD
:1024C0009FBF8FEF07C080910B01806180930B014C
:1024D0009FBF81E080930604C0E0D0E086C1809178
:1024E000C00087FF1AC06091C6008091E00A9091F9
:1024F000E10AAC014F5F5F4F4F7750702091E20AC5
:102500003091E30A4217530741F0805A954FFC017E
:1025100060835093E10A4093E00AE091AF04F091A8
:10252000B0044091BE045091BF046091C00470910A
:10253000C10480819181A281B381480F591F6A1F14
:102540007B1F4093BE045093BF046093C0047093FC
:10255000C104141615061606170644F5139A808949
:102560009189A289B389481B590B6A0B7B0B409355
:10257000BE045093BF046093C0047093C1041398C9
:1025800080918C0490918D04A0918E04B0918F0461
:1025900020910304820F911DA11DB11D80938C0415
:1025A00090938D04A0938E04B0938F04E091AF04B8
:1025B000F091B0044091C2045091C3046091C404EE
:1025C0007091C50484819581A681B781480F591FF8
:1025D0006A1F7B1F4093C2045093C3046093C404DA
:1025E0007093C504141615061606170644F5469A88
:1025F00080899189A289B389481B590B6A0B7B0B8F
:102600004093C2045093C3046093C4047093C50400
:1026100046988091900490919104A0919204B09179
:10262000930420910404820F911DA11DB11D80937C
:10263000900490939104A0939204B0939304E0913A
:10264000AF04F091B0044091C6045091C70460916A
:10265000C8047091C90480859185A285B385480F0F
:10266000591F6A1F7B1F4093C6045093C704609391
:10267000C8047093C904141615061606170644F507
:10268000409A80899189A289B389481B590B6A0BAA
:102690007B0B4093C6045093C7046093C8047093A7
:1026A000C90440988091940490919504A091960457
:1026B000B091970420910504820F911DA11DB11DB9
:1026C0008093940490939504A0939604B0939704F8
:1026D000E091AF04F091B0048091CA049091CB04D2
:1026E000A091CC04B091CD0444855585668577854D
:1026F000840F951FA61FB71F8093CA049093CB0425
:10270000A093CC04B093CD04181619061A061B0624
:102710000CF042C09FB7F89480910B0180648093C5
:102720000B019FBFE091AF04F091B0048091CA0407
:102730009091CB04A091CC04B091CD0440895189F3
:1027400062897389841B950BA60BB70B8093CA040F
:102750009093CB04A093CC04B093CD049FB7F8948E
:1027600080910B018F7B80930B019FBF8091980418
:1027700090919904A0919A04B0919B042091060431
:10278000820F911DA11DB11D80939804909399040F
:10279000A0939A04B0939B048091AB049091AC04F5
:1027A000A091AD04B091AE040196A11DB11D80931E
:1027B000AB049093AC04A093AD04B093AE048091AD
:1027C000AB049091AC04A091AD04B091AE042196FD
:1027D000E091AF04F091B004408951896289738916
:1027E00084179507A607B70738F48091B50490E0E1
:1027F000C817D9070CF473CE4091AB045091AC04C8
:102800006091AD047091AE04E091AF04F091B0041A
:1028100084899589A689B78984179507A607B7077C
:1028200008F4DCC00091BA041091BB042091BC04F0
:102830003091BD04448D558D668D778DAA27059FF7
:10284000B12D169FC001269F900D259F800D911DD3
:10285000069FB00D811D9A1F159FB00D811D9A1FF7
:10286000249FB00D811D9A1F149FB10D8A1F9A1FBE
:10287000B6958A1F9A1F112424AD35AD280F391F34
:102880003093B9042093B80480AD91ADA2ADB3AD3F
:10289000A90160E070E084179507A607B70720F448
:1028A0009093B9048093B8046091B8047091B9040E
:1028B000FCE961347F0728F42EE46132720748F0A6
:1028C00002C060E47CE9769567957695679584E02B
:1028D00007C087E26131780730F07695679582E02E
:1028E0008093B50408C081E08093B504603271051F
:1028F00010F460E270E06052704098E06030790758
:10290000E0F0272F30E0220F331F220F331F205B10
:102910003E4FF901329685919491AA27699FE00173
:10292000689FC10DDA1F0694CA1FDA1F1124F9012E
:10293000459154914C1B5D0B1FC0CB01969587951B
:102940008C7F805B9A4FFC01459154910296FC016B
:10295000A591B491862F90E087709070A89F900108
:10296000A99F300DB89F300D1124D3E036952795DF
:10297000DA95E1F7421B530B44365105A0F4E0E031
:10298000F2E006C09091C00095FFFCCF8093C60096
:1029900081918823B9F78FE59AE04AE050E00E94E0
:1029A000508044E650E0509389004093880060E0F6
:1029B00070E08091BA049091BB04A091BC04B091E6
:1029C000BD04840F951FA61FB71F8093BA04909370
:1029D000BB04A093BC04B093BD04F6C04091AB040B
:1029E0005091AC046091AD047091AE04808D918DD6
:1029F000A28DB38D84179507A607B70708F0DCC032
:102A00000091B1041091B2042091B3043091B40448
:102A1000448D558D668D778DAA27059FB12D169F04
:102A2000E001269FD00D259FC00DD11D069FB00D42
:102A3000C11DDA1F159FB00DC11DDA1F249FB00DF7
:102A4000C11DDA1F149FB10DCA1FDA1FB695CA1F28
:102A5000DA1F11248091B8049091B904E05CFF4F13
:102A60008C179D0718F48081918102C08C1B9D0BEF
:102A700040815181628173818C0120E030E0041734
:102A800015072607370708F4CA01ECE981349E07C9
:102A900028F4FEE481329F0748F002C080E49CE9FC
:102AA000969587959695879524E007C027E2813112
:102AB000920730F09695879522E02093B50408C0E0
:102AC00021E02093B5048032910510F480E290E07B
:102AD000BC016052704088E060307807E0F0272F3A
:102AE00030E0220F331F220F331F205B3E4FF901CE
:102AF000329685919491AA27699FE001689FC10D44
:102B0000DA1F0694CA1FDA1F1124F9014591549166
:102B10004C1B5D0B1FC0CB01969587958C7F805B0E
:102B20009A4FFC01459154910296FC01A591B491F4
:102B3000862F90E087709070A89F9001A99F300D1C
:102B4000B89F300D1124E3E036952795EA95E1F71B
:102B5000421B530B44365105A0F4E0E0F2E006C0FE
:102B60009091C00095FFFCCF8093C600819188238F
:102B7000B9F78FE59AE04AE050E00E94508044E6C1
:102B800050E0509389004093880060E070E08091AD
:102B9000B1049091B204A091B304B091B404840F35
:102BA000951FA61FB71F8093B1049093B204A09302
:102BB000B304B093B40408C08091B6049091B704F4
:102BC00090938900809388004091AB045091AC04AD
:102BD0006091AD047091AE04E091AF04F091B00447
:102BE00080899189A289B389481759076A077B07A9
:102BF00080F01092B0041092AF049091E60A809198
:102C0000E50A981731F08091E50A8F5F8F70809305
:102C1000E50AFF91EF91DF91CF91BF91AF919F9125
:102C20008F917F916F915F914F913F912F911F9164
:102C30000F910F900BBE0F900FBE0F901F90189525
:102C4000099A3C9A9A9AEAE0F1E080818061808357
:102C50008081846080830D9A159A0F9A179A3A9A08
:102C6000429A989AA09A8081826080839FB7F89454
:102C7000ABE0B1E08C9182608C939FBF0898109A72
:102C80000C98149A3F98479A0A98129A0E98169A96
:102C90003D98459A0B9A159A3E9A179A389A429AF5
:102CA000808180648083A09A8081816080839FB7C7
:102CB000F8948C9182608C939FBFA1E8B0E08C91D6
:102CC0008F7E8C938C9188608C93E0E8F0E080811B
:102CD0008D7F808380818E7F808380818F738083CE
:102CE00080818F7C80838C91887F82608C9380E050
:102CF00090E4909389008093880010928500109250
:102D00008400EFE6F0E080818260808381E0809340
:102D10000704789408959091E60A8091E50A98173F
:102D200041F00E94BE7581E00E942A2D0E94DA5E69
:102D3000F2CF0895CF93DF93EFB7F894EC01888139
:102D40009981AA81BB8180938C0490938D04A09378
:102D50008E04B0938F04EB0188819981AA81BB8195
:102D60008093900490939104A0939204B093930461
:102D7000EA0188819981AA81BB8180939404909310
:102D80009504A0939604B0939704E90188819981F2
:102D9000AA81BB818093980490939904A0939A048C
:102DA000B0939B04EFBFDF91CF9108952FB7F894B4
:102DB000FC0180819181A281B381809398049093DA
:102DC0009904A0939A04B0939B042FBF08950F9386
:102DD0001F939FB7F894E82FF0E0EE0FFF1FEE0F60
:102DE000FF1FE457FB4F00811181228133819FBF78
:102DF000B801C9011F910F9108950E948B1680E5BB
:102E000099E00E94A42C159A179A429AA09A0895C4
:102E100080916F008D7F80936F0006C08091E50ADE
:102E20008F5F8F708093E50A9091E60A8091E50AA2
:102E3000981751F41092B0041092AF0480916F0073
:102E4000826080936F0008959091E60A8091E50A70
:102E5000981751F3E3CFCF93DF93EC019C012C5FE4
:102E60003F4F898D9A8D41E050E060E070E00E9414
:102E70003E228823A1F08D899E89AF89B88D009765
:102E8000A105B10571F48C819D81AE81BF818D8BCF
:102E90009E8BAF8BB88F89818068898302C080E068
:102EA00001C081E0DF91CF910895CF92DF92EF9240
:102EB000FF920F931F93CF938C01FC01818992891C
:102EC000A389B489803EFFEF9F07FFE1AF07F0E0E1
:102ED000BF0708F079C0C8010E942B17882309F4A6
:102EE00073C00E943E20882309F46EC0D801599611
:102EF000ED91FC915A971496CD90DD90ED90FC9059
:102F000017978EEF9FEFAFEFBFEFC80ED91EEA1EE7
:102F1000FB1E058404C0CC0CDD1CEE1CFF1C0A94B7
:102F2000D2F786859785A089B189C80ED91EEA1E79
:102F3000FB1E81E08093DB04C092DE06D092DF06A8
:102F4000E092E006F092E10680E092E0EEEDF4E03F
:102F5000DF019C011D9221503040E1F7C1E011C01A
:102F6000B701A6014C0F511D611D711D8091DC043C
:102F70009091DD042EED34E00E940B0E882321F1A8
:102F8000CF5FD8015996ED91FC915A978481C8176B
:102F900038F380E092E0A0E0B0E0058404C0880F40
:102FA000991FAA1FBB1F0A94D2F7F80141895289C1
:102FB00063897489480F591F6A1F7B1F418B528B8D
:102FC000638B748B81E001C080E0CF911F910F91E2
:102FD000FF90EF90DF90CF900895CF93DF93EC01B7
:102FE0008C859D85AE85BF8541E0662309F440E070
:102FF000BC01CD010E947B20882351F0888990E09C
:1030000025E0880F991F2A95E1F782529B4F02C055
:1030100080E090E0DF91CF910895FC0190E080E0A6
:103020002EE23081303269F0983029F4DB01A80FAC
:10303000B11D2C938F5F3081DB01A80FB11D3C9334
:103040008F5F9F5F31969B3061F7680F711DFB01A9
:1030500010820895CF93DF93EB01FC01238122239B
:1030600089F02250223020F48FE28883198208C030
:1030700060E00E94ED17009729F0BE010E940D1834
:1030800081E001C080E0DF91CF910895CF93DF937D
:10309000EA01FB012BE030E231932150E9F7DC013A
:1030A00030E047E01CC04A3069F138E04AE017C020
:1030B000E21741F1FC010196E491EE23C9F74317B1
:1030C00008F12132F8F02F37E8F4FB01E30FF11D8E
:1030D000822F81568A3108F4205220833F5F9A2F35
:1030E0008B2F2D91222339F02F3229F02E32D9F255
:1030F0008AE599E0DFCF9883898381E0FB019081A5
:10310000903209F480E0DF91CF9108950F931F93DF
:10311000CF93DF93EC018B018B81882309F040C0B2
:10312000FB018789803109F041C082E08B831D8AD1
:103130001E8A1F8A188E808D918DA0E0B0E035E048
:10314000880F991FAA1FBB1F3A95D1F7898B9A8BBD
:10315000AB8BBC8B13C083E08B83F801428D538D06
:10316000648D758D4D8B5E8B6F8B788F9E012F5E7E
:103170003F4FC8010E943821882391F01A8F098F90
:1031800081E089831C821D821E821F821886198617
:103190001A861B861C861D861E861F86188A01C0FD
:1031A00080E0DF91CF911F910F9108958032C1F798
:1031B000D2CF2F923F924F925F926F927F928F92D7
:1031C0009F92AF92BF92CF92DF92EF92FF920F93B6
:1031D0001F93CF93DF9300D000D0CDB7DEB79C8391
:1031E0008B83662E272E2A01DC0113968C91139770
:1031F000882309F4D2C011968C91119780FFCDC01D
:10320000E7C02A01481A590A5201862C922CEB81F8
:10321000FC813496FA83E983212C02E0302EB7C07A
:10322000EB81FC8180859185A285B3857FEF672E38
:1032300071E0772E6822792223816C017D0119E0EB
:10324000F694E794D794C7941A95D1F7418D528D8F
:103250005E834D83223061F4DA015A964D915D917F
:103260006D917C915D974C0D5D1D6E1D7F1D4EC057
:10327000ED81FE81048101500C216114710411F56E
:10328000002301F50097A105B10559F4EB81FC81FC
:1032900085899689A789B08D84839583A683B78312
:1032A00011C0AB81BC8114964D915D916D917C9163
:1032B00017978D819E8129813A810E94B5208823AC
:1032C00009F46BC0AB81BC815996ED91FC915A9782
:1032D00014964D915D916D917C911797425050409D
:1032E00060407040058404C0440F551F661F771F5F
:1032F0000A94D2F786859785A089B189480F591F0E
:103300006A1F7B1F400F511D611D711DC101861970
:10331000970985018A159B0508F48C01B2E00030FD
:103320001B0709F073C08091DE069091DF06A09123
:10333000E006B091E106481759076A077B0709F4D0
:1033400065C08091DC049091DD0494010E94DF0C43
:10335000882341F422C0B30162527B4FC401A8010B
:103360000E9448AE800E911EA80160E070E0EB81E3
:10337000FC8180859185A285B385840F951FA61F4A
:10338000B71F80879187A287B387A01AB10AA114BB
:10339000B10409F045CFC20102C08FEF9FEF26961E
:1033A0000FB6F894DEBF0FBECDBFDF91CF911F9156
:1033B0000F91FF90EF90DF90CF90BF90AF909F90D4
:1033C0008F907F906F905F904F903F902F900895D7
:1033D000AB81BC8151964D915D916D917C915497DB
:1033E00018968D919D910D90BC91A02D820120E0A9
:1033F00030E06A017B01C81AD90AEA0AFB0A0C15F7
:103400001D052E053F0508F0FCCEFECECB01BA010E
:1034100040E00E947B20882309F09DCFBECFCF9350
:10342000DF930F92CDB7DEB7BE016F5F7F4F41E0F4
:1034300050E00E94D9188130910519F4898190E0FB
:1034400002C08FEF9FEF0F90DF91CF9108950F9300
:103450001F93CF93DF938C01EB01FC0183818230BA
:1034600020F180859185A285B3858F719070A070C1
:10347000B0700097A105B105C1F4C801BE0140E2DA
:1034800050E00E94D9188032910519F0009769F434
:103490000EC08881882359F0853E79F38E3269F316
:1034A0008B8583FDEACF80E203C08FEF01C080E00F
:1034B000DF91CF911F910F910895CF92DF92EF92FC
:1034C000FF92CF93DF93EC018B81823038F1C88477
:1034D000D984EA84FB84CE010E940F1A97FD1EC096
:1034E00088859985AA85BB854F96A11DB11D8887C2
:1034F0009987AA87BB87D701C60125E0B695A7950E
:10350000979587952A95D1F78F7090E035E0880FD1
:10351000991F3A95E1F782529B4F02C080E090E0FC
:10352000DF91CF91FF90EF90DF90CF9008958F9231
:103530009F92AF92BF92CF92DF92EF92FF920F9342
:103540001F93CF93DF93EC014A015B012B81222370
:1035500009F475C089899A89AB89BC898417950754
:10356000A607B70708F46BC078C081149104A104C2
:10357000B10449F41C821D821E821F82188619869E
:103580001A861B865AC0488559856A857B85E98DD0
:10359000FA8D258530E0275F3F4FDB01CA01019797
:1035A000A109B109022E04C0B695A79597958795F4
:1035B0000A94D2F7750164010894C108D108E108A2
:1035C000F10804C0F694E794D794C7942A95D2F7EB
:1035D000C816D906EA06FB0628F041155105610513
:1035E000710549F48D899E89AF89B88D8C839D833F
:1035F000AE83BF8316C0C81AD90AEA0AFB0A11C0F3
:103600004C815D816E817F81898D9A8D98010E94A8
:10361000B5200894C108D108E108F108882321F4F5
:103620000EC08E010C5F1F4FC114D104E104F104E0
:1036300039F788869986AA86BB8681E001C080E03A
:10364000DF91CF911F910F91FF90EF90DF90CF907E
:10365000BF90AF909F908F900895223009F085CF52
:10366000E8CF40E050E060E070E00E94971A0895D3
:103670000F931F93CF93DF938C01FC0183818823E9
:10368000C9F1818187FF33C0C80161E00E94ED1755
:10369000EC01009779F18881853E61F1F801838121
:1036A000823040F481899289A389B4898C8F9D8F5F
:1036B000AE8FBF8FF80185899689A789B08D9B8FC2
:1036C0008A8FBD8BAC8BE091D504F091D6043097F6
:1036D00051F0BE016A5E7F4FCE0148961995888DE4
:1036E000998D9B8B8A8BF80181818F7781830E94D2
:1036F0003E2004C081E0F801808380E0DF91CF911B
:103700001F910F910895CF93DF93EC010E94381B16
:103710001B82DF91CF910895CF93DF93EC018B81D2
:10372000882321F0CE010E94381B1B82DF91CF91AC
:1037300008954F925F926F927F928F929F92AF9275
:10374000BF92EF92FF920F931F93CF93DF9300D01E
:103750000F92CDB7DEB77C014A015B01FC0183818A
:10376000813009F085C0818181FF82C095C00097BA
:10377000A105B10509F47AC0F7014084518462843F
:103780007384C701B501A4010E94971A882309F424
:103790006FC0F701818D928D81149104A104B10451
:1037A00079F4458956896789708D0E944F23882353
:1037B00009F45EC0F701158A168A178A108E3CC07C
:1037C000F70144815581668177819E012F5F3F4FCC
:1037D0000E94B520882309F44BC0F701818D928D9A
:1037E00049815A816B817C81FC012789203149F410
:1037F000483FFFEF5F07F0E06F07F0E07F07E0F47E
:1038000008C0483F2FEF52072FEF62072FE07207E3
:1038100098F40E944F23882359F1F7014481558180
:1038200066817781818D928D0FEF1FEF2FEF3FE043
:103830000E94A6218823E1F0F701818A928AA38A57
:10384000B48A818180688183C7010E94381B8823E4
:1038500079F0B501A401481459046A047B0410F4FA
:10386000B301A201C7010E94971A03C081E001C001
:1038700080E00F900F900F900F90DF91CF911F91EC
:103880000F91FF90EF90BF90AF909F908F907F909F
:103890006F905F904F900895F70181899289A38975
:1038A000B48984179507A607B70708F060CFE0CF63
:1038B000CF93DF93EC0140E050E060E070E00E94C5
:1038C000991B882369F0CE0161E00E94ED170097F3
:1038D00039F025EEFC0120831B820E943E2001C0AE
:1038E00080E0DF91CF9108951F93CF93DF93EC0198
:1038F000142FE62FF0E035E0EE0FFF1F3A95E1F7C9
:10390000E252FB4F8385817121F0842F827109F08F
:103910005DC08091DE069091DF06A091E006B09137
:10392000E1068C879D87AE87BF87688B4489558960
:1039300060E070E0BA0155274427828D938DA0E0A6
:10394000B0E0482B592B6A2B7B2B4D8B5E8B6F8BFA
:10395000788F838590E088719070009751F4848D02
:10396000958DA68DB78D898B9A8BAB8BBC8B81E0A7
:103970000DC08031910551F59E012F5E3F4F898D1D
:103980009A8D0E943821882309F184E08B83812F4E
:103990008F7089831C821D821E821F821886198661
:1039A0001A861B8614FF18C0CE0140E050E060E08C
:1039B00070E00E94991B882351F00EC049895A89F2
:1039C0006B897C89CE010E94971A02C01B8280E01D
:1039D000DF91CF911F91089515FDF0CF81E0F8CFD1
:1039E0007F928F929F92AF92BF92CF92DF92EF928F
:1039F000FF920F931F93CF93DF935C01EB01942E03
:103A0000852E722E898D9A8DF501928F818FCB0133
:103A10000E94311B10E037C0CE010E945D1ABC012C
:103A2000009709F490C0D701C60135E0B695A79577
:103A3000979587953A95D1F7082F0F70FB018081F4
:103A4000882311F0853EB1F4112379F48091DE06CC
:103A50009091DF06A091E006B091E106F501848720
:103A60009587A687B787008B11E0FB0180818823AB
:103A700051F417C0892D982D4BE050E00E943BAEC9
:103A8000009709F46FC0C884D984EA84FB848989CB
:103A90009A89AB89BC89C816D906EA06FB0608F4E0
:103AA000BBCF76FE50C071FE4EC0112351F0F50120
:103AB0000089C50161E00E94ED17EC01009769F4EF
:103AC00042C08B81823009F43EC0CE010E9455175E
:103AD0008823C9F1CEEDD4E000E080E2FE0111922E
:103AE0008A95E9F7FE01A92DB82D8BE00D90019282
:103AF0008150E1F7E091D504F091D604309739F088
:103B0000BE01625F7F4FCE014096199508C081E2E9
:103B100098E2998B888B80E098E09F878E878889D0
:103B200099899B8B8A8B998F888F8E859F859F8B98
:103B30008E8B0E943E20882331F0C501602F472DD7
:103B40000E94741C01C080E0DF91CF911F910F9102
:103B5000FF90EF90DF90CF90BF90AF909F908F90AD
:103B60007F90089577FEE9CFEECF5F926F927F92BC
:103B70008F929F92AF92BF92CF92DF92EF92FF927D
:103B80000F931F93CF93DF93CDB7DEB7C354D040CD
:103B90000FB6F894DEBF0FBECDBF4C016B0124966B
:103BA0005FAF4EAF2497522E1FA21AA61C861F8607
:103BB0006115710509F47AC0FC018381882309F03D
:103BC00075C0FA0180818F3291F405C03196249638
:103BD000FFAFEEAF24972496EEADFFAD2497808122
:103BE0008F32A1F3F60183818250823050F4860136
:103BF00057E2E52EF12CEC0EFD1E3701BE2CAF2C4A
:103C000011C0F601618D728DCE010C960E9486184E
:103C1000882309F44BC08E01045F1F4FE9CF870151
:103C2000EB2CFA2C24968EAD9FAD2497BE016F5FCE
:103C30007F4FAE014E5B5F4F0E944618882331F4E0
:103C400035C031962496FFAFEEAF24972496EEADA3
:103C5000FFAD249780818F32A1F38823E9F0C7015B
:103C6000B801AE014F5F5F4F21E00E94F01C882336
:103C7000E9F00C151D0529F0C8010E94381BF80158
:103C80001382E614F70459F64CE0E42EF12CEC0E06
:103C9000FD1E0B2D1A2DC6CFC401B801AE014F5F1A
:103CA0005F4F252D0E94F01C082F01C000E0CE01BF
:103CB0000C960E948C1BCE0187960E948C1B802F35
:103CC000CD5BDF4F0FB6F894DEBF0FBECDBFDF91E7
:103CD000CF911F910F91FF90EF90DF90CF90BF9009
:103CE000AF909F908F907F906F905F9008951F93FB
:103CF000CF93DF93CDB7DEB76B970FB6F894DEBFE7
:103D00000FBECDBF9C01AB0119821C82CE01019672
:103D1000B90122E00E94B51D882331F0CE01019641
:103D20000E94581C182F01C010E0CE0101960E947D
:103D30008C1B812F6B960FB6F894DEBF0FBECDBFE4
:103D4000DF91CF911F9108952F923F924F925F92F2
:103D50006F927F928F929F92BF92CF92DF92EF925B
:103D6000FF920F931F93CF93DF9300D000D0CDB776
:103D7000DEB78C01B62EC72E5E834D83DC01139611
:103D80008C911397813009F059C111968C9111973C
:103D900081FF54C170C1F8014189528963897489D6
:103DA00080859185A285B38584179507A607B707F7
:103DB00031F0C8010E94971A882309F43FC14D8051
:103DC0005E802B2C3C2C07C1F801218D328DF9012E
:103DD000B480BA94AC01BD01032E39E076956795A5
:103DE000579547953A95D1F7302DB4224FEF642E71
:103DF00041E0742E68227922BB2009F04BC0611487
:103E0000710409F047C0D80114964D915D916D91F0
:103E10007C911797411551056105710559F4559627
:103E20008D919D910D90BC91A02D0097A105B1059C
:103E300061F525C0C9019E012F5F3F4F0E94B5204B
:103E4000882309F4FBC089819A81AB81BC81F80188
:103E5000218D328DF9012789203149F4883FFFEF08
:103E60009F07F0E0AF07F0E0BF0748F40EC0883FBF
:103E70002FEF92072FEFA2072FE0B20730F0C80113
:103E80000E942B17882331F4D9C0F80184839583CD
:103E9000A683B78380E092E08619970942018415D2
:103EA000950508F44C01D8015996ED91FC915A976B
:103EB0001496CD90DD90ED90FC9017978EEF9FEFCC
:103EC000AFEFBFEFC80ED91EEA1EFB1E058404C06B
:103ED000CC0CDD1CEE1CFF1C0A94D2F7868597855E
:103EE000A089B189C80ED91EEA1EFB1ECB0CD11CBD
:103EF000E11CF11C90E0891692E0990639F5809159
:103F0000DE069091DF06A091E006B091E1068C15E7
:103F10009D05AE05BF0571F41092DB048FEF9FEF96
:103F2000AFEFBFEF8093DE069093DF06A093E0062D
:103F3000B093E1068091DC049091DD04B701A60105
:103F400091010E940B0E882391F578C061147104D1
:103F5000F9F4F80180859185A285B385418952895C
:103F60006389748984179507A607B70788F00E94AC
:103F70003E20882309F462C081E08093DB04C09274
:103F8000DE06D092DF06E092E006F092E10608C07D
:103F9000C701B60141E00E947B20882309F44EC08E
:103FA000C30182529B4FB101A4010E9448AEA401FB
:103FB00060E070E0F80180859185A285B385840F6B
:103FC000951FA61FB71F80879187A287B387280CEC
:103FD000391C48185908F80180859185A285B38558
:103FE0004114510409F0F0CE4189528963897489E2
:103FF000481759076A077B0740F4818B928BA38B84
:10400000B48B8181806881830DC08091D5049091AB
:10401000D604009739F08D819E81009719F0818137
:1040200080688183F801818183FF05C0C8010E94F7
:10403000381B882319F08D819E8105C081E0D8014D
:104040008C938FEF9FEF26960FB6F894DEBF0FBECE
:10405000CDBFDF91CF911F910F91FF90EF90DF9037
:10406000CF90BF909F908F907F906F905F904F9078
:104070003F902F90089582FD8ECEA1CE8091DB04DB
:10408000882399F14091DE065091DF066091E006A9
:104090007091E1068091DC049091DD042EED34E016
:1040A0000E940B0E882319F14091D7045091D80437
:1040B0006091D9047091DA044115510561057105CB
:1040C00091F08091DC049091DD042EED34E00E94AB
:1040D0000B0E882371F01092D7041092D80410921E
:1040E000D9041092DA041092DB0481E0089580E094
:1040F000089580E00895CF92DF92EF92FF92CF93E0
:104100006B017C01C42F8091DE069091DF06A091A7
:10411000E006B091E1068C159D05AE05BF05C1F026
:104120000E943E208823D1F08091DC049091DD0430
:10413000B701A6012EED34E00E94DF0C882371F058
:10414000C092DE06D092DF06E092E006F092E10631
:1041500081E0CC2321F08093DB0401C080E0CF918B
:10416000FF90EF90DF90CF900895CF92DF92EF9283
:10417000FF920F931F93CF93DF93EC016A017B01B2
:10418000890189859A85AB85BC850196A11DB11DE4
:1041900084179507A607B70708F460C08F89803198
:1041A00029F4BB27AF2D9E2D8D2D0CC0803209F038
:1041B00055C0DB01CA0147E0B695A795979587954D
:1041C0004A95D1F74B895C896D897E89840F951F4B
:1041D000A61FB71F4091DE065091DF066091E006F2
:1041E0007091E10684179507A607B70739F0BC015F
:1041F000CD0140E00E947B20882381F18F898031AE
:1042000091F48FEF90E0A0E0B0E0C822D922EA223A
:10421000FB22F601EE0FFF1FE252FB4F80819181DE
:10422000A0E0B0E014C08FE790E0A0E0B0E0C822CA
:10423000D922EA22FB22F601EE0FFF1FEE0FFF1F2D
:10424000E252FB4F80819181A281B381BF70F8015E
:1042500080839183A283B38381E001C080E0DF91FA
:10426000CF911F910F91FF90EF90DF90CF90089525
:104270006F927F928F929F92AF92BF92CF92DF9276
:10428000EF92FF920F931F93CF93DF9300D00F9283
:10429000CDB7DEB78C0149835A836B837C833901A8
:1042A000CC24DD247601812CE2E09E2EA12CB12CC1
:1042B00049815A816B817C81C8019E012F5F3F4FEC
:1042C0000E94B520882371F1D501C401F80105844D
:1042D00004C0880F991FAA1FBB1F0A94D2F7C80EEB
:1042E000D91EEA1EFB1E89819A81AB81BC81278978
:1042F000203149F4883FFFEF9F07F0E0AF07F0E07F
:10430000BF0748F4D5CF883F2FEF92072FEFA207C2
:104310002FE0B20768F2F301C082D182E282F38219
:1043200081E001C080E00F900F900F900F90DF911F
:10433000CF911F910F91FF90EF90DF90CF90BF90A2
:10434000AF909F908F907F906F9008954F925F9263
:104350006F927F928F929F92AF92BF92CF92DF9295
:10436000EF92FF920F931F93CF93DF93EC014A01DB
:104370005B0128013901423051056105710508F4DE
:104380006BC089859A85AB85BC850196A11DB11D41
:1043900084179507A607B70708F45EC08F89803198
:1043A00029F4C52ED62EE72EFF240CC0803209F04A
:1043B00053C06A017B0187E0F694E794D794C794D1
:1043C0008A95D1F78B899C89AD89BE89C80ED91E83
:1043D000EA1EFB1EC701B60141E00E947B20882334
:1043E000D9F18F89803181F48FEF90E0A0E0B0E0C7
:1043F00088229922AA22BB22F401EE0FFF1FE2526B
:10440000FB4F5182408213C08FE790E0A0E0B0E004
:1044100088229922AA22BB22F401EE0FFF1FEE0F81
:10442000FF1FE252FB4F40825182628273828A896F
:10443000823080F08D819E81AF81B8858C0D9D1D6D
:10444000AE1DBF1D8093D7049093D804A093D904C8
:10445000B093DA0481E001C080E0DF91CF911F9139
:104460000F91FF90EF90DF90CF90BF90AF909F9013
:104470008F907F906F905F904F9008952F923F9212
:104480004F925F926F927F928F929F92AF92BF9264
:10449000CF92DF92EF92FF920F931F93CF93DF9310
:1044A000CDB7DEB72F970FB6F894DEBF0FBECDBFE6
:1044B0001C014C875D876E877F873B872A87DC01DD
:1044C00019962D913D914D915C911C972F5F3F4F17
:1044D0004F4F5F4F2E833F8348875987EA85FB857F
:1044E00040805180628073804114510461047104E2
:1044F00031F00894411C511C611C711C10C0DC017E
:104500004D905D906D907C90B1E0BD832C853D8594
:104510004E855F85213031054105510509F01D8229
:1045200053014201CC24DD247601F101818592857D
:10453000A385B485C816D906EA06FB0608F093C021
:104540002E813F8148855985281539054A055B0527
:1045500050F422E0822E912CA12CB12C32E0432E7B
:10456000512C612C712CC101B501A4019E012F5F5A
:104570003F4F0E94B520882309F475C049815A81B4
:104580006B817C81D501C4010196A11DB11D41152E
:1045900051056105710519F02C013D010DC084190B
:1045A0009509A609B7092C853D854E855F8582173B
:1045B0009307A407B50759F00894C11CD11CE11C4E
:1045C000F11C0894811C911CA11CB11CAECFC1012F
:1045D000A401B5010FEF1FEF2FEF3FE00E94A621CE
:1045E000882391F440C0680179010894C108D1087A
:1045F000E108F108C101B701A6010E94A6218823A4
:1046000091F19701860102C095018401401651067F
:104610006206730640F3AA85BB854D915D916D914D
:104620007C911397411551056105710539F0C10160
:10463000930182010E94A6218823A9F0EA85FB85C7
:104640004082518262827382FD81FF2371F008945F
:10465000411C511C611C711CD1014D925D926D92E7
:104660007C92139702C080E001C081E02F960FB6C4
:10467000F894DEBF0FBECDBFDF91CF911F910F9198
:10468000FF90EF90DF90CF90BF90AF909F908F9072
:104690007F906F905F904F903F902F900895AF92D2
:1046A000BF92CF92DF92EF92FF920F931F93CF931F
:1046B000DF9300D00F92CDB7DEB75C016A017B01BA
:1046C00082E090E0A0E0B0E0F50180839183A283D6
:1046D000B383C501B701A6019E012F5F3F4F0E9422
:1046E000B520882341F1C501B701A60100E010E023
:1046F00020E030E00E94A6218823E9F0C980DA801A
:10470000EB80FC80F5018789803151F4F8EFCF16FA
:10471000FFEFDF06F0E0EF06F0E0FF0650F4D9CF40
:1047200088EFC8168FEFD8068FEFE8068FE0F806FF
:1047300080F281E001C080E00F900F900F900F9009
:10474000DF91CF911F910F91FF90EF90DF90CF906D
:10475000BF90AF9008956F927F928F929F92AF9289
:10476000BF92CF92DF92EF92FF921F93CF93DF938E
:10477000EC01142F7093DD046093DC041F8A82E047
:1047800090E0A0E0B0E088839983AA83BB83109275
:10479000DB041092D7041092D8041092D90410921E
:1047A000DA048FEF9FEFAFEFBFEF8093DE069093B9
:1047B000DF06A093E006B093E106442389F145307B
:1047C00008F008C160E070E080E090E040E00E9406
:1047D0007B20882309F4FEC0E12FF0E0A4E0EE0F77
:1047E000FF1FAA95E1F7E457F94F808190E08F779A
:1047F0009070009709F0EEC084859585A685B785F1
:1048000084369105A105B10508F4E4C08084918443
:10481000A284B38481149104A104B10421F4DAC008
:10482000882499245401C501B40140E00E947B20F2
:10483000882309F4CFC08091E9049091EA0422E032
:104840008030920709F0C6C03091EE04332309F49A
:10485000C1C08091EC049091ED04009709F4BAC0B6
:104860002091EB04222309F4B5C03A8B2C831D86DA
:1048700030E041E050E006C0812F8F5F8D87183017
:1048800008F0A8C01D85CA01012E02C0880F991F1B
:104890000A94E2F72817390779F78091F404909188
:1048A000F504009719F0A0E0B0E008C0809102057F
:1048B00090910305A0910405B09105058D839E8319
:1048C000AF83B8872091EC043091ED046901EE24A8
:1048D000FF24C80CD91CEA1CFB1CCB8ADC8AED8A9D
:1048E000FE8A6090EF047090F004798E688E2091BB
:1048F000EE0430E040E050E0BC01CD010E94CEAAC1
:10490000DC01CB018C0D9D1DAE1DBF1D8A8F9B8FC1
:10491000AC8FBD8FA301E5E0440F551FEA95E1F789
:1049200041505E4F452F5527469560E070E0480F97
:10493000591F6A1F7B1F4E875F87688B798B809119
:10494000F1049091F204009719F0A0E0B0E008C0E3
:104950008091FE049091FF04A0910005B0910105A3
:10496000841A950AA60AB70A880E991EAA1EBB1EAB
:1049700004C0B694A794979487941A95D2F7898621
:104980009A86AB86BC8685EF88168FE0980680E015
:10499000A80680E0B80618F48CE08F8B1BC025EFCA
:1049A00082162FEF920620E0A20620E0B20610F455
:1049B00080E10DC080910A0590910B05A0910C0536
:1049C000B0910D058A8F9B8FAC8FBD8F80E28F8B4E
:1049D00081E001C080E0DF91CF911F91FF90EF90C7
:1049E000DF90CF90BF90AF909F908F907F906F900F
:1049F0000895CF93DF930F92CDB7DEB76983049606
:104A0000BE016F5F7F4F41E050E00E94A41E0F90F7
:104A1000DF91CF910895DB010D900020E9F7AD0102
:104A200041505040461B570B04960E94A41E089507
:104A3000CF93DF93CAE6D9E0FE0107C09091C00092
:104A400095FFFCCF8093C600319684918823B1F7FF
:104A5000EDE9FAE007C09091C00095FFFCCF80938C
:104A6000C600319684918823B1F78091C00085FFFC
:104A7000FCCF8AE08093C600FE018491EAE6F9E06B
:104A800008C09091C00095FFFCCF8093C60031967E
:104A900084918823B1F7EDEAFAE007C09091C00055
:104AA00095FFFCCF8093C600319684918823B1F79F
:104AB0004091031050910410609105107091061000
:104AC0008FE59AE022E030E00E942B81E5EBFAE0EE
:104AD00007C09091C00095FFFCCF8093C60031962F
:104AE00084918823B1F7409107105091081060918C
:104AF000091070910A108FE59AE022E030E00E94E0
:104B00002B81E8EBFAE007C09091C00095FFFCCF45
:104B10008093C600319684918823B1F740910B10A1
:104B200050910C1060910D1070910E108FE59AE06D
:104B300022E030E00E942B81EBEBFAE007C090917D
:104B4000C00095FFFCCF8093C600319684918823E6
:104B5000B1F740910F1050911010609111107091A9
:104B600012108FE59AE022E030E00E942B818091C4
:104B7000C00085FFFCCF8AE08093C600FE018491CF
:104B8000EAE6F9E008C09091C00095FFFCCF809361
:104B9000C600319684918823B1F7EEEBFAE007C0A6
:104BA0009091C00095FFFCCF8093C6003196849110
:104BB0008823B1F78091C00085FFFCCF8AE0809305
:104BC000C600FE018491EAE6F9E008C09091C000B9
:104BD00095FFFCCF8093C600319684918823B1F76E
:104BE000E8EDFAE007C09091C00095FFFCCF8093FC
:104BF000C600319684918823B1F7409113105091EB
:104C0000141060911510709116108FE59AE022E053
:104C100030E00E942B81E1EEFAE007C09091C000E5
:104C200095FFFCCF8093C600319684918823B1F71D
:104C300040911710509118106091191070911A102E
:104C40008FE59AE022E030E00E942B81E4EEFAE06A
:104C500007C09091C00095FFFCCF8093C6003196AD
:104C600084918823B1F740911B1050911C106091E2
:104C70001D1070911E108FE59AE022E030E00E9436
:104C80002B81E7EEFAE007C09091C00095FFFCCFC2
:104C90008093C600319684918823B1F740911F100C
:104CA0005091201060912110709122108FE59AE0B0
:104CB00022E030E00E942B818091C00085FFFCCF74
:104CC0008AE08093C600FE018491EAE6F9E008C01C
:104CD0009091C00095FFFCCF8093C60031968491DF
:104CE0008823B1F7EAEEFAE007C09091C00095FF83
:104CF000FCCF8093C600319684918823B1F78091D0
:104D0000C00085FFFCCF8AE08093C600FE0184913D
:104D1000EAE6F9E008C09091C00095FFFCCF8093CF
:104D2000C600319684918823B1F7E8E0FBE007C024
:104D30009091C00095FFFCCF8093C600319684917E
:104D40008823B1F74091F30F5091F40F6091F50F64
:104D50007091F60F8FE59AE02AE030E00E94E57F3F
:104D6000E1E1FBE007C09091C00095FFFCCF80938C
:104D7000C600319684918823B1F74091F70F509186
:104D8000F80F6091F90F7091FA0F8FE59AE02AE021
:104D900030E00E94E57FE4E1FBE007C09091C000B5
:104DA00095FFFCCF8093C600319684918823B1F79C
:104DB0004091FB0F5091FC0F6091FD0F7091FE0F21
:104DC0008FE59AE02AE030E00E94E57FE7E1FBE032
:104DD00007C09091C00095FFFCCF8093C60031962C
:104DE00084918823B1F74091FF0F5091001060919A
:104DF0000110709102108FE59AE02AE030E00E94E5
:104E0000E57F8091C00085FFFCCF8AE08093C600DB
:104E1000FE018491EAE6F9E008C09091C00095FF98
:104E2000FCCF8093C600319684918823B1F7EAE1E4
:104E3000FBE007C09091C00095FFFCCF8093C600B7
:104E4000319684918823B1F78091C00085FFFCCF13
:104E50008AE08093C600FE018491EAE6F9E008C08A
:104E60009091C00095FFFCCF8093C600319684914D
:104E70008823B1F7EFE4FBE007C09091C00095FFF5
:104E8000FCCF8093C600319684918823B1F740917E
:104E9000EB0F5091EC0F6091ED0F7091EE0F8FE5DD
:104EA0009AE022E030E00E942B81E8E5FBE007C0B9
:104EB0009091C00095FFFCCF8093C60031968491FD
:104EC0008823B1F74091E70F5091E80F6091E90F07
:104ED0007091EA0F8FE59AE022E030E00E942B818A
:104EE0008091C00085FFFCCF8AE08093C600FE0160
:104EF0008491EAE6F9E008C09091C00095FFFCCFEC
:104F00008093C600319684918823B1F7EBE5FBE0EE
:104F100007C09091C00095FFFCCF8093C6003196EA
:104F200084918823B1F78091C00085FFFCCF8AE08F
:104F30008093C600FE018491EAE6F9E008C09091F2
:104F4000C00095FFFCCF8093C600319684918823E2
:104F5000B1F7E4EFFBE007C09091C00095FFFCCFF4
:104F60008093C600319684918823B1F74091EF0F6A
:104F70005091F00F6091F10F7091F20F8FE59AE070
:104F800022E030E00E942B81EDEFFBE007C0909122
:104F9000C00095FFFCCF8093C60031968491882392
:104FA000B1F74091D70F5091D80F6091D90F709100
:104FB000DA0F8FE59AE022E030E00E942B81E0E0FA
:104FC000FCE007C09091C00095FFFCCF8093C60025
:104FD000319684918823B1F7409123105091241089
:104FE00060912510709126108FE59AE02AE030E05C
:104FF0000E94E57FE3E0FCE007C09091C00095FFD0
:10500000FCCF8093C600319684918823B1F74091FC
:10501000E30F5091E40F6091E50F7091E60F8FE57B
:105020009AE022E030E00E942B81E6E0FCE007C03D
:105030009091C00095FFFCCF8093C600319684917B
:105040008823B1F74091DF0F5091E00F6091E10F9D
:105050007091E20F8FE59AE022E030E00E942B8110
:10506000E9E0FCE007C09091C00095FFFCCF809381
:10507000C600319684918823B1F74091DB0F50919F
:10508000DC0F6091DD0F7091DE0F8FE59AE022E07A
:1050900030E00E942B818091C00085FFFCCF8AE028
:1050A0008093C600FE018491EAE6F9E008C0909181
:1050B000C00095FFFCCF8093C60031968491882371
:1050C000B1F7ECE0FCE007C09091C00095FFFCCF89
:1050D0008093C600319684918823B1F78091C000F7
:1050E00085FFFCCF8AE08093C600FE01C491EAE60A
:1050F000F9E008C08091C00085FFFCCFC093C600D6
:105100003196C491CC23B1F7EAE1FCE007C090915D
:10511000C00095FFFCCF8093C60031968491882310
:10512000B1F7409136045091370460913804709182
:1051300039048FE59AE022E030E00E942B81E4E21E
:10514000FCE007C09091C00095FFFCCF8093C600A3
:10515000319684918823B1F76091320470913304C1
:1051600080913404909135042FE632E143E05EE310
:105170000E943AA7AB01BC018FE59AE022E030E043
:105180000E942B81E7E2FCE007C09091C00095FFF0
:10519000FCCF8093C600319684918823B1F760914B
:1051A0002E0470912F0480913004909131042FE6E9
:1051B00032E143E05EE30E9408AAAB01BC018FE547
:1051C0009AE022E030E00E942B818091C00085FFB0
:1051D000FCCF8AE08093C600DF91CF910895CF93F2
:1051E000DF930F920F92CDB7DEB78091541090915C
:1051F00055109E012F5F3F4F009719F42A553041FB
:1052000002C0281B390B3A83298389819A810F9028
:105210000F90DF91CF910895BC0180910808909183
:105220000908843091050CF06EC020910A08309175
:105230000B0840E650E0249FC001259F900D349F4D
:10524000900D1124845F974F0E9467AEEAE6F9E063
:1052500007C09091C00095FFFCCF8093C6003196A7
:1052600084918823B1F7E0E7F9E007C09091C0008E
:1052700095FFFCCF8093C600319684918823B1F7C7
:1052800020910A0830910B0880E690E0289FF001F9
:10529000299FF00D389FF00D1124E45FF74F06C0F1
:1052A0009091C00095FFFCCF8093C6008191882328
:1052B000B9F7EBE7F9E007C09091C00095FFFCCF8C
:1052C0008093C600319684918823B1F78091C00005
:1052D00085FFFCCF8AE08093C60080910A089091F8
:1052E0000B08019664E070E00E9401AB90930B08FC
:1052F00080930A088091080890910908019690937C
:105300000908809308080895809A889A0895809AD9
:10531000889808958091960990919709019660E088
:1053200070E00E9455AB462F572F682F792FCB0185
:10533000BA0108958091960990919709019660E0CD
:1053400070E04AE050E00E94D4AC0895682FE091EC
:105350009009F091910940E650E0E49F9001E59FAB
:10536000300DF49F300D1124C901845F974F70E018
:105370000E945CAE9C01909397098093960981E00E
:105380002115310509F480E008950E9425A3DC0170
:10539000CB018093A8099093A909A093AA09B0937F
:1053A000AB09E0919009F0919109E457F64F8081A3
:1053B0008823A1F4EDE3FFE007C09091C00095FFC2
:1053C000FCCF8093C600319684918823B1F78091F9
:1053D000C00085FFFCCF8AE08093C60008958FE56A
:1053E0009AE00E945E7FE5E3FFE007C09091C00075
:1053F00095FFFCCF8093C600319684918823B1F746
:1054000040919C0950919D0960919E0970919F095E
:105410004F5F5F4F6F4F7F4F8FE59AE02AE030E09C
:105420000E94FA7F8091C00085FFFCCF8AE08093C4
:10543000C6000E94C52908956F927F928F929F9215
:10544000AF92BF92CF92DF92EF92FF920F931F9392
:10545000CF9385E4682E84E0782E0DE017E090EB82
:10546000C92E99E0D92E20E2E22E27E0F22EC0E0EC
:10547000F30181913F010E94A629882309F10E942E
:105480008A294B015C01F7018081882319F460911E
:10549000C00901C061E070E080E090E00E94D5A703
:1054A000F80120813181428153810E9408AA9B0129
:1054B000AC01C501B4010E945AA6DC01CB0105C0B4
:1054C000F80180819181A281B381F601808391836B
:1054D000A283B383CF5F0C5F1F4F84E090E0C80EC0
:1054E000D91E0894E11CF11CC43011F686E40E9418
:1054F000A6298823E1F00E948A296B017C01609330
:10550000CA097093CB098093CC099093CD0920E010
:1055100030E040E050E00E9436A9181644F4C092F2
:105520001C04D0921D04E0921E04F0921F04CF913F
:105530001F910F91FF90EF90DF90CF90BF90AF90B1
:105540009F908F907F906F9008950E941C2A89E40D
:105550000E94A629882329F00E948A29DC01CB0118
:1055600004C080E090E0A0E0B0E08093CE0990938A
:10557000CF09A093D009B093D1098AE40E94A6294B
:10558000882329F00E948A29DC01CB0104C080E035
:1055900090E0A0E0B0E08093D2099093D309A0936B
:1055A000D409B093D50908958F929F92AF92BF927C
:1055B000CF92DF92EF92FF920F931F93CF93DF93DF
:1055C0000E9425A3DC01CB018093A8099093A9092F
:1055D000A093AA09B093AB0960910A0470910B04DF
:1055E000C0EBD9E034E0C32ED12CCC0EDD1E48E058
:1055F000A42EB12CAC0EBD1E5CE0852E912C8C0E21
:105600009D1E882777FD8095982F0E94D5A7209111
:105610001C0430911D0440911E0450911F040E94EF
:1056200008AA20E030E040E752E40E943AA720E0D8
:1056300030E048EC52E40E943AA77B018C01CE0195
:10564000B601A5019401E0E0CE2EE7E0DE2E0E9437
:105650000C948091B0099091B109A091B209B091D8
:10566000B30980930D0790930E07A0930F07B09393
:1056700010078091B4099091B509A091B609B09135
:10568000B7098093110790931207A0931307B09363
:1056900014078091B8099091B909A091BA09B09105
:1056A000BB098093150790931607A0931707B09333
:1056B00018078091BC099091BD09A091BE09B091D5
:1056C000BF098093190790931A07A0931B07B09303
:1056D0001C07DF91CF911F910F91FF90EF90DF900A
:1056E000CF90BF90AF909F908F9008954F925F9210
:1056F0006F927F92AF92BF92CF92DF92EF920F9311
:105700001F93CF93C82F6091CE097091CF098091DC
:10571000D0099091D1092091D2093091D3094091BB
:10572000D4095091D5090E9443A92B013C016091F5
:105730000A0470910B0400D000D00DB71EB70F5FA4
:105740001F4F882777FD8095982F0E94D5A720911D
:105750001C0430911D0440911E0450911F040E94AE
:1057600008AA20E030E040E752E40E943AA720E097
:1057700030E048EC52E40E943AA75B016C01F8016A
:105780004082518262827382C48380910007858344
:105790008DE097E060EB79E04EEC59E020E001E02D
:1057A000A2E0EA2E0E941A8B8091B0099091B10973
:1057B000A091B209B091B30980930D0790930E07A1
:1057C000A0930F07B09310078091B4099091B50989
:1057D000A091B609B091B709809311079093120771
:1057E000A0931307B09314078091B8099091B90959
:1057F000A091BA09B091BB09809315079093160741
:10580000A0931707B09318078091BC099091BD0928
:10581000A091BE09B091BF098093190790931A0710
:10582000A0931B07B0931C078DB79EB706960FB6C3
:10583000F8949EBF0FBE8DBF0E9425A3DC01CB0153
:105840008093A8099093A909A093AA09B093AB09E2
:10585000CF911F910F91EF90DF90CF90BF90AF90BD
:105860007F906F905F904F9008958091FE0608950D
:1058700067707070E82FF0E0E05FF94EE491EB3074
:1058800028F4E830A0F4E63090F106C0EE30D0F015
:10589000EF50E33060F521C08091B1008C7F8093A0
:1058A000B1008091B100862B8093B1000895809162
:1058B00091008C7F8093910080919100862B809342
:1058C000910008958091A1008C7F8093A100809128
:1058D000A100862B8093A1000895809121018C7FE7
:1058E0008093210180912101862B809321010895CD
:1058F000CF93DF93EC0105C082EE96E00E943CA4BA
:105900002196FE0164916623B9F7DF91CF91089546
:105910000F931F93CF93DF938C01CAEDD9E0CE0193
:10592000B80144E150E00E947CAEF80101900020F3
:10593000E9F73197E01BF10BEC0FFD1F1082DF91AF
:10594000CF911F910F910895FC01349120E0AAEDB1
:10595000B9E08A1B9B0B332349F0243139F03D9386
:105960002F5FFD01E80FF91F3491F5CF1C920895C8
:105970000E9445788091FE068823C1F581E08093DE
:10598000FE0680919C0990919D09A0919E09B0917D
:105990009F098093C6099093C709A093C809B09343
:1059A000C909EFE3FCE007C09091C00095FFFCCF70
:1059B0008093C600319684918823B1F7EAE6FFE030
:1059C00007C09091C00095FFFCCF8093C600319630
:1059D00084918823B1F78091C00085FFFCCF8AE0D5
:1059E0008093C60082EE9FE00E94A42C0895F89454
:1059F0000E944578159A179A429AA09A8CE060E026
:105A00000E9483A2EFE3FCE007C09091C00095FFE5
:105A1000FCCF8093C600319684918823B1F7E0E4EF
:105A2000FFE007C09091C00095FFFCCF8093C600B7
:105A3000319684918823B1F78091C00085FFFCCF17
:105A40008AE08093C60081E69FE00E94A42C0E9419
:105A50008729FFCF0F931F930E9425A3DC01CB0161
:105A60004091C2095091C3096091C4097091C50960
:105A70000091A8091091A9092091AA093091AB09B8
:105A8000801B910BA20BB30B481759076A077B07C2
:105A900038F4411551056105710511F00E94F72C8C
:105AA0008091210490912204A0912304B0912404B8
:105AB0000097A105B10539F10E9425A3DC01CB01B6
:105AC0004091A8095091A9096091AA097091AB0968
:105AD000841B950BA60BB70B409121045091220417
:105AE0006091230470912404481759076A077B07C3
:105AF00050F49091E60A8091E50A981721F4159ADE
:105B0000179A429AA09A0E94B5931F910F910895F7
:105B10002F923F924F925F926F927F928F929F92BD
:105B2000AF92BF92CF92DF92EF92FF920F931F93AB
:105B3000CF93DF93CDB7DEB76E970FB6F894DEBF85
:105B40000FBECDBF30E6632E712CEBEEFCE034903F
:105B50004AE0542EE8EEFCE044901CC28D3051F037
:105B60008A3321F490919309992321F04F355105FF
:105B70000CF4F1C14115510509F4F5C280910A08F0
:105B800090910B08869D7001879DF00C969DF00CFE
:105B900011244E0D5F1D445F574FFA011082209172
:105BA0009309222309F0D2C1109293098457964F8A
:105BB000FC0110828701045F174FC8016EE470E09A
:105BC0000E945CAE009709F410C1909397098093EE
:105BD0009609801B910B8E0D9F1D835F974F60E090
:105BE00070E04AE050E00E94D4ACDC01CB0180932D
:105BF000980990939909A0939A09B0939B09809072
:105C00009C0990909D09A0909E09B0909F09B501B4
:105C1000A4014F5F5F4F6F4F7F4F84179507A60713
:105C2000B70709F43AC020910A0830910B08269D65
:105C3000C001279D900D369D900D1124845F974FD4
:105C400064E172E00E948BAE009739F5EFE3FCE06F
:105C500007C09091C00095FFFCCF8093C60031969D
:105C600084918823B1F7E6E4FCE007C09091C0007E
:105C700095FFFCCF8093C600319684918823B1F7BD
:105C80008FE59AE0B501A4012AE030E00E94FA7F96
:105C90008091C00085FFFCCF91C080910A0890914F
:105CA0000B08869D7001879DF00C969DF00C1124C9
:105CB0002CE0C22E28E0D22ECE0CDF1CC6016AE2F8
:105CC00070E00E945CAE009721F452C003272F5F62
:105CD00002C020E000E0F701E20FF11DE45FF74FA2
:105CE00030813A3299F790939709809396098C19ED
:105CF0009D098E0D9F1D835F974F60E070E00E94AD
:105D000055AB0E94A2A7AB01BC01802F90E0841785
:105D1000950709F459C0EFE3FCE007C09091C0007B
:105D200095FFFCCF8093C600319684918823B1F70C
:105D3000E8E7FCE007C09091C00095FFFCCF80939E
:105D4000C600319684918823B1F740919C09509107
:105D50009D0960919E0970919F098FE59AE02AE064
:105D600030E00E94FA7F8091C00085FFFCCF26C002
:105D7000EFE3FCE007C09091C00095FFFCCF80935B
:105D8000C600319684918823B1F7E6E9FCE007C0AC
:105D90009091C00095FFFCCF8093C600319684910E
:105DA0008823B1F78FE59AE0B501A4012AE030E03D
:105DB0000E94FA7F8091C00085FFFCCF8AE080932B
:105DC000C6000E94EF2947C08091980990919909D7
:105DD000A0919A09B0919B0980939C0990939D0989
:105DE000A0939E09B0939F093BC0C8016AE270E08E
:105DF0000E945CAE0097A1F1EFE3FCE007C0909138
:105E0000C00095FFFCCF8093C60031968491882313
:105E1000B1F7EFEBFCE007C09091C00095FFFCCF1D
:105E20008093C600319684918823B1F740919C09F4
:105E300050919D0960919E0970919F098FE59AE0AC
:105E40002AE030E00E94FA7F8091C00085FFFCCFFD
:105E50008AE08093C600109295091092940924C29A
:105E600080910A0890910B08869D7001879DF00C27
:105E7000969DF00C11248701045F174FC80167E459
:105E800070E00E945CAE009709F44AC090939709B5
:105E900080939609801B910B8E0D9F1D835F974FFA
:105EA00060E070E00E9455AB0E94A2A7DC01CB012C
:105EB00084309105A8F58091FE068823C9F480916D
:105EC0002407882369F5842DE8EEFCE008C0909152
:105ED000C00095FFFCCF8093C60031968491882343
:105EE000B1F78091C00085FFFCCF5092C60018C06A
:105EF000832DEBEEFCE008C09091C00095FFFCCF35
:105F00008093C600319684918823B1F78091C000B8
:105F100085FFFCCF5092C60083E69DE00E94A42C32
:105F200080910A0890910B08019664E070E00E944D
:105F300001AB90930B0880930A0880910808909118
:105F40000908019690930908809308081092950912
:105F5000109294091FC08B3319F491E09093930928
:105F6000909193099923B1F420910A0830910B087C
:105F7000269DF001279DF00D369DF00D1124E40FB4
:105F8000F51FE45FF74F80834F5F5F4F5093950994
:105F9000409394098091E00A9091E10A2091E20AED
:105FA0003091E30A821B930B8F779070009709F46E
:105FB00076C18091080890910908843091050CF011
:105FC0006EC18FE59AE00E94427F809392094091D2
:105FD0009409509195098A3009F0C0CDCBCD8091BC
:105FE000940990919509009709F40DC15DC14D3058
:105FF00091F04A3321F420919309222361F02091FA
:106000009409309195092F3531052CF4FFEF8F3F1E
:106010009F0709F0D9C08091FE079091FF07A091DA
:106020000008B09101084091F6075091F707609180
:10603000F8077091F90784179507A607B70708F4C2
:106040008CC0862DEDE6FDE008C09091C00095FF64
:10605000FCCF8093C600319684918823B1F780915C
:10606000C00085FFFCCFE092C6000E9425A3DC01A2
:10607000CB018093A0099093A109A093A209B093AA
:10608000A3094091A4095091A5096091A6097091B6
:10609000A709841B950BA60BB70BBC01CD0128EEFD
:1060A00033E040E050E00E9414AB8DB79EB70897F4
:1060B0000FB6F8949EBF0FBE8DBF0DB71EB70F5F12
:1060C0001F4FEDB7FEB792828182F80133822282A0
:1060D000CA01B9012CE330E040E050E00E9414AB6B
:1060E000DC01CB01F80135832483978386830E94EA
:1060F000A5AE852D2DB73EB7285F3F4F0FB6F8945C
:106100003EBF0FBE2DBFEAE6F9E008C09091C00087
:1061100095FFFCCF8093C600319684918823B1F718
:10612000F40106C09091C00095FFFCCF8093C6009B
:1061300081918823B9F78091C00085FFFCCFE09260
:10614000C600C4010E94882C84E297E00E940B8B59
:1061500084E297E061E00E946F88809194099091B9
:106160009509009719F4109293099EC020910A088E
:1061700030910B082A9DF0012B9DF00D3A9DF00DFA
:106180001124E80FF91FE45FF74F1082F901E4577B
:10619000F64FC0828091080890910908019690936B
:1061A000090880930808C901019664E070E00E9424
:1061B00001AB90930B0880930A08109293091092F8
:1061C00095091092940934C04B3311F4C09293098D
:1061D00080919309882361F580910A0890910B08BA
:1061E0008A9DF0018B9DF00D9A9DF00D1124E20F18
:1061F000F31FE45FF74F40832F5F3F4F30939509C4
:106200002093940915C0B0E6AB2EB12CCC24C394D6
:10621000EDE6FDE064901AE0E12E4E010894811C49
:10622000911C09E1202E02E0302EEAE6F9E05490BC
:106230008091FE079091FF07A0910008B09101089E
:106240004091F6075091F7076091F8077091F907B0
:1062500084179507A607B70738F58091080890912D
:1062600009088430910504F58091E3079091E407D3
:10627000A091E507B091E6078093FE079093FF0792
:10628000A0930008B09301088BED97E00E940F1ACD
:10629000482F809392098A3009F0A9CEBCCE809114
:1062A0002507882309F09BCE6E960FB6F894DEBFC3
:1062B0000FBECDBFDF91CF911F910F91FF90EF9057
:1062C000DF90CF90BF90AF909F908F907F906F9016
:1062D0005F904F903F902F900895CF9382E161E0BF
:1062E0000E9483A2C4E15B9A65E070E080E090E0E8
:1062F0000E9461A35B9865E070E080E090E00E94FE
:1063000061A3C15081F7CF910895CF9382E161E0FD
:106310000E9483A2CAE05B9A63E070E080E090E0B4
:106320000E9461A35B9863E070E080E090E00E94CF
:1063300061A3C15081F7CF91089588E260E00E9487
:1063400083A28AE260E00E9483A283E160E00E946F
:1063500083A286E260E00E9483A2A19A9FB7F8948C
:10636000EBE0F1E08081806880839FBF5A9A5F9A5A
:106370000895CF93DF93CDB7DEB7A8970FB6F89403
:10638000DEBF0FBECDBF0E949D31DE019196E8E2D7
:10639000F2E088E001900D928150E1F7DE0159961C
:1063A000E0E3F2E088E001900D928150E1F7DE0138
:1063B0005196E8E3F2E088E001900D928150E1F718
:1063C000DE011996E0E4F2E088E001900D92815040
:1063D000E1F7DE011196E8E4F2E088E001900D9229
:1063E0008150E1F782EE96E064E144E020E00E9413
:1063F00070A582EE96E061E0AE014F5D5F4F0E94B6
:10640000F8A482EE96E062E0AE01475E5F4F0E9424
:10641000F8A482EE96E063E0AE014F5E5F4F0E940B
:10642000F8A482EE96E064E0AE01475F5F4F0E9401
:10643000F8A482EE96E065E0AE014F5F5F4F0E94E8
:10644000F8A48CEE9FE00E94A42CA8960FB6F894B6
:10645000DEBF0FBECDBFDF91CF910895CF92DF9207
:10646000EF92FF92CF93C1E09199C0E08091090132
:1064700087FFC260C090EE09D090EF09E090F0096C
:10648000F090F1090E9425A3DC01CB01C816D906C2
:10649000EA06FB0610F44A9BC460C093FD064091D7
:1064A000FD0641708091FD0681FD4260242F30E0A1
:1064B0008091F7069091F80628173907F1F14230DC
:1064C00059F0433079F04130A1F081309105A1F0CD
:1064D0008230910591F51EC0009771F083309105CF
:1064E00061F518C08230910539F08130910529F5A8
:1064F00011C08330910561F48091F9069091FA06FC
:10650000A091FB06B091FC060196A11DB11D0DC026
:10651000009799F48091F9069091FA06A091FB06F4
:10652000B091FC060197A109B1098093F9069093F7
:10653000FA06A093FB06B093FC063093F80620936E
:10654000F706CF91FF90EF90DF90CF900895FC0178
:1065500011821282108281E083831286138608954D
:10656000AF92BF92CF92DF92EF92FF920F931F9361
:10657000CF93DF93EC0199858885981719F48B8167
:10658000882331F081E08B8382EE96E00E9468A53B
:10659000F88400E010E0AF2CBB24A7FCB0941DC22F
:1065A000443009F4E2C045307CF4413009F446C07F
:1065B00042301CF44423A9F00EC2423009F477C0E3
:1065C000433009F008C2A1C0463009F43FC146304B
:1065D0000CF4F9C0473009F487C1483009F0FBC119
:1065E000CCC18B81882351F082EE96E060E0402F91
:1065F0000E943AA587E190E10E94782C28813327F8
:1066000027FD30958C2D90E02817390709F0E3C15C
:106610008091FD0682FFDFC10E9425A3DC01CB0132
:106620008C509E4FAF4FBF4F8093EE099093EF0970
:10663000A093F009B093F10981E0CAC18B8188234E
:1066400051F082EE96E060E0402F0E943AA58FE183
:1066500090E10E94782C2881332727FD30958C2DDE
:1066600090E02817390709F0B6C18091FD0682FF36
:10667000B2C10E9425A3DC01CB018C509E4FAF4FCD
:10668000BF4F8093EE099093EF09A093F009B09368
:10669000F109109235071092340784E297E00E94C6
:1066A000488484E297E061E00E946F8892C18B8108
:1066B000882351F082EE96E060E0402F0E943AA5D8
:1066C0008AE290E10E94782C2881332727FD3095BB
:1066D0008C2D90E02817390709F07DC18091FD06C7
:1066E00082FF79C10E9425A3DC01CB018C509E4F13
:1066F000AF4FBF4F8093EE099093EF09A093F0093D
:10670000B093F10980E592E02DC08B81882351F090
:1067100082EE96E060E0402F0E943AA58CE390E183
:106720000E94782C2881332727FD30958C2D90E00E
:106730002817390709F04FC18091FD0682FF4BC130
:106740000E9425A3DC01CB018C509E4FAF4FBF4F61
:106750008093EE099093EF09A093F009B093F109AB
:1067600084E592E00E940C2934C18B81882351F08A
:1067700082EE96E060E0402F0E943AA587E490E127
:106780000E94782C2881332727FD30958C2D90E0AE
:106790002817390709F01FC18091FD0682FF1BC130
:1067A0000E9425A3DC01CB018C509E4FAF4FBF4F01
:1067B0008093EE099093EF09A093F009B093F1094B
:1067C00088E592E0CFCF8B81882351F082EE96E06E
:1067D00060E0402F0E943AA583E590E10E94782C6A
:1067E0002881332727FD30958C2D90E02817390715
:1067F00009F0F1C08091FD0682FFEDC00E9425A343
:10680000DC01CB018C509E4FAF4FBF4F8093EE0900
:106810009093EF09A093F009B093F10984EB90E015
:1068200060E00E9422759093230A8093220A80E000
:1068300090E0A4E3B3E48093180A9093190AA0931C
:106840001A0AB0931B0A86E490E042C08B81882329
:1068500051F082EE96E060E0402F0E943AA580E67B
:1068600090E10E94782C2881332727FD30958C2DCC
:1068700090E02817390709F0AEC08091FD0682FF2D
:10688000AAC00E9425A3DC01CB018C509E4FAF4FC4
:10689000BF4F8093EE099093EF09A093F009B09356
:1068A000F10980EF90E060E00E9422759093230A46
:1068B0008093220A80E090E0A0E7B3E48093180A76
:1068C0009093190AA0931A0AB0931B0A84E690E0E9
:1068D0000E946A759093210A8093200A87E06FEFE7
:1068E00070E00E9433A175C08B81882351F082EE45
:1068F00096E060E0402F0E943AA58DE690E10E946C
:10690000782C2881332727FD30958C2D90E028178F
:10691000390709F060C08091FD0682FF5CC00E94CB
:1069200025A3DC01CB018C509E4FAF4FBF4F80930E
:10693000EE099093EF09A093F009B093F10980E07C
:1069400090E060E00E9422759093230A8093220ACF
:1069500080E090E0A0E0B0E08093180A9093190ADC
:10696000A0931A0AB0931B0A80E090E00E946A7517
:106970009093210A8093200A2CC08B81882351F0A8
:1069800082EE96E060E0402F0E943AA587E790E112
:106990000E94782C2881332727FD30958C2D90E09C
:1069A00028173907C1F48091FD0682FF14C00E94A8
:1069B00025A3DC01CB018C509E4FAF4FBF4F80937E
:1069C000EE099093EF09A093F009B093F10983E0E9
:1069D00089830E9485310F5F1F4FC02E402F4F0DBE
:1069E0005885852F992787FD9095039698012A0D44
:1069F0003B1D821793070CF0D3CD8A85882309F0BD
:106A000088C05987C090F906D090FA06E090FB063E
:106A1000F090FC061B828C819D81AE81BF81A70115
:106A20009601281B390B4A0B5B0BDA01C90104964E
:106A3000A11DB11D89309105A105B10508F069C0FE
:106A400082EE96E060E048810E943AA582EE96E0F0
:106A500060E20E943CA48885F7FE06C081508887CA
:106A600087FF51C018864FC035E1C316D104E10439
:106A7000F1045CF08F5F8887863014F085E08887AA
:106A80006FE0C62ED12CE12CF12CC092F906D092E9
:106A9000FA06E092FB06F092FC06CC82DD82EE82E2
:106AA000FF82C701B60125E030E040E050E00E94DF
:106AB00036AB2883243011F483E0888388818930C1
:106AC00014F088E0888399858885981711F081E013
:106AD0008B8382EE96E060E048810E943AA588812F
:106AE000992787FD90952885332727FD3095820FBC
:106AF000931F009711F06EE301C063E082EE96E011
:106B00000E943CA406C054E0C52ED12CE12CF12CEF
:106B1000BCCFDF91CF911F910F91FF90EF90DF904D
:106B2000CF90BF90AF9008952F923F924F925F9277
:106B30006F927F928F929F92AF92BF92CF92DF928D
:106B4000EF92FF920F931F93CF93DF93CDB7DEB7F2
:106B5000A2970FB6F894DEBF0FBECDBF8C01DC014B
:106B600019969C91199718968C911897981729F453
:106B700013968C911397882339F081E0F801838371
:106B800082EE96E00E9468A5D80113968C91139727
:106B9000882379F080912607882339F084E297E0F2
:106BA0000E94E3898093090A04C01092090AF8013F
:106BB0001086D8011896BC901897882499247724B9
:106BC0002B2D332727FD309538A32F8F21503040B0
:106BD0003AA329A347E2442E47E0542EA42C652C67
:106BE0001E010894211C311C5EC1BB2029F031E03C
:106BF000B31609F090C036C0D80113968C91139744
:106C0000882351F082EE96E060E0482D0E943AA57C
:106C100080E292E10E94782CF8012081332727FD41
:106C200030958C2D90E02817390709F038C18091F4
:106C3000FD0682FF34C10E9425A3DC01CB018C50EC
:106C40009E4FAF4FBF4F8093EE099093EF09A093F3
:106C5000F009B093F10981E0D80111968C930E945C
:106C600085311DC1F8018381882369F182EE96E0A8
:106C700060E0482D0E943AA582EE96E065E672E05B
:106C80000E942BA48BE597E067E277E00E942A1828
:106C9000809127078F3229F488E292E10E94782CB4
:106CA00012C082EE96E067E672E00E942BA482EEAC
:106CB00096E067E277E00E942BA482EE96E069E618
:106CC00072E00E942BA4D8012C91332727FD309528
:106CD0008C2D90E02817390709F0E1C08091FD065E
:106CE00082FFDDC00E9425A3DC01CB018C509E4FAA
:106CF000AF4FBF4F8093EE099093EF09A093F00937
:106D0000B093F10984E297E00E94DC8AF8011086D2
:106D10000E94853180C029A13AA1280D391D80919A
:106D2000090A90E0821793070CF4B9C0D8011396B2
:106D30008C911397882301F16B2D625084E297E0C8
:106D40000E94998982EE96E060E0482D0E943AA563
:106D500081E392E10E94782C80913307882331F0FF
:106D600082EE96E067E672E00E942BA482EE96E047
:106D700067E277E00E942BA4F8012081332727FDEA
:106D800030958C2D90E02817390709F088C0809144
:106D9000FD0682FF84C00E9425A3DC01CB018C503C
:106DA0009E4FAF4FBF4F8093EE099093EF09A09392
:106DB000F009B093F1096B2D625084E297E00E94D4
:106DC00099898091330727E2C22E27E0D22EEE2444
:106DD000FF24882349F42AC0D6018C9190E00E94B8
:106DE0001BAEF60181936F01C701F20101900020F3
:106DF000E9F7E852F7400894E11CF11C8E179F0751
:106E000058F384E297E067E277E00E94328AD80183
:106E100018961C9218977724739441C0F6018081CC
:106E200090E00E941BAED6018D936D01C701F20167
:106E300001900020E9F7E852F7400894E11CF11CAA
:106E40008E179F0758F300D000D0EDB7FEB73196EC
:106E5000ADB7BEB712963C922E9211972DE632E056
:106E600033832283A48265820E94A5AE4DB75EB7AC
:106E70004A5F5F4F0FB6F8945EBF0FBE4DBFC101B2
:106E80000E940C2984E792E00E940C290E946D3137
:106E9000D80111961C9287E297E00E94882CB39447
:106EA0000894811C911CC82CF8014085842F9927D7
:106EB00087FD909503962F8D38A1280D391D8217D7
:106EC00093070CF092CEA090090A8285882309F0DE
:106ED000B2C04187C090F906D090FA06E090FB0658
:106EE000F090FC06138284819581A681B781A70169
:106EF0009601281B390B4A0B5B0BDA01C90104967A
:106F0000A11DB11D89309105A105B10508F093C0FF
:106F1000BA2CB39482EE96E060E040810E943AA5DC
:106F200082EE96E060E20E943CA4D80118968C9113
:106F30001897F7FE0AC0815018968C93189787FF10
:106F400082C018961C9218977EC0B5E1CB16D1046A
:106F5000E104F10434F18F5FF80180872B2D30E0DC
:106F6000A90142505040992787FD909584179507B5
:106F70001CF08A2D825080876901CC0CDD1CCC0C62
:106F8000DD1CC20ED31EFFE0CF16D1042CF4EE247C
:106F9000D7FCE094FE2C05C0EFE0CE2ED12CE12CE6
:106FA000F12CC092F906D092FA06E092FB06F0921C
:106FB000FC06D8011496CD92DD92ED92FC921797C3
:106FC000C701B60125E030E040E050E00E9436AB5A
:106FD000F8012083243011F483E08083D8012C91C0
:106FE000332727FD30958B2D90E0821793070CF403
:106FF000BC92F80191858085981711F081E0838318
:1070000082EE96E060E0D8014C910E943AA5F8012A
:107010008081992787FD90952085332727FD30951E
:10702000820F931F009711F06EE301C063E082EEC0
:1070300096E00E943CA4772061F081E0D80113968D
:107040008C93139706C074E0C72ED12CE12CF12C41
:10705000A8CFA2960FB6F894DEBF0FBECDBFDF91CA
:10706000CF911F910F91FF90EF90DF90CF90BF9045
:10707000AF909F908F907F906F905F904F903F90D8
:107080002F900895AF92BF92CF92DF92EF92FF922E
:107090000F931F93CF93DF93EC018B85882361F0CF
:1070A0000E94A19F882399F480912507882379F471
:1070B00081E08B831B860BC00E94A19F882321F453
:1070C00080912507882319F081E08B838B87998530
:1070D0008885981719F48B81882331F081E08B83A0
:1070E00082EE96E00E9468A5F88400E010E0AF2CE4
:1070F000BB24A7FCB094EFE3FCE0D490E8E8F2E115
:10710000E49002C14130C9F142301CF4442341F003
:10711000D6C0423009F467C0433009F0D0C090C0F7
:107120008B81882351F082EE96E060E0402F0E9430
:107130003AA583E392E10E94782C2881332727FD2A
:1071400030958C2D90E02817390709F0DBC080912D
:10715000FD0682FFD7C00E9425A3DC01CB018C5025
:107160009E4FAF4FBF4F8093EE099093EF09A093CE
:10717000F009B093F109198233C08B81882381F023
:1071800082EE96E060E0402F0E943AA58B8588232E
:1071900019F48EE392E102C089E492E10E94782C16
:1071A0002881332727FD30958C2D90E0281739074B
:1071B00009F0A8C08091FD0682FFA4C00E9425A30B
:1071C000DC01CB018C509E4FAF4FBF4F8093EE0937
:1071D0009093EF09A093F009B093F10982E08983BD
:1071E0000E9485318FC08B81882351F082EE96E01A
:1071F00060E0402F0E943AA584E592E10E94782C3D
:107200002881332727FD30958C2D90E028173907EA
:1072100009F078C08091FD0682FF74C00E9425A30A
:10722000DC01CB018C509E4FAF4FBF4F8093EE09D6
:107230009093EF09A093F009B093F10984E0CFCFC8
:107240008B818823B1F082EE96E060E0402F0E94AF
:107250003AA54F990AC080912507882319F08FE538
:1072600092E105C08FE692E102C08FE792E10E94B1
:10727000782C4F9947C02881332727FD30958C2DD6
:1072800090E02817390709F03DC08091FD0682FF84
:1072900039C084E297E00E940B8B0E9425A3DC0199
:1072A000CB018C509E4FAF4FBF4F8093EE09909310
:1072B000EF09A093F009B093F10985E090CF8D2DEF
:1072C000EFE3FCE008C09091C00095FFFCCF8093F5
:1072D000C600319684918823B1F78E2DE8E8F2E15B
:1072E00008C09091C00095FFFCCF8093C6003196F6
:1072F00084918823B1F78091C00085FFFCCF8AE09C
:107300008093C6000F5F1F4FC02E402F4F0D588532
:10731000852F992787FD9095039698012A0D3B1D8F
:10732000821793070CF0EECE8A85882309F087C078
:107330005987C090F906D090FA06E090FB06F090CD
:10734000FC061B828C819D81AE81BF81A7019601C5
:10735000281B390B4A0B5B0BDA01C9010496A11DEE
:10736000B11D89309105A105B10508F068C082EE14
:1073700096E060E048810E943AA582EE96E060E2E5
:107380000E943CA48885F7FE06C08150888787FF4D
:1073900050C018864EC035E1C316D104E104F10493
:1073A00054F08F5F888718160CF418866FE0C62E8D
:1073B000D12CE12CF12CC092F906D092FA06E09281
:1073C000FB06F092FC06CC82DD82EE82FF82C701D2
:1073D000B60125E030E040E050E00E9436AB288363
:1073E000243011F483E088838881843014F083E0B2
:1073F000888399858885981711F081E08B8382EEC8
:1074000096E060E048810E943AA58881992787FD2F
:1074100090952885332727FD3095820F931F00977D
:1074200011F06EE301C063E082EE96E00E943CA49E
:1074300006C054E0C52ED12CE12CF12CBCCFDF913D
:10744000CF911F910F91FF90EF90DF90CF90BF9061
:10745000AF900895FC0160817181828193810E94C7
:10746000A2A7DC01CB01FC0164E670E00E9401AB45
:10747000CB012AE030E0B9010E9401AB805D80932E
:107480000F0ACF01B9010E9401AB482FCB01B9010E
:107490000E9401AB805D8093100A405D4093110A09
:1074A0001092120A8FE09AE00895FC0180812AE090
:1074B00030E090E0B9010E9401AB482FCB01B90147
:1074C0000E9401AB805D80930F0A405D4093100ADB
:1074D0001092110A8FE09AE00895FC018081918159
:1074E00064E670E00E9401ABCB012AE030E0B90114
:1074F0000E9401AB805D80930F0A80819181B90168
:107500000E9401ABCB01B9010E9401AB805D809369
:10751000100A80819181B9010E9401AB805D809346
:10752000110A1092120A8FE09AE00895FC018081FE
:10753000918168EE73E00E9401ABCB012AE030E05C
:10754000B9010E9401AB805D80930F0A8081918117
:1075500064E670E00E9401ABCB01B9010E9401AB6F
:10756000805D8093100A80819181B9010E9401ABF6
:10757000CB01B9010E9401AB805D8093110A80812B
:107580009181B9010E9401AB805D8093120A109233
:10759000130A8FE09AE00895FC0160817181828175
:1075A000938120E030E040E251E40E9408AA0E946A
:1075B000A2A79B0177FD02C08BE201C08DE2809300
:1075C0000F0A37FF03C0309521953F4FC90160E195
:1075D00077E20E9401ABCB01EAE0F0E0BF010E943C
:1075E00001AB805D8093100AC90168EE73E00E94D0
:1075F00001ABCB01BF010E9401AB805D8093110AFA
:10760000C90164E670E00E9401ABCB01BF010E949A
:1076100001AB805D8093120AC901BF010E9401ABDA
:10762000282FCB01BF010E9401AB805D8093130A1C
:107630008EE28093140A205D2093150A1092160A98
:107640008FE09AE008956F927F928F929F92AF920F
:10765000BF92CF92DF92EF92FF920F931F93CF933F
:10766000DF93CDB7DEB7A0970FB6F894DEBF0FBE9D
:10767000CDBF8C01FC0191858085981719F4838119
:10768000882339F081E0F801838382EE96E00E943E
:1076900068A5F801A084882499246A2C772467FCC3
:1076A00070946FC5433009F4F8C144304CF4413054
:1076B00009F443C042300CF036C1442359F05EC592
:1076C000453009F4B1C345300CF4B6C2463009F078
:1076D00055C586C4F8018381882351F082EE96E077
:1076E00060E0482D0E943AA58DED90E10E94782C33
:1076F000F8012081332727FD30958B2D90E0281746
:10770000390709F03BC58091FD0682FF37C50E940D
:1077100025A3DC01CB018C509E4FAF4FBF4F809310
:10772000EE099093EF09A093F009B093F10984E07A
:10773000F80181830E94853121C5F8018381882366
:10774000A1F182EE96E060E0482D0E943AA588EE15
:1077500090E10E94782C82EE96E06DE0482D0E9428
:107760003AA58091220A9091230A60E00E946D75EB
:1077700020E030E040E05FE30E945AA60E94A2A70A
:10778000882777FD8095982F0E94D5A7DC01CB0133
:107790008D8F9E8FAF8FB8A3CE014D960E942A3A4F
:1077A000BC0182EE96E00E942BA4F801808199270B
:1077B00087FD90952B2D30E08217930709F0DEC4EA
:1077C0008091FD0682FF6DC0828591E089278287C6
:1077D0008823F1F08091220A9091230A60E00E94B0
:1077E0006D7520E030E040E05FE30E945AA60E9401
:1077F000A2A7DC01CB01AA2797FDA095BA2F809301
:10780000F9069093FA06A093FB06B093FC0639C0E4
:107810006091F9067091FA068091FB069091FC0642
:107820000E94D5A76B017C010E94A2A7DC01CB01BD
:1078300060E00E9422759093230A8093220AC092EE
:10784000180AD092190AE0921A0AF0921B0AF8015B
:107850002081332727FD3095C901880F991F880F94
:10786000991F820F931FAA2797FDA095BA2F809387
:10787000F9069093FA06A093FB06B093FC060E94CB
:1078800085310E9425A3DC01CB018C509E4FAF4F68
:10789000BF4F8093EE099093EF09A093F009B09346
:1078A000F109F8018285882309F468C48091F906FA
:1078B0009091FA06A091FB06B091FC06B7FF08C0B4
:1078C0001092F9061092FA061092FB061092FC062E
:1078D0008091F9069091FA06A091FB06B091FC0602
:1078E0008530F1E09F07F0E0AF07F0E0BF0764F0FC
:1078F00084E091E0A0E0B0E08093F9069093FA066E
:10790000A093FB06B093FC0682EE96E06DE04B2D53
:107910000E943AA58091F9069091FA06988B8F877C
:10792000CE010F9624C4F8018381882331F182EEC1
:1079300096E060E0482D0E943AA582EF90E10E9417
:10794000782C82EE96E06DE0482D0E943AA5609179
:10795000FF0670E080E090E00E94D3A7DC01CB013D
:10796000898F9A8FAB8FBC8FCE0149960E942A3A9D
:10797000BC0182EE96E00E942BA4F80120813327FF
:1079800027FD30958B2D90E02817390709F0F6C3B5
:107990008091FD0682FF39C0828591E08927828728
:1079A000882371F08091FF0690E0A0E0B0E0809322
:1079B000F9069093FA06A093FB06B093FC0615C057
:1079C000C901880F991F880F991F820F931FAA273B
:1079D00097FDA095BA2F8093F9069093FA06A0938D
:1079E000FB06B093FC060E9485310E9425A3DC01B2
:1079F000CB018C509E4FAF4FBF4F8093EE099093B9
:107A0000EF09A093F009B093F109F801828588236A
:107A100009F4B4C38091F9069091FA06A091FB068F
:107A2000B091FC06B7FF08C01092F9061092FA0652
:107A30001092FB061092FC068091F9069091FA06CE
:107A4000A091FB06B091FC068F3F9105A105B10501
:107A500069F064F08FEF90E0A0E0B0E08093F90669
:107A60009093FA06A093FB06B093FC066091F9068A
:107A70006093FF0687E070E00E9433A182EE96E0FB
:107A80006DE04B2D0E943AA58091F9069091FA067F
:107A90009E878D87CE010D966AC3F8018381882366
:107AA00039F182EE96E060E0482D0E943AA58EEF13
:107AB00090E10E94782C82EE96E06DE0482D0E94C5
:107AC0003AA5609136047091370480913804909102
:107AD00039040E94A2A7DC01CB019C878B87CE01D1
:107AE0000B960E94963ABC0182EE96E00E942BA46F
:107AF000F801C080DD24C7FCD0948B2D90E0C8161F
:107B0000D90609F03BC38091FD0682FF4CC08285F7
:107B100091E089278287882369F06091360470910B
:107B2000370480913804909139040E94A2A7DC01A7
:107B3000CB011FC06091F9067091FA068091FB0697
:107B40009091FC060E94D5A7DC01CB0180933604FE
:107B500090933704A0933804B0933904C601880F7A
:107B6000991F880F991F8C0D9D1DAA2797FDA09521
:107B7000BA2F8093F9069093FA06A093FB06B09370
:107B8000FC060E9425A3DC01CB018C509E4FAF4F19
:107B9000BF4F8093EE099093EF09A093F009B09343
:107BA000F1090E948531F8018285882309F4E6C233
:107BB0008091F9069091FA06A091FB06B091FC061F
:107BC000181619061A061B0664F081E090E0A0E082
:107BD000B0E08093F9069093FA06A093FB06B09369
:107BE000FC068091F9069091FA06A091FB06B091EF
:107BF000FC068730F7E29F07F0E0AF07F0E0BF0731
:107C000064F086E097E2A0E0B0E08093F9069093FC
:107C1000FA06A093FB06B093FC0682EE96E06DE0B8
:107C20004B2D0E943AA58091F9069091FA069A8709
:107C30008987CE010996D1C1F8018381882369F132
:107C400082EE96E060E0482D0E943AA587E091E13F
:107C50000E94782C82EE96E06DE0482D0E943AA5B5
:107C60006091320470913304809134049091350412
:107C70002FE632E143E05EE30E943AA7DC01CB014C
:107C80008D8B9E8BAF8BB88FCE0145960E94CC3AE0
:107C9000BC0182EE96E00E942BA4F801C080DD2496
:107CA000C7FCD0948B2D90E0C816D90609F066C2A7
:107CB0008091FD0682FF64C0828591E089278287DA
:107CC0008823C9F0609132047091330480913404A8
:107CD0009091350420E030E040E251E40E9408AA8F
:107CE0002FE632E143E05EE30E943AA70E94A2A79A
:107CF000DC01CB012BC06091F9067091FA068091EE
:107D0000FB069091FC060E94D5A720E030E040E2FF
:107D100051E40E943AA72FE632E143E05EE30E947D
:107D200008AADC01CB018093320490933304A09322
:107D30003404B0933504C601880F991F880F991F2A
:107D40008C0D9D1DAA2797FDA095BA2F8093F9064B
:107D50009093FA06A093FB06B093FC060E9425A31D
:107D6000DC01CB018C509E4FAF4FBF4F8093EE098B
:107D70009093EF09A093F009B093F1090E94853127
:107D8000F8018285882309F4F9C18091F906909160
:107D9000FA06A091FB06B091FC06B7FF08C010924E
:107DA000F9061092FA061092FB061092FC068091DA
:107DB000F9069091FA06A091FB06B091FC06873077
:107DC000F7E29F07F0E0AF07F0E0BF0764F086E05E
:107DD00097E2A0E0B0E08093F9069093FA06A093B2
:107DE000FB06B093FC0682EE96E06DE04B2D0E9400
:107DF0003AA56091F9067091FA068091FB06909180
:107E0000FC060E94D5A720E030E040E251E40E9449
:107E10003AA7DC01CB01898B9A8BAB8BBC8BCE0153
:107E200041960E94CC3AA5C1F8018381882369F16B
:107E300082EE96E060E0482D0E943AA580E191E153
:107E40000E94782C82EE96E06DE0482D0E943AA5C3
:107E500060912E0470912F04809130049091310430
:107E60002FE632E143E05EE30E9408AA0E94A2A747
:107E7000DC01CB0198878F83CE0107960E94963A4A
:107E8000BC0182EE96E00E942BA4F801C080DD24A4
:107E9000C7FCD0948B2D90E0C816D90609F06EC1AE
:107EA0008091FD0682FF58C0828591E089278287F4
:107EB0008823C9F060912E0470912F0480913004C2
:107EC0009091310420E030E040EA50E40E943AA76B
:107ED0002FE632E143E05EE30E943AA70E94A2A7A8
:107EE000DC01CB011FC06091F9067091FA06809108
:107EF000FB069091FC060E94D5A7DC01CB01809384
:107F00002E0490932F04A0933004B0933104C60143
:107F1000880F991F880F991F8C0D9D1DAA2797FD0B
:107F2000A095BA2F8093F9069093FA06A093FB06CA
:107F3000B093FC060E9425A3DC01CB018C509E4F20
:107F4000AF4FBF4F8093EE099093EF09A093F009D4
:107F5000B093F1090E948531F8018285882309F4E4
:107F60000DC18091F9069091FA06A091FB06B0919F
:107F7000FC06B7FF08C01092F9061092FA0610929C
:107F8000FB061092FC068091F9069091FA06A091EA
:107F9000FB06B091FC068730F7E29F07F0E0AF07E1
:107FA000F0E0BF0764F086E097E2A0E0B0E08093E5
:107FB000F9069093FA06A093FB06B093FC0682EEB6
:107FC00096E06DE04B2D0E943AA58091F9069091C4
:107FD000FA069E838D83CE0105960E94963AC9C00B
:107FE000F8018381882339F182EE96E060E0482D24
:107FF0000E943AA589E191E10E94782C82EE96E0F8
:108000006DE0482D0E943AA560912A0470912B04DE
:1080100080912C0490912D040E94A2A7DC01CB0139
:108020009C838B83CE0103960E946D3ABC0182EE45
:1080300096E00E942BA4F801C080DD24C7FCD094F8
:108040008B2D90E0C816D90609F098C08091FD06E6
:1080500082FF4CC0828591E089278287882369F05E
:1080600060912A0470912B0480912C0490912D042E
:108070000E94A2A7DC01CB011FC06091F90670919C
:10808000FA068091FB069091FC060E94D5A7DC01C0
:10809000CB0180932A0490932B04A0932C04B093DB
:1080A0002D04C601880F991F880F991F8C0D9D1DE7
:1080B000AA2797FDA095BA2F8093F9069093FA0608
:1080C000A093FB06B093FC060E9425A3DC01CB0124
:1080D0008C509E4FAF4FBF4F8093EE099093EF09A6
:1080E000A093F009B093F1090E948531F8018285CF
:1080F000882309F443C08091F9069091FA06A09173
:10810000FB06B091FC06B7FF08C01092F90610926A
:10811000FA061092FB061092FC068091F9069091E7
:10812000FA06A091FB06B091FC068F3DF3E09F0795
:10813000F0E0AF07F0E0BF0764F08EED93E0A0E061
:10814000B0E08093F9069093FA06A093FB06B093F3
:10815000FC0682EE96E06DE04B2D0E943AA58091E0
:10816000F9069091FA069A838983CE0101960E94BE
:108170006D3ABC0182EE96E00E942BA40894811C0B
:10818000911CB82C482D4A0DF8015085852F992750
:1081900087FD909503969401260D371D821793074E
:1081A0000CF080CA8285882309F090C05187C09066
:1081B000F906D090FA06E090FB06F090FC061382D8
:1081C00084819581A681B781A7019601281B390B6F
:1081D0004A0B5B0BDA01C9010496A11DB11D893060
:1081E0009105A105B10508F071C082EE96E060E04E
:1081F00040810E943AA582EE96E060E20E943CA493
:10820000F8018085F7FE06C08150808787FF58C03F
:10821000108656C0F5E1CF16D104E104F10464F0F4
:108220008F5FF8018087843014F083E08087EFE06F
:10823000CE2ED12CE12CF12CC092F906D092FA0668
:10824000E092FB06F092FC06F801C482D582E68239
:10825000F782C701B60125E030E040E050E00E941F
:1082600036ABF8012083243011F483E08083F801D9
:108270008081873014F086E08083F80191858085C5
:10828000981711F081E0838382EE96E060E0F801B8
:1082900040810E943AA5F8018081992787FD909539
:1082A0002085332727FD3095820F931F009711F00B
:1082B0006EE301C063E082EE96E00E943CA406C03B
:1082C00074E0C72ED12CE12CF12CB6CFA0960FB6BE
:1082D000F894DEBF0FBECDBFDF91CF911F910F91FC
:1082E000FF90EF90DF90CF90BF90AF909F908F90D6
:1082F0007F906F900895FC016081718182819381EC
:1083000020E030E048EC52E40E9408AA0E94A2A7B4
:108310009B0177FD02C08BE201C08DE280930F0AC2
:1083200037FF03C0309521953F4FC90160E177E2E7
:108330000E9401ABCB01EAE0F0E0BF010E9401AB7B
:10834000805D8093100AC90168EE73E00E9401AB62
:10835000CB01BF010E9401AB805D8093110AC9016E
:1083600064E670E00E9401ABCB01BF010E9401AB4B
:10837000805D8093120A8EE28093130AC901BF01C7
:108380000E9401AB282FCB01BF010E9401AB805D91
:108390008093140A205D2093150A1092160A8FE02C
:1083A0009AE008952F923F924F925F926F927F9240
:1083B0008F929F92AF92BF92CF92DF92EF92FF92F5
:1083C0000F931F93CF93DF93CDB7DEB7E6970FB62A
:1083D000F894DEBF0FBECDBF8C01FC019185808576
:1083E000981719F48381882339F081E0F801838399
:1083F00082EE96E00E9468A5F8016084262D33275E
:1084000027FD30953EAB2DAB220F331F220F331FBC
:108410002153304F3AAB29AB4DA95EA9440F551FEC
:10842000440F551F495F5F4E5CAB4BAB2224332496
:1084300038AA2FA6262C28010C940C4D58E025169E
:1084400009F415C35215ACF062E0261609F45AC1BE
:10845000621544F0222049F171E0271611F00C94C6
:10846000F94C5AC0F2018381F6E0F2150CF01BC200
:10847000C6C32EE0221609F47AC622153CF0F2019A
:108480008381FCE0F2150CF080C47FC520E1221648
:1084900011F40C94D54A22160CF478C731E1231656
:1084A00011F00C94F94C0C94E44BF2018381882375
:1084B00051F082EE96E060E04FA50E943AA582E27C
:1084C00091E10E94782CF2012081332727FD30951D
:1084D0008C2D90E02817390711F00C94F94C8091FD
:1084E000FD0682FD02C00C94F94C0E9425A3DC011C
:1084F000CB018C509E4FAF4FBF4F8093EE099093AE
:10850000EF09A093F009B093F10984E0F2018183AF
:108510000E9485310C94F94CF2018381882389F102
:1085200082EE96E060E04FA50E943AA58DE291E1CF
:108530000E94782C82EE96E06DE04FA50E943AA54D
:108540006091EB0F7091EC0F8091ED0F9091EE0F19
:1085500020E030E048EC52E40E943AA70E94A2A733
:10856000DC01CB019A8F898FCE0149960E946D3A2A
:10857000BC0182EE96E00E942BA483E391E10E946D
:10858000782CF2010081112707FD10958C2D90E0C9
:108590000817190711F00C94F94C8091FD0682FF21
:1085A0005EC0828591E0892782878823C9F0609127
:1085B000EB0F7091EC0F8091ED0F9091EE0F0E94F8
:1085C000A2A724E630E040E050E00E9436AB2093C2
:1085D000F9063093FA064093FB065093FC062DC033
:1085E0006091F9067091FA068091FB069091FC0665
:1085F00024E630E040E050E00E94CEAA0E94D5A7D9
:10860000DC01CB018093EB0F9093EC0FA093ED0F67
:10861000B093EE0FC801880F991F880F991F800F24
:10862000911FAA2797FDA095BA2F8093F9069093E2
:10863000FA06A093FB06B093FC060E9425A3DC017A
:10864000CB018C509E4FAF4FBF4F8093EE0990935C
:10865000EF09A093F009B093F1090E948531F2016E
:108660008285882311F40C94F94C8091F90690913D
:10867000FA06A091FB06B091FC0685309105A10594
:10868000B10564F485E090E0A0E0B0E08093F906E5
:108690009093FA06A093FB06B093FC068091F9062E
:1086A0009091FA06A091FB06B091FC068F3DF3E095
:1086B0009F07F0E0AF07F0E0BF0764F08EED93E0B6
:1086C000A0E0B0E08093F9069093FA06A093FB0631
:1086D000B093FC0682EE96E06DE04C2D0E943AA528
:1086E0008091F9069091FA06988F8F8BCE0147966C
:1086F0000E946D3ABC0182EE96E00E942BA486E3B4
:1087000091E140C4F2018381882339F182EE96E041
:1087100060E04FA50E943AA589E391E10E94782C80
:1087200082EE96E06DE04FA50E943AA56091E30FBE
:108730007091E40F8091E50F9091E60F0E94A2A73F
:10874000DC01CB019E8B8D8BCE0145960E946D3A4C
:10875000BC0182EE96E00E942BA4F2010081112759
:1087600007FD10958C2D90E00817190711F00C9457
:10877000F94C8091FD0682FF4CC0828591E08927EB
:108780008287882369F06091E30F7091E40F8091F4
:10879000E50F9091E60F0E94A2A7DC01CB011FC05C
:1087A0006091F9067091FA068091FB069091FC06A3
:1087B0000E94D5A7DC01CB018093E30F9093E40FD7
:1087C000A093E50FB093E60FC801880F991F880F9B
:1087D000991F800F911FAA2797FDA095BA2F80930C
:1087E000F9069093FA06A093FB06B093FC060E944C
:1087F00025A3DC01CB018C509E4FAF4FBF4F809320
:10880000EE099093EF09A093F009B093F1090E944B
:108810008531F2018285882311F40C94F94C809102
:10882000F9069091FA06A091FB06B091FC06181685
:1088300019061A061B0664F081E090E0A0E0B0E0A3
:108840008093F9069093FA06A093FB06B093FC067A
:108850008091F9069091FA06A091FB06B091FC0672
:108860008F3DF3E09F07F0E0AF07F0E0BF0764F053
:108870008EED93E0A0E0B0E08093F9069093FA06C5
:10888000A093FB06B093FC0682EE96E06DE04C2DC3
:108890000E943AA58091F9069091FA069C8B8B8BE9
:1088A000CE014396E1C08823F1F182EE96E060E0CC
:1088B0004FA50E943AA585E491E10E94782C23E01F
:1088C000221619F48CE491E111C034E0231619F456
:1088D0008FE491E10BC045E0241619F482E591E1A3
:1088E00005C056E0251621F485E591E10E94782C1B
:1088F00082EE96E06DE04C2D0E943AA5EBA9FCA912
:1089000060817181828193810E94A2A7DC01CB01E9
:108910009A8B898BCE0141960E946D3ABC0182EE02
:1089200096E00E942BA4F2010081112707FD10950B
:108930008C2D90E00817190711F00C94F94C8091D8
:10894000FD0682FF48C0828591E0892782878823BF
:1089500059F0EBA9FCA960817181828193810E9409
:10896000A2A7DC01CB011DC06091F9067091FA0647
:108970008091FB069091FC060E94D5A7DC01CB01FB
:10898000EBA9FCA980839183A283B383C801880FDC
:10899000991F880F991F800F911FAA2797FDA095F7
:1089A000BA2F8093F9069093FA06A093FB06B09332
:1089B000FC060E9425A3DC01CB018C509E4FAF4FDB
:1089C000BF4F8093EE099093EF09A093F009B09305
:1089D000F1090E948531F2018285882311F40C94FB
:1089E000F94C8091F9069091FA06A091FB06B0919E
:1089F000FC06181619061A061B0664F081E090E0C2
:108A0000A0E0B0E08093F9069093FA06A093FB06ED
:108A1000B093FC068091F9069091FA06A091FB06AE
:108A2000B091FC068F3DF3E09F07F0E0AF07F0E068
:108A3000BF0764F08EED93E0A0E0B0E08093F9060C
:108A40009093FA06A093FB06B093FC0682EE96E0A4
:108A50006DE04C2D0E943AA58091F9069091FA069E
:108A6000988B8F87CE010F960E946D3ABDC7F20199
:108A70008381882339F182EE96E060E04FA50E9461
:108A80003AA588E591E10E94782C82EE96E06DE0AF
:108A90004FA50E943AA56091EF0F7091F00F809161
:108AA000F10F9091F20F0E94A2A7DC01CB019E87EB
:108AB0008D87CE010D960E946D3ABC0182EE96E044
:108AC0000E942BA4F2010081112707FD10958C2D27
:108AD00090E00817190709F08CC78091FD0682FF06
:108AE0004CC0828591E089278287882369F0609154
:108AF000EF0F7091F00F8091F10F9091F20F0E94A3
:108B0000A2A7DC01CB011FC06091F9067091FA06A3
:108B10008091FB069091FC060E94D5A7DC01CB0159
:108B20008093EF0F9093F00FA093F10FB093F20F9B
:108B3000C801880F991F880F991F800F911FAA27BE
:108B400097FDA095BA2F8093F9069093FA06A0930B
:108B5000FB06B093FC060E9425A3DC01CB018C50E0
:108B60009E4FAF4FBF4F8093EE099093EF09A093B4
:108B7000F009B093F1090E948531F20182858823C2
:108B800009F437C78091F9069091FA06A091FB0687
:108B9000B091FC06B7FF08C01092F9061092FA06D1
:108BA0001092FB061092FC068091F9069091FA064D
:108BB000A091FB06B091FC068F3DF3E09F07F0E02B
:108BC000AF07F0E0BF0764F08EED93E0A0E0B0E007
:108BD0008093F9069093FA06A093FB06B093FC06E7
:108BE00082EE96E06DE04C2D0E943AA58091F90648
:108BF0009091FA069C878B87CE010B9635CF882300
:108C000039F182EE96E060E04FA50E943AA58FE52B
:108C100091E10E94782C82EE96E06DE04FA50E94D3
:108C20003AA56091D70F7091D80F8091D90F90918C
:108C3000DA0F0E94A2A7DC01CB019A878987CE01B7
:108C400009960E946D3ABC0182EE96E00E942BA428
:108C5000F2010081112707FD10958C2D90E0081777
:108C6000190709F0C6C68091FD0682FF4CC08285B7
:108C700091E089278287882369F06091D70F7091EE
:108C8000D80F8091D90F9091DA0F0E94A2A7DC0132
:108C9000CB011FC06091F9067091FA068091FB0626
:108CA0009091FC060E94D5A7DC01CB018093D70FE1
:108CB0009093D80FA093D90FB093DA0FC801880F03
:108CC000991F880F991F800F911FAA2797FDA095C4
:108CD000BA2F8093F9069093FA06A093FB06B093FF
:108CE000FC060E9425A3DC01CB018C509E4FAF4FA8
:108CF000BF4F8093EE099093EF09A093F009B093D2
:108D0000F1090E948531F2018285882309F471C638
:108D10008091F9069091FA06A091FB06B091FC06AD
:108D2000B7FF08C01092F9061092FA061092FB06DF
:108D30001092FC068091F9069091FA06A091FB062C
:108D4000B091FC068F3DF3E09F07F0E0AF07F0E045
:108D5000BF0764F08EED93E0A0E0B0E08093F906E9
:108D60009093FA06A093FB06B093FC0682EE96E081
:108D70006DE04C2D0E943AA58091F9069091FA067B
:108D800098878F83CE0107966FCE882309F444C05D
:108D900082EE96E060E04FA50E943AA58BE691E155
:108DA0000E94782C29E0221619F482E791E111C083
:108DB0003AE0231619F485E791E10BC04BE0241645
:108DC00019F488E791E105C05CE0251621F48BE7F2
:108DD00091E10E94782C82EE96E06DE04C2D0E948D
:108DE0003AA5E9A9FAA9608171818281938124E67B
:108DF00030E040E050E00E9414AB3E832D83CE0172
:108E000005960E946D3ABC0182EE96E00E942BA46A
:108E10008EE791E10E94782CF2010081112707FD75
:108E200010958C2D90E00817190709F0E2C5809184
:108E3000FD0682FF56C0828591E0892782878823BC
:108E4000A9F0E9A9FAA9608171818281938124E660
:108E500030E040E050E00E9436AB2093F9063093BA
:108E6000FA064093FB065093FC0629C06091F90670
:108E70007091FA068091FB069091FC0624E630E0A2
:108E800040E050E00E94CEAADC01CB01E9A9FAA99A
:108E900080839183A283B383C801880F991F880FB1
:108EA000991F800F911FAA2797FDA095BA2F809335
:108EB000F9069093FA06A093FB06B093FC060E9475
:108EC00025A3DC01CB018C509E4FAF4FBF4F809349
:108ED000EE099093EF09A093F009B093F1090E9475
:108EE0008531F2018285882309F483C58091F906D2
:108EF0009091FA06A091FB06B091FC06181619068F
:108F00001A061B0664F081E090E0A0E0B0E08093D8
:108F1000F9069093FA06A093FB06B093FC068091A5
:108F2000F9069091FA06A091FB06B091FC068F3DE0
:108F3000F3E09F07F0E0AF07F0E0BF0764F08EEDCD
:108F400093E0A0E0B0E08093F9069093FA06A09336
:108F5000FB06B093FC0682EE96E06DE04C2D0E947D
:108F60003AA58091F9069091FA069C838B83CE01F5
:108F700003960E946D3ABC0182EE96E00E942BA4FB
:108F800081E891E10E94782C34C5882389F182EE32
:108F900096E060E04FA50E943AA584E891E10E9426
:108FA000782C82EE96E06DE04FA50E943AA5609184
:108FB000E70F7091E80F8091E90F9091EA0F20E0A0
:108FC00030E048EC52E40E943AA7DC01CB018BA7C9
:108FD0009CA7ADA7BEA7CE018B960E942A3ABC01E2
:108FE00082EE96E00E942BA480E991E10E94782C09
:108FF000F2010081112707FD10958C2D90E00817D4
:10900000190709F0F6C48091FD0682FF5EC08285D3
:1090100091E0892782878823C9F06091E70F7091DA
:10902000E80F8091E90F9091EA0F0E94A2A724E631
:1090300030E040E050E00E9436AB2093F9063093D8
:10904000FA064093FB065093FC062DC06091F9068A
:109050007091FA068091FB069091FC0624E630E0C0
:1090600040E050E00E94CEAA0E94D5A7DC01CB01CF
:109070008093E70F9093E80FA093E90FB093EA0F66
:10908000C801880F991F880F991F800F911FAA2769
:1090900097FDA095BA2F8093F9069093FA06A093B6
:1090A000FB06B093FC060E9425A3DC01CB018C508B
:1090B0009E4FAF4FBF4F8093EE099093EF09A0935F
:1090C000F009B093F1090E948531F201828588236D
:1090D00009F48FC48091F9069091FA06A091FB06DD
:1090E000B091FC068A309105A105B10564F48AE0CF
:1090F00090E0A0E0B0E08093F9069093FA06A09388
:10910000FB06B093FC068091F9069091FA06A091B7
:10911000FB06B091FC068F3DF3E09F07F0E0AF0740
:10912000F0E0BF0764F08EED93E0A0E0B0E0809344
:10913000F9069093FA06A093FB06B093FC0682EE24
:1091400096E06DE04C2D0E943AA58091F906909131
:10915000FA069A838983CE0101960E946D3ABC017A
:1091600082EE96E00E942BA483E991E10BCFF201FD
:1091700083818823C9F082EE96E060E04FA50E94CB
:109180003AA586E991E10E94782C82EE96E06BE0A8
:109190004FA50E943AA583E090E10E947B41BC016B
:1091A00082EE96E00E942BA4F2016080772467FC97
:1091B00070948C2D90E06816790609F01AC480919D
:1091C000FD0682FF8AC0828591E0892782878823F5
:1091D00099F06091031070910410809105109091A6
:1091E000061020E030E048EC52E40E9408AA0E94F9
:1091F000A2A7DC01CB0157C06091F9067091FA0675
:109200008091FB069091FC060E94D5A720E030E0FB
:1092100048EC52E40E943AA7062FF72EE82ED92EEA
:109220006091B70F7091B80F8091B90F9091BA0FFC
:109230000E94D5A74B015C01802F9F2DAE2DBD2D27
:10924000BC01CD0120910310309104104091051014
:10925000509106100E943AA79B01AC01C501B401D0
:109260000E9408AA0E94D8A96093B70F7093B80F04
:109270008093B90F9093BA0F802F9F2DAE2DBD2DE7
:109280008093031090930410A0930510B0930610E0
:10929000C301880F991F880F991F860D971DAA2754
:1092A00097FDA095BA2F8093F9069093FA06A093A4
:1092B000FB06B093FC060E9425A3DC01CB018C5079
:1092C0009E4FAF4FBF4F8093EE099093EF09A0934D
:1092D000F009B093F1090E948531F201828588235B
:1092E00009F487C38091F9069091FA06A091FB06D4
:1092F000B091FC0685309105A105B10564F485E0C7
:1093000090E0A0E0B0E08093F9069093FA06A09375
:10931000FB06B093FC068091F9069091FA06A091A5
:10932000FB06B091FC068034F2E49F07FFE0AF0734
:10933000F0E0BF0764F08FE392E4AFE0B0E0809329
:10934000F9069093FA06A093FB06B093FC0682EE12
:1093500096E06BE04C2D0E943AA56091F906709161
:10936000FA068091FB069091FC060E94D5A720E0AA
:1093700030E048EC52E40E943AA7DC01CB018FA315
:1093800098A7A9A7BAA7CE0187962CC3F20183811B
:109390008823C9F082EE96E060E04FA50E943AA5CE
:1093A00082EA91E10E94782C82EE96E06BE04FA574
:1093B0000E943AA587E090E10E947B41BC0182EEC9
:1093C00096E00E942BA4F2016080772467FC7094E1
:1093D0008C2D90E06816790609F00BC38091FD068C
:1093E00082FF8AC0828591E089278287882399F04D
:1093F00060910710709108108091091090910A10E7
:1094000020E030E048EC52E40E9408AA0E94A2A7A3
:10941000DC01CB0157C06091F9067091FA0680918A
:10942000FB069091FC060E94D5A720E030E048ECB6
:1094300052E40E943AA7062FF72EE82ED92E60910B
:10944000BB0F7091BC0F8091BD0F9091BE0F0E9419
:10945000D5A74B015C01802F9F2DAE2DBD2DBC01EA
:10946000CD012091071030910810409109105091C2
:109470000A100E943AA79B01AC01C501B4010E94E9
:1094800008AA0E94D8A96093BB0F7093BC0F809369
:10949000BD0F9093BE0F802F9F2DAE2DBD2D8093BD
:1094A000071090930810A0930910B0930A10C301FD
:1094B000880F991F880F991F860D971DAA2797FD62
:1094C000A095BA2F8093F9069093FA06A093FB0615
:1094D000B093FC060E9425A3DC01CB018C509E4F6B
:1094E000AF4FBF4F8093EE099093EF09A093F0091F
:1094F000B093F1090E948531F2018285882309F435
:1095000078C28091F9069091FA06A091FB06B0917D
:10951000FC0685309105A105B10564F485E090E075
:10952000A0E0B0E08093F9069093FA06A093FB06C2
:10953000B093FC068091F9069091FA06A091FB0683
:10954000B091FC068034F2E49F07FFE0AF07F0E043
:10955000BF0764F08FE392E4AFE0B0E08093F906D8
:109560009093FA06A093FB06B093FC0682EE96E079
:109570006BE04C2D0E943AA56091F9067091FA06B5
:109580008091FB069091FC060E94D5A720E030E078
:1095900048EC52E40E943AA7DC01CB018BA39CA3C8
:1095A000ADA3BEA3CE0183961DC2F20183818823A1
:1095B000C9F082EE96E060E04FA50E943AA58EEADF
:1095C00091E10E94782C82EE96E06BE04FA50E941C
:1095D0003AA58BE090E10E947B41BC0182EE96E0CF
:1095E0000E942BA4F2016080772467FC70948C2D7C
:1095F00090E06816790609F0FCC18091FD0682FFB3
:109600008AC0828591E089278287882399F06091BA
:109610000B1070910C1080910D1090910E1020E0A5
:1096200030E048EC52E40E9408AA0E94A2A7DC01A4
:10963000CB0157C06091F9067091FA068091FB0644
:109640009091FC060E94D5A720E030E048EC52E45F
:109650000E943AA7062FF72EE82ED92E6091BF0F51
:109660007091C00F8091C10F9091C20F0E94D5A739
:109670004B015C01802F9F2DAE2DBD2DBC01CD0176
:1096800020910B1030910C1040910D1050910E1044
:109690000E943AA79B01AC01C501B4010E9408AA2F
:1096A0000E94D8A96093BF0F7093C00F8093C10F21
:1096B0009093C20F802F9F2DAE2DBD2D80930B1048
:1096C00090930C10A0930D10B0930E10C301880F4F
:1096D000991F880F991F860D971DAA2797FDA095A2
:1096E000BA2F8093F9069093FA06A093FB06B093E5
:1096F000FC060E9425A3DC01CB018C509E4FAF4F8E
:10970000BF4F8093EE099093EF09A093F009B093B7
:10971000F1090E948531F2018285882309F469C12B
:109720008091F9069091FA06A091FB06B091FC0693
:1097300085309105A105B10564F485E090E0A0E0D5
:10974000B0E08093F9069093FA06A093FB06B093DD
:10975000FC068091F9069091FA06A091FB06B09163
:10976000FC068034F2E49F07FFE0AF07F0E0BF079C
:1097700064F08FE392E4AFE0B0E08093F906909359
:10978000FA06A093FB06B093FC0682EE96E06BE02F
:109790004C2D0E943AA56091F9067091FA068091CD
:1097A000FB069091FC060E94D5A720E030E048EC33
:1097B00052E40E943AA7DC01CB018F8F98A3A9A3A2
:1097C000BAA3CE014F960EC1F20183818823C9F05E
:1097D00082EE96E060E04FA50E943AA58AEB91E107
:1097E0000E94782C82EE96E06BE04FA50E943AA58D
:1097F0008FE090E10E947B41BC0182EE96E00E94E6
:109800002BA4F2016080772467FC70948C2D90E08B
:109810006816790609F0EDC08091FD0682FF8AC0C6
:10982000828591E089278287882399F060910F10C3
:1098300070911010809111109091121020E030E082
:1098400048EC52E40E9408AA0E94A2A7DC01CB01C6
:1098500057C06091F9067091FA068091FB069091CD
:10986000FC060E94D5A720E030E048EC52E40E94BC
:109870003AA7062FF72EE82ED92E6091C30F7091CC
:10988000C40F8091C50F9091C60F0E94D5A74B01C0
:109890005C01802F9F2DAE2DBD2DBC01CD012091EF
:1098A0000F103091101040911110509112100E9421
:1098B0003AA79B01AC01C501B4010E9408AA0E940D
:1098C000D8A96093C30F7093C40F8093C50F909372
:1098D000C60F802F9F2DAE2DBD2D80930F1090931E
:1098E0001010A0931110B0931210C301880F991F8C
:1098F000880F991F860D971DAA2797FDA095BA2F4F
:109900008093F9069093FA06A093FB06B093FC06A9
:109910000E9425A3DC01CB018C509E4FAF4FBF4F5F
:109920008093EE099093EF09A093F009B093F109A9
:109930000E948531F2018285882309F45AC0809102
:10994000F9069091FA06A091FB06B091FC068530CD
:109950009105A105B10564F485E090E0A0E0B0E0D8
:109960008093F9069093FA06A093FB06B093FC0649
:109970008091F9069091FA06A091FB06B091FC0641
:109980008034F2E49F07FFE0AF07F0E0BF0764F028
:109990008FE392E4AFE0B0E08093F9069093FA068B
:1099A000A093FB06B093FC0682EE96E06BE04C2D94
:1099B0000E943AA56091F9067091FA068091FB0623
:1099C0009091FC060E94D5A720E030E048EC52E4DC
:1099D0000E943AA7DC01CB018B8F9C8FAD8FBE8F8D
:1099E000CE014B960E947B41BC0182EE96E00E9424
:1099F0002BA423942FA538A92F5F3F4F38AB2FA757
:109A000049A95AA94C5F5F4F5AAB49AB6BA97CA9D6
:109A10006C5F7F4F7CAB6BABCFA4F2014085842F92
:109A2000992787FD909503962FA538A96DA97EA942
:109A3000260F371F8217930714F00C941E428201E1
:109A40008285882309F090C04187C090F906D090A4
:109A5000FA06E090FB06F090FC0613828481958163
:109A6000A681B781A7019601281B390B4A0B5B0B16
:109A7000DA01C9010496A11DB11D89309105A10526
:109A8000B10508F071C082EE96E060E040810E946E
:109A90003AA582EE96E060E20E943CA4F201808545
:109AA000F7FE06C08150808787FF58C0108656C0D9
:109AB000F5E1CF16D104E104F10464F08F5FF20107
:109AC00080878F3014F08EE080879FE0C92ED12CE4
:109AD000E12CF12CC092F906D092FA06E092FB0636
:109AE000F092FC06F801C482D582E682F782C701B3
:109AF000B60125E030E040E050E00E9436ABF801CE
:109B00002083243011F483E08083F8018081823146
:109B100014F081E18083F80191858085981711F018
:109B200081E0838382EE96E060E0F80140810E944C
:109B30003AA5F8018081992787FD909520853327E4
:109B400027FD3095820F931F009711F06EE301C03F
:109B500063E082EE96E00E943CA406C084E0C82E3A
:109B6000D12CE12CF12CB6CFE6960FB6F894DEBFDF
:109B70000FBECDBFDF91CF911F910F91FF90EF905E
:109B8000DF90CF90BF90AF909F908F907F906F901D
:109B90005F904F903F902F9008952F923F924F9259
:109BA0005F926F927F928F929F92AF92BF92CF926D
:109BB000DF92EF92FF920F931F93CF93DF93CDB776
:109BC000DEB7A0970FB6F894DEBF0FBECDBF5C0125
:109BD000FC0191858085981719F48381882339F0D9
:109BE00081E0F501838382EE96E00E9468A5F5018D
:109BF00020841E8E1D8E222D332727FD309538A3FD
:109C00002F8FCAC4423009F4ACC3433034F4442328
:109C100071F0413009F0BAC43DC0443009F4FCC1D0
:109C200044300CF403C1453009F0B0C4DEC2F50184
:109C30008381882351F082EE96E060E04D8D0E9492
:109C40003AA589EA90E10E94782CF501208133271A
:109C500027FD3095832D90E02817390709F096C429
:109C60008091FD0682FF92C40E9425A3DC01CB01F6
:109C70008C509E4FAF4FBF4F8093EE099093EF09EA
:109C8000A093F009B093F10981E0F50181830E946E
:109C900085317CC4F5018381882349F182EE96E009
:109CA00060E04D8D0E943AA581EB90E10E94782CF6
:109CB00082EE96E06DE04D8D0E943AA560910A0417
:109CC00070910B04882777FD8095982F0E94D5A767
:109CD000DC01CB01898F9A8FAB8FBC8FCE01499667
:109CE0000E942A3ABC0182EE96E00E942BA4F50164
:109CF0002081332727FD3095832D90E028173907E1
:109D000009F044C48091FD0682FF3CC0828591E049
:109D100089278287882389F080910A0490910B0417
:109D2000AA2797FDA095BA2F8093F9069093FA067B
:109D3000A093FB06B093FC0615C0C901880F991FBC
:109D4000880F991F820F931FAA2797FDA095BA2FFE
:109D50008093F9069093FA06A093FB06B093FC0655
:109D60000E9485310E9425A3DC01CB018C509E4FBF
:109D7000AF4FBF4F8093EE099093EF09A093F00986
:109D8000B093F109F5018285882309F4FFC380911E
:109D9000F9069091FA06A091FB06B091FC06181600
:109DA00019061A061B0664F081E090E0A0E0B0E01E
:109DB0008093F9069093FA06A093FB06B093FC06F5
:109DC0008091F9069091FA06A091FB06B091FC06ED
:109DD0008139F1E09F07F0E0AF07F0E0BF0764F0E2
:109DE00080E991E0A0E0B0E08093F9069093FA0654
:109DF000A093FB06B093FC068091F9069091FA06B9
:109E000090930B0480930A0481E080931D0782EEF7
:109E100096E06DE0432D0E943AA58091F90690915D
:109E2000FA0698878F83CE01079698C2F501838141
:109E30008823A1F182EE96E060E04D8D0E943AA564
:109E400089EB90E10E94782C82EE96E06DE04D8DDA
:109E50000E943AA58091220A9091230A60E00E9414
:109E60006D7520E030E040E05FE30E945AA60E945A
:109E7000A2A7882777FD8095982F0E94D5A7DC019F
:109E8000CB018D8B9E8BAF8BB88FCE0145960E94F8
:109E90002A3ABC0182EE96E00E942BA4F501808153
:109EA000992787FD9095232D30E08217930709F0BD
:109EB0006DC38091FD0682FF6DC0828591E0892788
:109EC00082878823F1F08091220A9091230A60E032
:109ED0000E946D7520E030E040E05FE30E945AA6EA
:109EE0000E94A2A7DC01CB01AA2797FDA095BA2F5B
:109EF0008093F9069093FA06A093FB06B093FC06B4
:109F000039C06091F9067091FA068091FB06909134
:109F1000FC060E94D5A76B017C010E94A2A7DC0170
:109F2000CB0160E00E9422759093230A8093220A5D
:109F3000C092180AD092190AE0921A0AF0921B0AEB
:109F4000F5012081332727FD3095C901880F991F1E
:109F5000880F991F820F931FAA2797FDA095BA2FEC
:109F60008093F9069093FA06A093FB06B093FC0643
:109F70000E9485310E9425A3DC01CB018C509E4FAD
:109F8000AF4FBF4F8093EE099093EF09A093F00974
:109F9000B093F109F5018285882309F4F7C2809115
:109FA000F9069091FA06A091FB06B091FC06B7FF66
:109FB00008C01092F9061092FA061092FB06109251
:109FC000FC068091F9069091FA06A091FB06B091EB
:109FD000FC068530F1E09F07F0E0AF07F0E0BF0737
:109FE00064F084E091E0A0E0B0E08093F906909303
:109FF000FA06A093FB06B093FC0682EE96E06DE0B5
:10A00000432D0E943AA58091F9069091FA069E830D
:10A010008D83CE010596A2C1F5018381882399F134
:10A0200082EE96E060E04D8D0E943AA583EC90E1CF
:10A030000E94782C82EE96E06DE04D8D0E943AA54C
:10A040008091200A9091210A0E94DD7720E030E083
:10A0500040E05FE30E945AA60E94A2A7882777FDEE
:10A060008095982F0E94D5A7DC01CB01898B9A8B14
:10A07000AB8BBC8BCE0141960E942A3ABC0182EE8A
:10A0800096E00E942BA4F5018081992787FD909589
:10A09000232D30E08217930709F078C28091FD06E6
:10A0A00082FF61C0828591E0892782878823E9F059
:10A0B0008091200A9091210A0E94DD7720E030E013
:10A0C00040E05FE30E945AA60E94A2A7DC01CB01F8
:10A0D000AA2797FDA095BA2F8093F9069093FA06C8
:10A0E000A093FB06B093FC062EC06091F906709118
:10A0F000FA068091FB069091FC060E94D5A70E946B
:10A10000A2A7DC01CB010E946A759093210A80937B
:10A11000200AF5012081332727FD3095C901880FDA
:10A12000991F880F991F820F931FAA2797FDA0954B
:10A13000BA2F8093F9069093FA06A093FB06B0938A
:10A14000FC060E9485310E9425A3DC01CB018C50C6
:10A150009E4FAF4FBF4F8093EE099093EF09A093AE
:10A16000F009B093F109F5018285882309F40EC244
:10A170008091F9069091FA06A091FB06B091FC0639
:10A18000B7FF08C01092F9061092FA061092FB066B
:10A190001092FC068091F9069091FA06A091FB06B8
:10A1A000B091FC068530F1E09F07F0E0AF07F0E0EA
:10A1B000BF0764F084E091E0A0E0B0E08093F9068E
:10A1C0009093FA06A093FB06B093FC0682EE96E00D
:10A1D0006DE0432D0E943AA58091F9069091FA0610
:10A1E0009C838B83CE010396B9C0F50183818823BC
:10A1F00031F182EE96E060E04D8D0E943AA58AEC46
:10A2000090E10E94782C82EE96E06DE04D8D0E94E8
:10A210003AA56091FF0670E080E090E00E94D3A72D
:10A22000DC01CB018D879E87AF87B88BCE010D9661
:10A230000E942A3ABC0182EE96E00E942BA4F5010E
:10A240002081332727FD3095832D90E0281739078B
:10A2500009F09CC18091FD0682FF39C0828591E0A2
:10A2600089278287882371F08091FF0690E0A0E023
:10A27000B0E08093F9069093FA06A093FB06B093A2
:10A28000FC0615C0C901880F991F880F991F820FFE
:10A29000931FAA2797FDA095BA2F8093F906909354
:10A2A000FA06A093FB06B093FC060E9485310E943B
:10A2B00025A3DC01CB018C509E4FAF4FBF4F809345
:10A2C000EE099093EF09A093F009B093F109F5011D
:10A2D0008285882309F45AC18091F9069091FA0683
:10A2E000A091FB06B091FC06B7FF08C01092F906DA
:10A2F0001092FA061092FB061092FC068091F90665
:10A300009091FA06A091FB06B091FC068F3F910553
:10A31000A105B10569F064F08FEF90E0A0E0B0E036
:10A320008093F9069093FA06A093FB06B093FC067F
:10A330006091F9066093FF0687E070E00E9433A108
:10A3400082EE96E06DE0432D0E943AA58091F906D9
:10A350009091FA069A838983CE0101960E946D3A04
:10A3600010C1F50183818823C9F082EE96E060E098
:10A370004D8D0E943AA586ED90E10E94782C82EEE8
:10A3800096E06DE04D8D0E943AA58FE090E10E942D
:10A390007B41BC0182EE96E00E942BA4F5018080F7
:10A3A000992487FC9094832D90E08816990609F0F3
:10A3B000EDC08091FD0682FF8AC0828591E08927E9
:10A3C0008287882399F060910F107091101080910E
:10A3D00011109091121020E030E048EC52E40E94FD
:10A3E00008AA0E94A2A7DC01CB0157C06091F90620
:10A3F0007091FA068091FB069091FC060E94D5A709
:10A4000020E030E048EC52E40E943AA7C62E172F15
:10A41000082FF92E6091C30F7091C40F8091C50F62
:10A420009091C60F0E94D5A72B013C018C2D912F36
:10A43000A02FBF2DBC01CD0120910F103091101025
:10A4400040911110509112100E943AA79B01AC014B
:10A45000C301B2010E9408AA0E94D8A96093C30F49
:10A460007093C40F8093C50F9093C60F8C2D912FBE
:10A47000A02FBF2D80930F1090931010A093111058
:10A48000B0931210C401880F991F880F991F880D6F
:10A49000991DAA2797FDA095BA2F8093F90690934E
:10A4A000FA06A093FB06B093FC060E9425A3DC01EC
:10A4B000CB018C509E4FAF4FBF4F8093EE099093CE
:10A4C000EF09A093F009B093F1090E948531F501DD
:10A4D0008285882309F45AC08091F9069091FA0682
:10A4E000A091FB06B091FC0685309105A105B10550
:10A4F00064F485E090E0A0E0B0E08093F9069093EA
:10A50000FA06A093FB06B093FC068091F9069091A1
:10A51000FA06A091FB06B091FC068034F2E49F0796
:10A52000FFE0AF07F0E0BF0764F08FE392E4AFE035
:10A53000B0E08093F9069093FA06A093FB06B093DF
:10A54000FC0682EE96E06DE0432D0E943AA56091F4
:10A55000F9067091FA068091FB069091FC060E9424
:10A56000D5A720E030E048EC52E40E943AA7DC0195
:10A57000CB0189879A87AB87BC87CE0109960E9459
:10A580007B41BC0182EE96E00E942BA42D8D3E8D76
:10A590002F5F3F4F3E8F2D8F3D8C432D420DF50198
:10A5A0005085852F992787FD909503962D8D3E8D9B
:10A5B0006F8D78A1260F371F821793070CF022CBDF
:10A5C0008285882309F090C05187C090F906D09009
:10A5D000FA06E090FB06F090FC06138284819581D8
:10A5E000A681B781A7019601281B390B4A0B5B0B8B
:10A5F000DA01C9010496A11DB11D89309105A1059B
:10A60000B10508F071C082EE96E060E040810E94E2
:10A610003AA582EE96E060E20E943CA4F5018085B6
:10A62000F7FE06C08150808787FF58C0108656C04D
:10A63000F5E1CF16D104E104F10464F08F5FF50178
:10A640008087833014F082E080870FE0C02ED12C09
:10A65000E12CF12CC092F906D092FA06E092FB06AA
:10A66000F092FC06F501C482D582E682F782C7012A
:10A67000B60125E030E040E050E00E9436ABF50145
:10A680002083243011F483E08083F50180818630BB
:10A6900014F085E08083F50191858085981711F08D
:10A6A00081E0838382EE96E060E0F50140810E94C4
:10A6B0003AA5F5018081992787FD9095208533275C
:10A6C00027FD3095820F931F009711F06EE301C0B4
:10A6D00063E082EE96E00E943CA406C014E0C12E26
:10A6E000D12CE12CF12CB6CFA0960FB6F894DEBF9A
:10A6F0000FBECDBFDF91CF911F910F91FF90EF90D3
:10A70000DF90CF90BF90AF909F908F907F906F9091
:10A710005F904F903F902F900895AF92BF92CF924D
:10A72000DF92EF92FF920F931F93CF93DF93EC0191
:10A7300099858885981719F48B81882331F081E0F9
:10A740008B8382EE96E00E9468A5F88400E010E01A
:10A75000AF2CBB24A7FCB0942AC2423009F4CCC071
:10A76000433034F4442359F0413009F01EC235C05F
:10A77000433009F450C1443009F017C2E2C18B8163
:10A78000882351F082EE96E060E0402F0E943AA5C7
:10A7900089E890E10E94782C2881332727FD3095A5
:10A7A0008C2D90E02817390709F0FFC18091FD0634
:10A7B00082FFFBC10E9425A3DC01CB018C509E4F80
:10A7C000AF4FBF4F8093EE099093EF09A093F0092C
:10A7D000B093F10981E08983E6C18B818823C9F0B8
:10A7E00082EE96E060E0402F0E943AA584E990E175
:10A7F0000E94782C82EE96E06BE0402F0E943AA5F2
:10A800008DE097E00E947B41BC0182EE96E00E94C1
:10A810002BA48881992787FD90952C2D30E08217F5
:10A82000930709F0C2C18091FD0682FF38C08A8576
:10A8300091E089278A87882329F088E792E00E949F
:10A840000C291DC08CE792E00E940C292881332737
:10A8500027FD3095C901880F991F880F991F820F16
:10A86000931FAA2797FDA095BA2F8093F90690937E
:10A87000FA06A093FB06B093FC060E9485310E9465
:10A8800025A3DC01CB018C509E4FAF4FBF4F80936F
:10A89000EE099093EF09A093F009B093F1098A852E
:10A8A000882309F482C18091F9069091FA06A0915B
:10A8B000FB06B091FC06181619061A061B061CF4B6
:10A8C00080E892E006C00097A105B10561F08DE82F
:10A8D00092E00E940C291092F9061092FA0610924A
:10A8E000FB061092FC0682EE96E06BE04C2D0E9477
:10A8F0003AA58DE097E01DC18B818823C9F082EED7
:10A9000096E060E0402F0E943AA588E990E10E941D
:10A91000782C82EE96E06BE0402F0E943AA581E110
:10A9200097E00E947B41BC0182EE96E00E942BA43E
:10A930008881992787FD90952C2D30E08217930709
:10A9400009F033C18091FD0682FF38C08A8591E00D
:10A9500089278A87882329F088E792E00E940C29BA
:10A960001DC08CE792E00E940C292881332727FD27
:10A970003095C901880F991F880F991F820F931F67
:10A98000AA2797FDA095BA2F8093F9069093FA060F
:10A99000A093FB06B093FC060E9485310E9425A37C
:10A9A000DC01CB018C509E4FAF4FBF4F8093EE091F
:10A9B0009093EF09A093F009B093F1098A85882359
:10A9C00009F4F3C08091F9069091FA06A091FB0674
:10A9D000B091FC06181619061A061B061CF48BE922
:10A9E00092E006C00097A105B10561F088EA92E007
:10A9F0000E940C291092F9061092FA061092FB069A
:10AA00001092FC0682EE96E06BE04C2D0E943AA577
:10AA100081E197E08EC08B818823C9F082EE96E0B9
:10AA200060E0402F0E943AA58CE990E10E94782CCA
:10AA300082EE96E06BE0402F0E943AA585E197E018
:10AA40000E947B41BC0182EE96E00E942BA488818B
:10AA5000992787FD90952C2D30E08217930709F0F8
:10AA6000A4C08091FD0682FF38C08A8591E08927C5
:10AA70008A87882329F088E792E00E940C291DC06C
:10AA80008CE792E00E940C292881332727FD30951E
:10AA9000C901880F991F880F991F820F931FAA273A
:10AAA00097FDA095BA2F8093F9069093FA06A0938C
:10AAB000FB06B093FC060E9485310E9425A3DC01B1
:10AAC000CB018C509E4FAF4FBF4F8093EE099093B8
:10AAD000EF09A093F009B093F1098A85882309F45E
:10AAE00064C08091F9069091FA06A091FB06B0919E
:10AAF000FC06181619061A061B061CF486EB92E0D3
:10AB000006C00097A105B10561F082EC92E00E94B9
:10AB10000C291092F9061092FA061092FB06109278
:10AB2000FC0682EE96E06BE04C2D0E943AA585E192
:10AB300097E00E947B41BC0182EE96E00E942BA42C
:10AB400034C08B81882351F082EE96E060E0402F84
:10AB50000E943AA580EA90E10E94782C2881332750
:10AB600027FD30958C2D90E028173907F1F480915E
:10AB7000FD0682FF1AC00E9425A3DC01CB018C5088
:10AB80009E4FAF4FBF4F8093EE099093EF09A09374
:10AB9000F009B093F1098FEC92E00E940C2986ED48
:10ABA00092E00E940C290E9485310F5F1F4FC02E3A
:10ABB000402F4F0D5885852F992787FD9095039637
:10ABC00098012A0D3B1D821793070CF0C6CD8A858C
:10ABD000882309F088C05987C090F906D090FA06FA
:10ABE000E090FB06F090FC061B828C819D81AE817B
:10ABF000BF81A7019601281B390B4A0B5B0BDA01B9
:10AC0000C9010496A11DB11D89309105A105B105A9
:10AC100008F069C082EE96E060E048810E943AA5A3
:10AC200082EE96E060E20E943CA48885F7FE06C0B2
:10AC30008150888787FF51C018864FC035E1C31601
:10AC4000D104E104F1045CF08F5F8887823014F056
:10AC500081E08887FFE0CF2ED12CE12CF12CC0922F
:10AC6000F906D092FA06E092FB06F092FC06CC823E
:10AC7000DD82EE82FF82C701B60125E030E040E0D0
:10AC800050E00E9436AB2883243011F483E088839F
:10AC90008881853014F084E08883998588859817A9
:10ACA00011F081E08B8382EE96E060E048810E94A3
:10ACB0003AA58881992787FD90952885332727FD18
:10ACC0003095820F931F009711F06EE301C063E08F
:10ACD00082EE96E00E943CA406C0E4E0CE2ED12C89
:10ACE000E12CF12CBCCFDF91CF911F910F91FF9000
:10ACF000EF90DF90CF90BF90AF9008952F923F924A
:10AD00004F925F926F927F928F929F92AF92BF927B
:10AD1000CF92DF92EF92FF920F931F93CF93DF9327
:10AD2000CDB7DEB72E970FB6F894DEBF0FBECDBFFE
:10AD30001C01FC0183818823F1F080910A04909129
:10AD40000B04AA2797FDA095BA2F8093F90690933C
:10AD5000FA06A093FB06B093FC0682EE96E00E94F2
:10AD600068A582EE96E060E040E00E943AA58DEF93
:10AD70009FE00E94782C80911E0A90911F0A60E04B
:10AD80000E946D7520E030E040E05FE30E945AA62B
:10AD90000E94A2A78B019C0180912504909126041A
:10ADA0000817190721F4F1018381882301F182EE4C
:10ADB00096E061E040E00E943AA5B801882777FD5F
:10ADC0008095982F0E94D5A7DC01CB018B879C87AB
:10ADD000AD87BE87CE010B960E942A3ABC0182EE57
:10ADE00096E00E942BA410932604009325048091E2
:10ADF000220A9091230A60E00E946D7520E030E005
:10AE000040E05FE30E945AA60E94A2A78B019C012A
:10AE100080912704909128040817190721F4F10163
:10AE20008381882301F182EE96E065E040E00E9494
:10AE30003AA5B801882777FD8095982F0E94D5A75D
:10AE4000DC01CB018F839887A987BA87CE0107964B
:10AE50000E942A3ABC0182EE96E00E942BA4109335
:10AE60002804009327048091A4099091A509A0913A
:10AE7000A609B091A7090097A105B10509F456C02C
:10AE800082EE96E060E041E00E943AA50E9425A390
:10AE90008090A4099090A509A090A609B090A70958
:10AEA0000091030A1091040A20E030E08016910618
:10AEB000A206B306D9F150E6C52E5AEED52EE12CE6
:10AEC000F12CA70196010E9414AB29013A01C5019A
:10AED000B401A70196010E9414AB8201021B130B5F
:10AEE000C8016CE370E00E94EDAAC82E6A83CE010F
:10AEF00002960E94553ABC0182EE96E00E942BA475
:10AF000088E090E10E94782CC982CE0101960E94CF
:10AF1000553ABC0182EE96E00E942BA48BE090E1B2
:10AF20000E94782C1093040A0093030A609115077D
:10AF300070911607809117079091180720E030E074
:10AF400048EC52E40E9408AA0E94A2A78B019C012F
:10AF50008091050A9091060A0817190721F4F1015A
:10AF600083818823B9F082EE96E06AE041E00E9496
:10AF70003AA58DE090E10E94782C85E197E00E944F
:10AF80007B41BC0182EE96E00E942BA41093060A3E
:10AF90000093050A40910A0450910B045E834D838F
:10AFA00080911D07662757FD6095762F882351F005
:10AFB00010921D074093F9065093FA066093FB0622
:10AFC0007093FC068091F9069091FA06A091FB0619
:10AFD000B091FC0684179507A607B70721F4F10185
:10AFE0002381222329F19E838D838A30910524F4C5
:10AFF0008AE090E09E838D838D819E81F3E0883E80
:10B000009F0724F087EE93E09E838D838D819E8140
:10B0100090930B0480930A04AA2797FDA095BA2F5A
:10B020008093F9069093FA06A093FB06B093FC0672
:10B030008D819E812091070A3091080A821793071B
:10B0400021F4F10123812223B9F09093080A80931F
:10B05000070A82EE96E060E042E00E943AA5CE0147
:10B0600005960E946D3ABC0182EE96E00E942BA4E8
:10B0700080E190E10E94782C0AED19E08091DA09D4
:10B08000882339F182EE96E060E043E00E943AA521
:10B0900082EE96E0B8010E942BA4F80101900020F6
:10B0A000E9F73197E01BF10BCC24DD2404E110E03B
:10B0B0000E1B110909C082EE96E065E672E00E945F
:10B0C0002BA40894C11CD11CC016D106A4F3109265
:10B0D000DA0980912507882339F1C090F607D090CE
:10B0E000F707E090F807F090F907C114D104E104E4
:10B0F000F104D1F06091FE077091FF078091000884
:10B100009091010824E630E040E050E00E94CEAA91
:10B11000A70196010E9414AB022F253631F4F101EC
:10B120008381882311F416C000E082EE96E06AE085
:10B1300042E00E943AA50B831C82CE0103960E9436
:10B140006D3ABC0182EE96E00E942BA483E190E16F
:10B150000E94782CF10113822E960FB6F894DEBF70
:10B160000FBECDBFDF91CF911F910F91FF90EF9058
:10B17000DF90CF90BF90AF909F908F907F906F9017
:10B180005F904F903F902F900895EF92FF920F9312
:10B190001F93CF93DF937C018B01C4E0D0E0F701D4
:10B1A00020813181C901019691838083F8016191E9
:10B1B0008F01C9010E94E4B0219789F784E090E0F3
:10B1C000DF91CF911F910F91FF90EF900895EF9233
:10B1D000FF920F931F93CF93DF937C018B01C0E10C
:10B1E000D0E0F70120813181C901019691838083EC
:10B1F000F80161918F01C9010E94E4B0219789F79C
:10B2000080E190E0DF91CF911F910F91FF90EF903F
:10B210000895EF92FF920F931F93CF93DF937C01DA
:10B220008B01C4E0D0E0F70120813181C901019692
:10B2300091838083F80161918F01C9010E94E4B07C
:10B24000219789F784E090E0DF91CF911F910F91D2
:10B25000FF90EF9008950F931F93CF93DF93CDB797
:10B26000DEB72A970FB6F894DEBF0FBECDBF80E3DE
:10B2700090E3A0E3B0E08F839887A987BA8784E63C
:10B2800090E09A838983CE010196BE01695F7F4F6A
:10B290000E94C558CE01019663E070E10E94E75814
:10B2A000CE01019663E170E10E94E75803EF1FE0D1
:10B2B00089819A819C012F5F3F4F3A832983F8014E
:10B2C00061918F010E94E4B0F0E103301F0781F724
:10B2D000CE0101966BEE7FE00E940959CE010196E6
:10B2E00067EE7FE00E940959CE0101966FEE7FE084
:10B2F0000E940959CE01019667ED7FE00E9409592D
:10B3000003E210E189819A819C012F5F3F4F3A83CC
:10B310002983F80161918F010E94E4B0F0E10732C6
:10B320001F0781F7CE01019663EE7FE00E94095965
:10B33000CE0101966FED7FE00E940959CE01019682
:10B340006BED7FE00E940959CE01019666E374E03F
:10B350000E940959CE01019662E374E00E940959E6
:10B36000CE0101966EE274E00E94095986E590E3F1
:10B37000A5E3B0E08B839C83AD83BE8384E690E03D
:10B380009A838983CE010196BE016D5F7F4F0E9433
:10B39000C558EAE6F9E007C09091C00095FFFCCFE0
:10B3A0008093C600319684918823B1F7E5E2FFE0EF
:10B3B00007C09091C00095FFFCCF8093C6003196E6
:10B3C00084918823B1F78091C00085FFFCCF8AE08B
:10B3D0008093C6002A960FB6F894DEBF0FBECDBF8D
:10B3E000DF91CF911F910F910895EF92FF920F93EC
:10B3F0001F93CF93DF937C018B01C0E1D0E0F70175
:10B40000808191819C012F5F3F4F318320830E9477
:10B41000DCB0F80181938F01219789F780E190E0FA
:10B42000DF91CF911F910F91FF90EF900895EF92D0
:10B43000FF920F931F93CF93DF937C018B01C4E0A6
:10B44000D0E0F701808191819C012F5F3F4F3183D4
:10B4500020830E94DCB0F80181938F01219789F746
:10B4600084E090E0DF91CF911F910F91FF90EF90DA
:10B470000895AF92BF92CF92DF92EF92FF920F9317
:10B480001F93CF93DF93CDB7DEB7EA970FB6F8944B
:10B49000DEBF0FBECDBFD82E84E690E09A838983AD
:10B4A00086E590E3A5E3B0E08B839C83AD83BE8308
:10B4B0001BE0E12EF12CEC0EFD1E8E01095F1F4FEB
:10B4C00089819A819C012F5F3F4F3A8329830E9493
:10B4D000DCB0F80181938F01EE15FF0589F7DD20BF
:10B4E00009F097C0CE010396BE01695F7F4F43E02C
:10B4F00050E00E946EAE009709F08BC0CE0101961D
:10B5000063E070E10E94F559CE01019663E170E1BC
:10B510000E94F55903EF1FE089819A819C012F5FFA
:10B520003F4F3A8329830E94DCB0F80181938F0159
:10B53000F0E103301F0781F7CE0101966BEE7FE04B
:10B540000E94175ACE01019667EE7FE00E94175ABB
:10B55000CE0101966FEE7FE00E94175ACE01019650
:10B5600067ED7FE00E94175A03E210E189819A811A
:10B570009C012F5F3F4F3A8329830E94DCB0F80182
:10B5800081938F01F0E107321F0781F7CE01019609
:10B5900063EE7FE00E94175ACE0101966FED7FE0C7
:10B5A0000E94175ACE0101966BED7FE00E94175A58
:10B5B000CE01019666E374E00E94175ACE0101960F
:10B5C00062E374E00E94175ACE0101966EE274E0C5
:10B5D0000E94175AEAE6F9E007C09091C00095FF73
:10B5E000FCCF8093C600319684918823B1F7E2E8BE
:10B5F000FAE007C09091C00095FFFCCF8093C60091
:10B60000319684918823B1F78091C00085FFFCCFEB
:10B61000CEC0DE019B96E9EFF2E080E101900D9251
:10B620008150E1F7DE015B96E9E0F3E080E1019013
:10B630000D928150E1F7DE011B96E9E1F3E080E134
:10B6400001900D928150E1F76BE2A62EB12CAC0E69
:10B65000BD1E43E050E1BE01655E7F4F03E110E196
:10B66000EBE0EE2EF12CEC0EFD1EF3EFCF2EFFE003
:10B67000DF2E24E030E0F50181919191A191B1910B
:10B680005F01FA0181939193A193B193AF01FB0103
:10B6900081919191A191B191BF01F8018193919311
:10B6A000A193B1938F01F70181919191A191B191F2
:10B6B0007F01F60181939193A193B1936F01215082
:10B6C0003040C9F680E090E8ABE3B5E48093EB0F3F
:10B6D0009093EC0FA093ED0FB093EE0F8093E70FD4
:10B6E0009093E80FA093E90FB093EA0F80E090E009
:10B6F000A0E0B0E08093EF0F9093F00FA093F10FD4
:10B70000B093F20F40E25EE460E070E040932310FB
:10B710005093241060932510709326108093D70FB8
:10B720009093D80FA093D90FB093DA0F80E090E0F8
:10B73000A0EAB1E48093E30F9093E40FA093E50FA8
:10B74000B093E60F8DEC9CECACECBEE38093DF0F86
:10B750009093E00FA093E10FB093E20F80E090E0B0
:10B76000A0EAB0E48093DB0F9093DC0FA093DD0F91
:10B77000B093DE0FEAE6F9E007C09091C00095FFB4
:10B78000FCCF8093C600319684918823B1F7E1EE17
:10B79000F2E006C09091C00095FFFCCF8093C600F8
:10B7A00081918823B9F78091C00085FFFCCF8AE0A2
:10B7B0008093C6000E941825EA960FB6F894DEBF63
:10B7C0000FBECDBFDF91CF911F910F91FF90EF90F2
:10B7D000DF90CF90BF90AF900895AF92BF92CF927D
:10B7E000DF92EF92FF920F931F93CF93DF93EC01C1
:10B7F00099858885981719F48B81882331F081E029
:10B800008B8382EE96E00E9468A5F88400E010E049
:10B81000AF2CBB24A7FCB09497E0E92E26E0D22EF3
:10B820002FC1423009F46FC0433034F4442371F027
:10B83000413009F023C138C0443009F4C1C044305C
:10B840000CF48EC0453009F019C1E9C08B81882302
:10B8500051F082EE96E060E0402F0E943AA586EC1F
:10B8600091E10E94782C2881332727FD30958C2D7B
:10B8700090E02817390709F001C18091FD0682FF89
:10B88000FDC00E9425A3DC01CB018C509E4FAF4F21
:10B89000BF4F8093EE099093EF09A093F009B09306
:10B8A000F10981E089832CC08B81882351F082EEDD
:10B8B00096E060E0402F0E943AA585ED91E10E945C
:10B8C000782C2881332727FD30958C2D90E0281780
:10B8D000390709F0D3C08091FD0682FFCFC00E94D6
:10B8E00025A3DC01CB018C509E4FAF4FBF4F8093FF
:10B8F000EE099093EF09A093F009B093F109D98272
:10B900000E948531BBC08B81882351F082EE96E086
:10B9100060E0402F0E943AA584EE91E10E94782CCD
:10B920002881332727FD30958C2D90E02817390783
:10B9300009F0A4C08091FD0682FFA0C00E9425A34B
:10B94000DC01CB018C509E4FAF4FBF4F8093EE096F
:10B950009093EF09A093F009B093F109E982D0CF59
:10B960008B81882351F082EE96E060E0402F0E94A8
:10B970003AA583EF91E10E94782C2881332727FD97
:10B9800030958C2D90E02817390709F077C0809109
:10B99000FD0682FF73C00E9485310E9425A3DC0151
:10B9A000CB018C509E4FAF4FBF4F8093EE099093C9
:10B9B000EF09A093F009B093F1090E942B595EC0E2
:10B9C0008B81882351F082EE96E060E0402F0E9448
:10B9D0003AA581E092E10E94782C2881332727FD47
:10B9E00030958C2D90E02817390709F047C08091D9
:10B9F000FD0682FF43C00E9485310E9425A3DC0121
:10BA0000CB018C509E4FAF4FBF4F8093EE09909368
:10BA1000EF09A093F009B093F10980E02DC08B816C
:10BA2000882351F082EE96E060E0402F0E943AA514
:10BA30008EE092E10E94782C2881332727FD3095F3
:10BA40008C2D90E028173907C9F48091FD0682FFFC
:10BA500015C00E9485310E9425A3DC01CB018C50CA
:10BA60009E4FAF4FBF4F8093EE099093EF09A09385
:10BA7000F009B093F10981E00E94395A0F5F1F4F1E
:10BA8000C02E402F4F0D5885852F992787FD909503
:10BA9000039698012A0D3B1D821793070CF0C1CE27
:10BAA0008A85882309F088C05987C090F906D0900C
:10BAB000FA06E090FB06F090FC061B828C819D81CB
:10BAC000AE81BF81A7019601281B390B4A0B5B0B86
:10BAD000DA01C9010496A11DB11D89309105A105A6
:10BAE000B10508F069C082EE96E060E048810E94EE
:10BAF0003AA582EE96E060E20E943CA48885F7FEBB
:10BB000006C08150888787FF51C018864FC035E135
:10BB1000C316D104E104F1045CF08F5F88878330A1
:10BB200014F082E088878FE0C82ED12CE12CF12C14
:10BB3000C092F906D092FA06E092FB06F092FC065B
:10BB4000CC82DD82EE82FF82C701B60125E030E0C3
:10BB500040E050E00E9436AB2883243011F483E0AB
:10BB600088838881863014F085E08883998588856C
:10BB7000981711F081E08B8382EE96E060E04881B7
:10BB80000E943AA58881992787FD909528853327BB
:10BB900027FD3095820F931F009711F06EE301C0CF
:10BBA00063E082EE96E00E943CA406C004E0C02E52
:10BBB000D12CE12CF12CBCCFDF91CF911F910F91B3
:10BBC000FF90EF90DF90CF90BF90AF900895CF920D
:10BBD000DF92EF92FF92CF93DF93EC0189B1992727
:10BBE00087FD9095809590958827990F881F9927B4
:10BBF00020910A0A30E082179307D1F081E08B830D
:10BC000089B18095881F8827881F80930A0A0E941F
:10BC1000B93184E297E04F9905C00E947C8381EBA3
:10BC200092E104C00E945F848FEB92E10E94A42CF9
:10BC3000898190912904891769F091E09B83109282
:10BC4000F9061092FA061092FB061092FC0618866E
:10BC5000809329044091F9065091FA066091FB0601
:10BC60007091FC068C819D81AE81BF814817590778
:10BC70006A077B0721F48091FD0682FF10C00E94B5
:10BC800025A3DC01CB018856954CAF4FBF4F809365
:10BC90000B0A90930C0AA0930D0AB0930E0A8981A7
:10BCA000833009F44FC0843028F48130D9F18230D8
:10BCB000F0F50DC0853009F455C0853008F446C054
:10BCC000863009F44BC0873009F04FC043C0CE0125
:10BCD0000E947E568091FD0682FF47C01A860E9410
:10BCE00025A3DC01CB018C509E4FAF4FBF4F8093FB
:10BCF000EE099093EF09A093F009B093F10981E068
:10BD000089830E9425A3DC01CB018856954CAF4F57
:10BD1000BF4F80930B0A90930C0AA0930D0AB09327
:10BD20000E0A23C0CE010E9442381A861EC08B859F
:10BD3000882321F0CE010E94CD4D17C0CE010E9474
:10BD4000B03213C0CE010E948D530FC0CE010E94AD
:10BD5000ED5B0BC0CE010E94D24107C0CE010E9414
:10BD6000233B03C0CE010E949435C0900B0AD090B3
:10BD70000C0AE0900D0AF0900E0A0E9425A3DC0147
:10BD8000CB01C816D906EA06FB0608F41982809191
:10BD9000F9069091FA06A091FB06B091FC068C83FF
:10BDA0009D83AE83BF83DF91CF91FF90EF90DF90B3
:10BDB000CF900895CF92DF92EF92FF920E9425A339
:10BDC0006B017C014091EE095091EF096091F009FF
:10BDD0007091F10980E090E0E1E0F0E0C416D50652
:10BDE000E606F7066CF4A091FD069F01082E02C03E
:10BDF000220F331F0A94E2F720952A232093FD0691
:10BE000001968830910551F79091FD068091F209D5
:10BE10009817A9F40E9425A3DC01CB014091F309F6
:10BE20005091F4096091F5097091F609841B950B06
:10BE3000A60BB70B84369105A105B105A0F0809142
:10BE4000FD068093F2090E9425A3DC01CB018093BB
:10BE5000F3099093F409A093F509B093F60987EFDD
:10BE600099E00E94E75DFF90EF90DF90CF900895FA
:10BE70002F923F924F925F926F927F928F929F92FA
:10BE8000AF92BF92CF92DF92EF92FF920F931F93E8
:10BE9000CF93DF93CDB7DEB7A2970FB6F894DEBF8E
:10BEA0000FBECDBF87E40E94A629882309F4DAC516
:10BEB0000E948A290E94A2A76430710509F441C03A
:10BEC0006530710554F46230710541F163307105DC
:10BED0006CF577FF19C00C9432726A35710509F45C
:10BEE00068C56B35710534F46C31710511F00C9433
:10BEF000327274C06B35710509F45FC56C3571051C
:10BF000011F00C9432725EC58091FE06882331F4E4
:10BF10000E941C2A0E94D42A0C947D728091FE06F5
:10BF2000882321F40E94A52A81E007C08091FE06A3
:10BF3000882339F40E94A52A80E00E94762B0C9475
:10BF40007D7280E89DE00E94A42C80E50E94A629D5
:10BF5000882339F00E948A290E94A7A76B017C01DF
:10BF600003C0CC24DD24760183E50E94A629882322
:10BF700061F00E948A2920E030E04AE754E40E9400
:10BF800008AA0E94A7A76B017C010E948B160E9441
:10BF900025A34B015C018C0C9D1CAE1CBF1C0E9498
:10BFA00025A3DC01CB018093A8099093A909A09354
:10BFB000AA09B093AB0907C00E94BE7581E00E9438
:10BFC0002A2D0E94DA5E0E9425A3DC01CB01881590
:10BFD0009905AA05BB0580F30C94327280911C046C
:10BFE00090911D04A0911E04B0911F048093AC0990
:10BFF0009093AD09A093AE09B093AF0980910A0464
:10C0000090910B0490931F0780931E0784E690E0A5
:10C0100090930B0480930A040E9425A3DC01CB01BA
:10C020008093A8099093A909A093AA09B093AB099A
:10C0300081E00E94200F80910D0790910E07A09142
:10C040000F07B09110078093B0099093B109A093A6
:10C05000B209B093B3098091110790911207A09192
:10C060001307B09114078093B4099093B509A09376
:10C07000B609B093B7098091150790911607A09162
:10C080001707B09118078093B8099093B909A09346
:10C09000BA09B093BB098091190790911A07A09132
:10C0A0001B07B0911C078093BC099093BD09A09316
:10C0B000BE09B093BF0980E090E0A0E0B0E08093BB
:10C0C0001C0490931D04A0931E04B0931F0488E5E4
:10C0D0000E94A629882361F489E50E94A629882365
:10C0E00039F48AE50E94A629882311F481E001C071
:10C0F00080E080932004882361F488E50E94A629CB
:10C10000882309F4E8C089E50E94A629882309F458
:10C11000E2C080E090E0A0E0B0E080930D07909353
:10C120000E07A0930F07B093100780931107909309
:10C130001207A0931307B09314078DE097E061E115
:10C1400077E045E157E029E137E00E94D39E80E0A7
:10C1500090ECA9E9B3EC8093B0099093B109A09356
:10C16000B209B093B3098093B4099093B509A09331
:10C17000B609B093B70920910C0430910D04409199
:10C180000E0450910F0420931C0430931D0440931F
:10C190001E0450931F04C0901004D0901104E0902E
:10C1A0001204F0901304C701B6010E9433A787FF61
:10C1B00008C0C0921C04D0921D04E0921E04F092AC
:10C1C0001F0460911C0470911D0480911E049091C5
:10C1D0001F0420E030E040E752E40E943AA77B01D0
:10C1E0008C0180EB99E064EB79E048EB59E02CEBB3
:10C1F00039E0F0E0CF2EF7E0DF2E0E940C940E9491
:10C200008B160F2EF0E08F2EF0E09F2EF0E0AF2E79
:10C21000F0E0BF2EF02D80920D0790920E07A092B5
:10C220000F07B09210078092110790921207A09208
:10C230001307B09214078DE097E061E177E045E1E4
:10C2400057E029E137E00E94D39E80910D0790913D
:10C250000E07A0910F07B09110078093B00990933B
:10C26000B109A093B209B093B309809111079091DD
:10C270001207A0911307B09114078093B40990930B
:10C28000B509A093B609B093B70960911C047091E9
:10C290001D0480911E0490911F0420E030E040E7CF
:10C2A00052E40E943AA77B018C0180EB99E064EB99
:10C2B00079E048EB59E02CEB39E00E940C94809235
:10C2C0001C0490921D04A0921E04B0921F040E94B0
:10C2D0008B160E94190F80912004882331F488E581
:10C2E0000E94A629882309F4E7C00F2EF0E08F2EC4
:10C2F000F0E09F2EF0E0AF2EF0E0BF2EF02D809208
:10C300000D0790920E07A0920F07B09210078DE0D4
:10C3100097E061E177E045E157E029E137E00E94ED
:10C32000D39E80E090ECA9E9B3EC8093B0099093A0
:10C33000B109A093B209B093B30960910C04709154
:10C340000D0480910E0490910F0460931C0470936F
:10C350001D0480931E0490931F0420E030E040E70A
:10C3600052E40E943AA77B018C0180EB99E064EBD8
:10C3700079E048EB59E02CEB39E0E0E0CE2EE7E045
:10C38000DE2E0E940C940E948B1680920D079092D4
:10C390000E07A0920F07B09210078DE097E061E1C1
:10C3A00077E045E157E029E137E00E94D39E80E045
:10C3B00090E0A0EAB0E48093B0099093B109A09313
:10C3C000B209B093B30960911C0470911D0480916F
:10C3D0001E0490911F0420E030E040E752E40E94E8
:10C3E0003AA77B018C0180EB99E064EB79E048EBA4
:10C3F00059E02CEB39E00E940C940E948B1680E0EF
:10C4000090E0A0E2B1EC8093B0099093B109A093C1
:10C41000B209B093B30960910C0470910D0480913E
:10C420000E0490910F0420E030E040E05FE30E94B2
:10C4300008AA9B01F82FE92F462F532F682F792F39
:10C4400040931C0450931D0460931E0470931F04BA
:10C45000822F932FAF2FBE2FBC01CD0120E030E003
:10C4600040E752E40E943AA77B018C0180EB99E0FF
:10C4700064EB79E048EB59E02CEB39E00E940C9436
:10C480000E948B1680920D0790920E07A0920F07C4
:10C49000B09210078092B0099092B109A092B209AF
:10C4A000B092B30980921C0490921D04A0921E04C5
:10C4B000B0921F040E94190F80912004882331F448
:10C4C00089E50E94A629882309F4E7C00F2EF0E031
:10C4D0008F2EF0E09F2EF0E0AF2EF0E0BF2EF02D7B
:10C4E0008092110790921207A0921307B09214073E
:10C4F0008DE097E061E177E045E157E029E137E041
:10C500000E94D39E80E090ECA9E9B3EC8093B4093B
:10C510009093B509A093B609B093B7096091100440
:10C5200070911104809112049091130460931C0483
:10C5300070931D0480931E0490931F0420E030E04C
:10C5400040E752E40E943AA77B018C0180EB99E01E
:10C5500064EB79E048EB59E02CEB39E0F0E0CF2ECA
:10C56000F7E0DF2E0E940C940E948B168092110738
:10C5700090921207A0921307B09214078DE097E0F3
:10C5800061E177E045E157E029E137E00E94D39E81
:10C5900080E090E0A0EAB0E48093B4099093B509FC
:10C5A000A093B609B093B70960911C0470911D0463
:10C5B00080911E0490911F0420E030E040E752E497
:10C5C0000E943AA77B018C0180EB99E064EB79E053
:10C5D00048EB59E02CEB39E00E940C940E948B163A
:10C5E00080E090E0A0E2B1EC8093B4099093B509AB
:10C5F000A093B609B093B70960911004709111042B
:10C60000809112049091130420E030E040E05FE359
:10C610000E9408AA9B01F82FE92F462F532F682F5D
:10C62000792F40931C0450931D0460931E04709353
:10C630001F04822F932FAF2FBE2FBC01CD0120E00E
:10C6400030E040E752E40E943AA77B018C0180EB86
:10C6500099E064EB79E048EB59E02CEB39E00E947B
:10C660000C940E948B168092110790921207A09250
:10C670001307B09214078092B4099092B509A09262
:10C68000B609B092B70980921C0490921D04A09242
:10C690001E04B0921F040E94190F80912004882369
:10C6A00031F48AE50E94A629882309F4E7C00F2EF9
:10C6B000F0E08F2EF0E09F2EF0E0AF2EF0E0BF2EE6
:10C6C000F02D8092150790921607A0921707B0924E
:10C6D00018078DE097E061E177E045E157E029E157
:10C6E00037E00E94D39E80E090E0A6E9B3EC80930F
:10C6F000B8099093B909A093BA09B093BB096091A6
:10C70000140470911504809116049091170460939D
:10C710001C0470931D0480931E0490931F0420E05A
:10C7200030E040E752E40E943AA77B018C0180EBA5
:10C7300099E064EB79E048EB59E02CEB39E0E0E07C
:10C74000CE2EE7E0DE2E0E940C940E948B16809283
:10C75000150790921607A0921707B09218078DE060
:10C7600097E061E177E045E157E029E137E00E9499
:10C77000D39E80E090E0A0E8BFE38093B809909357
:10C78000B909A093BA09B093BB0960911C047091D8
:10C790001D0480911E0490911F0420E030E040E7CA
:10C7A00052E40E943AA77B018C0180EB99E064EB94
:10C7B00079E048EB59E02CEB39E00E940C940E94A0
:10C7C0008B1680E090E0A0E0B0EC8093B8099093E5
:10C7D000B909A093BA09B093BB0960911404709190
:10C7E0001504809116049091170420E030E040E099
:10C7F0005FE30E9408AA9B01F82FE92F462F532FD1
:10C80000682F792F40931C0450931D0460931E04DD
:10C8100070931F04822F932FAF2FBE2FBC01CD0129
:10C8200020E030E040E752E40E943AA77B018C010F
:10C8300080EB99E064EB79E048EB59E02CEB39E0D0
:10C840000E940C940E948B168092150790921607F6
:10C85000A0921707B09218078092B8099092B90970
:10C86000A092BA09B092BB0980921C0490921D0458
:10C87000A0921E04B0921F040E94190F88E50E9426
:10C88000A6298823F1F00E949A29DC01CB010097A8
:10C89000A105B105B1F00E948A29209101073091CC
:10C8A000020740910307509104070E945AA6DC0139
:10C8B000CB0180930D0790930E07A0930F07B093C1
:10C8C000100789E50E94A6298823F1F00E949A2981
:10C8D000DC01CB010097A105B105B1F00E948A29C6
:10C8E00020910507309106074091070750910807EE
:10C8F0000E945AA6DC01CB01809311079093120786
:10C90000A0931307B09314078AE50E94A6298823F1
:10C91000F1F00E949A29DC01CB010097A105B10535
:10C92000B1F00E948A292091090730910A074091AD
:10C930000B0750910C070E945AA6DC01CB01809393
:10C94000150790931607A0931707B09318078DE06B
:10C9500097E061E177E045E157E029E137E00E94A7
:10C96000D39E8091AC099091AD09A091AE09B09190
:10C97000AF0980931C0490931D04A0931E04B093F0
:10C980001F0480911E0790911F0790930B048093C2
:10C990000A040E9425A3DC01CB018093A80990938F
:10C9A000A909A093AA09B093AB090E94190F0C948E
:10C9B00032721092C0090C94327281E08093C009E7
:10C9C0000C94327285E40E94A629882311F40E94F7
:10C9D0008B1645E4842E44E0942E51E0C52E57E09A
:10C9E000D52E6DE0E62E67E0F62E00E0F401819191
:10C9F0004F010E94A629882351F1033071F40E944F
:10CA00008A29DC01CB01F70180839183A283B38360
:10CA100089E197E00E94839F1AC00E948A29F6014B
:10CA200020813181428153810E945AA6DC01CB01D1
:10CA3000F70180839183A283B3838DE097E061E166
:10CA400077E045E157E029E137E00E94D39E0F5F90
:10CA500024E030E0C20ED31EE20EF31E043031F6A5
:10CA60000C9432728DE40E94A629882311F40C9450
:10CA700084710E948A290E94A2A76A36710509F46E
:10CA800003C76B3671050CF080C06C31710509F479
:10CA900024C26D317105C4F56531710509F4BCC15D
:10CAA00066317105BCF46131710509F480C16231F0
:10CAB000710534F46230710510F00C94327212C1B9
:10CAC0006231710509F41AC76431710511F00C94D3
:10CAD000327277C16831710509F4BFC169317105DE
:10CAE00054F46631710509F49DC16731710511F087
:10CAF0000C9432729DC16A31710509F4C6C16B3163
:10CB000071050CF0E4C1BBC16235710509F4EFC6D3
:10CB100063357105DCF46A32710509F4CCC26B32FD
:10CB2000710554F46E31710509F40FC26F3171054E
:10CB300011F00C9432724AC26035710509F4CFC607
:10CB40006135710511F00C943272CCC665357105F2
:10CB500009F421C76635710554F46335710509F48C
:10CB6000C9C66435710511F00C943272C7C66836B7
:10CB7000710509F4E8C2693671050CF05BC36C35C8
:10CB8000710511F00C9432721EC76C3C710511F4E2
:10CB90000C94996F6D3C71050CF047C067377105B7
:10CBA00011F40C94836E68377105E4F462377105F3
:10CBB00011F40C94A16D6337710554F46B36710553
:10CBC00009F48AC66D36710511F00C94327204C4F2
:10CBD0006337710509F495C76537710511F00C9439
:10CBE00032729DC76C38710509F40FC36D38710539
:10CBF00064F46837710511F40C947D6E6937710522
:10CC000011F00C9432720C947F6E693C710511F432
:10CC10000C943D6F6B3C710511F40C947B6F6E3B73
:10CC2000710511F00C94327283C531E06F327307D5
:10CC300011F40C94517181E0603378073CF56C3D40
:10CC4000710511F40C9445706D3D710564F46D3CF3
:10CC5000710511F40C94BD6F6E3C710511F00C94CC
:10CC600032720C94277091E06D32790711F40C94B4
:10CC70006A70E1E06E327E0714F00C944D716D3DE8
:10CC8000710511F00C9432720C945970F1E0653F0B
:10CC90007F0711F40C94667121E0663F720774F40B
:10CCA00031E06039730711F40C94607181E0643FE6
:10CCB000780711F00C9432720C94637191E0673F25
:10CCC000790711F40C946C71E1E0673F7E0714F46E
:10CCD0000C946871F3E0673E7F0711F00C94327298
:10CCE0000C946F7189E89DE00E94A42C80E50E945D
:10CCF000A629882339F00E948A290E94A7A76B01E0
:10CD00007C0103C0CC24DD24760183E50E94A629A2
:10CD1000882361F00E948A2920E030E04AE754E449
:10CD20000E9408AA0E94A7A76B017C010E948B1693
:10CD30000E9425A3DC01CB018093A8099093A90947
:10CD4000A093AA09B093AB09C114D104E104F10482
:10CD500041F10E9425A34B015C018C0C9D1CAE1C73
:10CD6000BF1C0E9425A3DC01CB0188159905AA05EB
:10CD7000BB0510F00C9432728091FD0682FF02C058
:10CD80000C9432720E94BE7581E00E942A2D0E948E
:10CD9000DA5EE7CF0E94BE7581E00E942A2D0E94D4
:10CDA000DA5E8091FD0682FFF5CF0C9432728AE93B
:10CDB0009DE00E94A42C159817984298A0980C9476
:10CDC0003272E3EAFDE007C09091C00095FFFCCF0E
:10CDD0008093C600319684918823B1F78091C0007A
:10CDE00085FFFCCF8AE08093C60084E297E00E9432
:10CDF0003983E3EBFDE007C09091C00095FFFCCFC5
:10CE00008093C600319684918823B1F78091C00049
:10CE100085FFFCCF0C942F7284E297E00E947C8304
:10CE20000C94327284E297E00E945F840C94327218
:10CE300000919609109197090C5F1F4FC8016AE293
:10CE400070E00E945CAE009719F00197FC0110821F
:10CE500084E297E0B80141E074C084E297E00E9468
:10CE600063840E9425A3DC01CB018093A4099093E5
:10CE7000A509A093A609B093A7090C94327284E285
:10CE800097E00E946A840C9432728091260788236E
:10CE900011F40C94327283E50E94A629882311F4C0
:10CEA0000C9432720E949A29AB01382F292F60937B
:10CEB000FE075093FF0780930008909301088BEDC5
:10CEC00097E0632F722F0E94971A0C94327284E2BB
:10CED00097E00E94AC870C943272809196099091F1
:10CEE000970904966AE270E00E945CAE8C0100979C
:10CEF000F9F0209190093091910940E650E0249F8B
:10CF0000C001259F900D349F900D1124845F974F91
:10CF10006EE470E00E945CAE60E270E00E945CAE85
:10CF200001969093970980939609F80131971082A2
:10CF300060919609709197096C5F7F4F84E297E04A
:10CF400040E00E946F840C943272809126078823FF
:10CF500011F40C94327284E297E00E9484898091EB
:10CF600096099091970904966AE270E00E945CAE7F
:10CF70008C010097F9F0209190093091910940E6D9
:10CF800050E0249FC001259F900D349F900D1124E7
:10CF9000845F974F6EE470E00E945CAE60E270E0E8
:10CFA0000E945CAE01969093970980939609F801D0
:10CFB0003197108260919609709197096C5F7F4F4D
:10CFC00084E297E00E9468860C9432720E9425A346
:10CFD000DC01CB018093A0099093A109A093A20941
:10CFE000B093A3094091A4095091A5096091A609A5
:10CFF0007091A709841B950BA60BB70BBC01CD0143
:10D0000028EE33E040E050E00E9414AB8DB79EB7AD
:10D0100008970FB6F8949EBF0FBE8DBF0DB71EB711
:10D020000F5F1F4FCE010196EDB7FEB7928381834C
:10D0300089E192E0F80193838283CA01B9012CE36C
:10D0400030E040E050E00E9414ABDC01CB01F8017D
:10D0500035832483978386830E94A5AEEAE6F9E0B0
:10D0600084912DB73EB7285F3F4F0FB6F8943EBF6F
:10D070000FBE2DBF08C09091C00095FFFCCF8093DC
:10D08000C600319684918823B1F7FE01319606C01F
:10D090009091C00095FFFCCF8093C60081918823BA
:10D0A000B9F78091C00085FFFCCF8AE08093C6006D
:10D0B000CE01019643C583E50E94A629882311F479
:10D0C0000C9432720E948A296B017C0180E50E94D7
:10D0D000A629882311F40C943272C701B6010E946C
:10D0E000A2A7DC01CB017C0197FF02C00C94327235
:10D0F0008F3F910519F014F00C9432720E948A2926
:10D100000E94A2A78B019C01E9E4F4E020E0819158
:10D1100091918017910711F40C9432722F5F2A338A
:10D12000B1F717FF02C00C943272802F61E00E94A9
:10D1300083A2802F6E2D0E94A4A2802FB7010E948F
:10D1400033A10C943272809100078093C10984E569
:10D150000E94A629882379F10E948A290E94A7A704
:10D160006093C109662339F1EAE6F9E007C09091BE
:10D17000C00095FFFCCF8093C60031968491882330
:10D18000B1F7EFE2F3E006C09091C00095FFFCCF4D
:10D190008093C60081918823B9F78FE59AE060916A
:10D1A000C10940E050E00E94F27F8091C00085FFFD
:10D1B000FCCF0C942F7283E50E94A629882309F1E5
:10D1C0000E948A296B017C010091C109802E99245B
:10D1D0000E94A2A7DC01CB01602F0E942275F401FE
:10D1E000EE0FFF1FEE5DF54F91838083F401EE0F8C
:10D1F000FF1FEE0FFF1FE85EF54FC082D182E28273
:10D20000F3820E9444780C94327283E50E94A6292E
:10D21000882311F40C9432720E948A290E94A2A7DA
:10D22000DC01CB010E946A759093210A8093200A49
:10D230000C943272809100078093C10984E50E94AA
:10D24000A629882379F10E948A290E94A7A76093C2
:10D25000C109662339F1EAE6F9E007C09091C00000
:10D2600095FFFCCF8093C600319684918823B1F757
:10D27000E6E4F3E006C09091C00095FFFCCF8093F8
:10D28000C60081918823B9F78FE59AE06091C109C2
:10D2900040E050E00E94F27F8091C00085FFFCCF0B
:10D2A0000C942F72E1ECFDE007C09091C00095FF57
:10D2B000FCCF8093C600319684918823B1F76091AA
:10D2C000C109E62FF0E0EE0FFF1FE25EF54F80810F
:10D2D00091810E946D75AB01BC018FE59AE021E060
:10D2E00030E00E942B81E7ECFDE007C09091C00088
:10D2F00095FFFCCF8093C600319684918823B1F7C7
:10D300006091C109E62FF0E0EE0FFF1FEE5DF54FD3
:10D31000808191810E946D75AB01BC018FE59AE01F
:10D3200021E030E00E942B81EAECFDE007C0909103
:10D33000C00095FFFCCF8093C6003196849188236E
:10D34000B1F780911C0A90911D0A0E94DD77AB0114
:10D35000BC018FE59AE021E030E00E942B81EEECE9
:10D36000FDE007C09091C00095FFFCCF8093C60000
:10D37000319684918823B1F78091200A9091210AF7
:10D380000E94DD77AB01BC018FE59AE021E030E03F
:10D390000E942B81E1EDFDE007C09091C00095FF58
:10D3A000FCCF8093C600319684918823B1F7809199
:10D3B000C10990E00E941C75BC018FE59AE04AE02B
:10D3C00050E00E942F808091C00085FFFCCF8AE052
:10D3D0008093C6000C947D72809100078093C109F0
:10D3E00084E50E94A629882379F10E948A290E9457
:10D3F000A7A76093C109662339F1EAE6F9E007C0FF
:10D400009091C00095FFFCCF8093C6003196849127
:10D410008823B1F7EDE5F3E006C09091C00095FFD9
:10D42000FCCF8093C60081918823B9F78FE59AE0FD
:10D430006091C10940E050E00E94F27F8091C000FD
:10D4400085FFFCCF0C942F7285ED9DE00E94A42CEB
:10D4500083E50E94A629882309F10E948A296B018D
:10D460007C010091C109802E99240E94A2A7DC01B1
:10D47000CB01602F0E942275F401EE0FFF1FEE5DBD
:10D48000F54F91838083F401EE0FFF1FEE0FFF1F16
:10D49000E85EF54FC082D182E282F3820E94447836
:10D4A0000E9425A32B013C018091C10990E0880FC7
:10D4B000991FFC01EE5DF54F2081318138A32F8F3C
:10D4C000825E954FFC010190F081E02DFAA3E9A363
:10D4D00088248A94982C5401E0EEFDE03490E3EE29
:10D4E000FDE02490E7EEFDE004911AE00FC1832DEA
:10D4F000E0EEFDE008C09091C00095FFFCCF809366
:10D50000C600319684918823B1F76091C109E62F56
:10D51000F0E0EE0FFF1FE25EF54F808191810E94E7
:10D520006D75AB01BC018FE59AE021E030E00E940F
:10D530002B81822DE3EEFDE008C09091C00095FFA5
:10D54000FCCF8093C600319684918823B1F7609117
:10D55000C1098FE59AE070E04AE050E00E942F8018
:10D56000802FE7EEFDE008C09091C00095FFFCCF52
:10D570008093C600319684918823B1F7B7FE03C02B
:10D58000E4E7F3E029C00E9425A3AB01BC01D5016B
:10D59000C40188579C4EAF4FBF4F841B950BA60B01
:10D5A000B70BBC01CD0128EE33E040E050E00E9413
:10D5B00014AB8FE59AE0BA01A9012AE030E00E949D
:10D5C000E57F8091C00085FFFCCF0DC09091C00029
:10D5D00095FFFCCF8093C60081918823B9F7809195
:10D5E000C00085FFFCCF1093C6000E9425A32B012D
:10D5F0003C010E94BE7581E00E942A2D0E94DA5EE5
:10D60000FFEF8F16FFEF9F06FFEFAF06FFEFBF069E
:10D6100089F56091C1092F8D38A189A19AA1E62FC2
:10D62000F0E0EE0FFF1FE25EF54F821793070CF05C
:10D6300042C7808191810E946D756B017C01609170
:10D64000C109E62FF0E0EE0FFF1FEE5DF54F808180
:10D6500091810E946D7520E030E040E85FE30E9418
:10D6600059A69B01AC01C701B6010E9436A987FFEC
:10D6700035C038C0B7FC36C06091C109E62FF0E074
:10D68000EE0FFF1FE25EF54F808191810E946D7564
:10D690006B017C016091C109E62FF0E0EE0FFF1FE6
:10D6A000EE5DF54F808191810E946D759B01AC010B
:10D6B000C701B6010E9459A60E94A2A7AB01BC01F6
:10D6C00077FF07C070956095509541955F4F6F4FFC
:10D6D0007F4F443051056105710524F00E9425A358
:10D6E0004B015C019FEF89169FEF99069FEFA906FA
:10D6F0009FEFB90659F0B7FCB8C60E9425A3681978
:10D700007909E3E168387E0708F0AFC60E9425A3D7
:10D71000DC01CB0184199509A609B709893EF3E01C
:10D720009F07F0E0AF07F0E0BF0708F0E0CE61CF61
:10D7300089EF9DE00E94A42C83E50E94A6298823FE
:10D7400061F00E948A290E94A2A7DC01CB010E94FD
:10D750006A759093210A8093200A0E9425A36B0189
:10D760007C01E6E0FEE0A490E9E0FEE08490EDE0DC
:10D77000FEE004911AE077C00E9425A3DC01CB01F2
:10D780008C199D09AE09BF09893E23E0920720E06C
:10D79000A20720E0B20708F45FC060910007E62FFF
:10D7A000F0E0EE0FFF1FE25EF54F808191810E9455
:10D7B0006D75AB01BC018A2DE6E0FEE008C09091DA
:10D7C000C00095FFFCCF8093C600319684918823DA
:10D7D000B1F78FE59AE022E030E00E942B81882D9E
:10D7E000E9E0FEE008C09091C00095FFFCCF809377
:10D7F000C600319684918823B1F7609100078FE5C8
:10D800009AE070E04AE050E00E942F80802FEDE027
:10D81000FEE008C09091C00095FFFCCF8093C60049
:10D82000319684918823B1F780911C0A90911D0A4A
:10D830000E94DD77AB01BC018FE59AE021E030E08A
:10D840000E942B818091C00085FFFCCF1093C60001
:10D850000E9425A36B017C010E94BE7581E00E949D
:10D860002A2D0E94DA5E8091200A9091210A20914F
:10D870001C0A30911D0A281739070CF47DCF81E16D
:10D880009EE00E94A42C01C683E50E94A62988235D
:10D89000F9F00E948A2920E030E040E050E00E9448
:10D8A00033A787FD0FC00E948A2920E030E04FE7B0
:10D8B00053E40E9436A918163CF00E948A290E945F
:10D8C000A7A703C060E001C06FEF6093FF06CAC561
:10D8D0008FEF8093FF06C6C51092FF06C3C5269A38
:10D8E0002E98C0C50E948B160E948729BBC5109236
:10D8F0002307B8C581E080932307B4C583E50E9460
:10D90000A6298823A9F00E948A2920E030E04AE76E
:10D9100054E40E9408AA0E94A7A7DC01CB018093CF
:10D92000210490932204A0932304B09324049AC565
:10D9300088E50E94A629882309F0B4C589E50E94DC
:10D94000A629882309F0AEC58AE50E94A629882366
:10D9500009F0A8C585E40E94A629882309F0A2C57C
:10D960000E948B16A09A0E94FD167CC5159A89E527
:10D970000E94A6298111179A8AE50E94A629811181
:10D98000429A85E40E94A6298111A09A8BE19EE02B
:10D990000E94A42C67C583E50E94A6290E948A29BB
:10D9A00020E030E04AE754E40E9408AA0E94A7A7BA
:10D9B000DC01CB018093C2099093C309A093C409F1
:10D9C000B093C5094FC585E494E09AA389A343E0C9
:10D9D000A42E40E1B42E53E1252E50E1352EE7EC84
:10D9E000FFE0F8A3EF8FDD244501E9A1FAA18191C1
:10D9F000FAA3E9A30E94A629882309F471C0F3E0E1
:10DA0000DF1609F064C00E948A292B013C0120E046
:10DA100030E040EA51E40E9433A787FF52C0F4018E
:10DA20006081718182819381A30192010E943AA752
:10DA3000F62EE72EC82EA92E6091DB0F7091DC0F19
:10DA40008091DD0F9091DE0FF7010F2F1E2F2C2DEF
:10DA50003A2DA90198010E9408AADC01CB0180930C
:10DA6000DB0F9093DC0FA093DD0FB093DE0FF1017D
:10DA700060817181828193812C2D3A2DA9019801B9
:10DA80000E9408AADC01CB01F10180839183A2836B
:10DA9000B383EF8DF8A160817181828193810E94AF
:10DAA000D3A72C2D3A2DA90198010E9408AA0E9403
:10DAB000A7A7DC01CB01EF8DF8A180839183A2831E
:10DAC000B383F401408251826282738209C00E9452
:10DAD0008A29DC01CB01F40180839183A283B38383
:10DAE000D39424E030E0820E931E220E331E8F8DDD
:10DAF00098A1049698A38F8F94E0D91609F075CF5A
:10DB0000B1C4EBE2FEE007C09091C00095FFFCCFEE
:10DB10008093C600319684918823B1F7A3C44091C5
:10DB200090095091910920E630E0429FC001439F47
:10DB3000900D529F900D11248F5E974F0E94882C5C
:10DB400091C4EBECFEE007C09091C00095FFFCCFC4
:10DB50008093C600319684918823B1F740910D07D8
:10DB600050910E0760910F07709110078FE59AE0B2
:10DB700022E030E00E942B81EEECFEE007C09091A5
:10DB8000C00095FFFCCF8093C60031968491882316
:10DB9000B1F74091110750911207609113077091EE
:10DBA00014078FE59AE022E030E00E942B81E1ED3E
:10DBB000FEE007C09091C00095FFFCCF8093C600A7
:10DBC000319684918823B1F740911507509116073B
:10DBD00060911707709118078FE59AE022E030E016
:10DBE0000E942B81E4EDFEE007C09091C00095FFFC
:10DBF000FCCF8093C600319684918823B1F7409181
:10DC0000190750911A0760911B0770911C078FE547
:10DC10009AE022E030E00E942B81E7EDFEE007C0B1
:10DC20009091C00095FFFCCF8093C60031968491FF
:10DC30008823B1F70E94E7160E94D5A72091031010
:10DC40003091041040910510509106100E943AA79F
:10DC5000AB01BC018FE59AE022E030E00E942B810D
:10DC6000E1EEFEE007C09091C00095FFFCCF8093ED
:10DC7000C600319684918823B1F781E00E94E716AF
:10DC80000E94D5A7209107103091081040910910EB
:10DC900050910A100E943AA7AB01BC018FE59AE0AF
:10DCA00022E030E00E942B81E4EEFEE007C090917C
:10DCB000C00095FFFCCF8093C600319684918823E5
:10DCC000B1F782E00E94E7160E94D5A720910B10C1
:10DCD00030910C1040910D1050910E100E943AA7F7
:10DCE000AB01BC018FE59AE022E030E00E942B817D
:10DCF0008091C00085FFFCCFB2C380E001C081E00D
:10DD00000E94200FAFC3E7EEFEE007C09091C00075
:10DD100095FFFCCF8093C600319684918823B1F79C
:10DD200080B180FD03C0E9E2F3E009C0ECE2F3E07A
:10DD300006C09091C00095FFFCCF8093C6008191F2
:10DD40008823B9F7EEEEFEE007C09091C00095FF82
:10DD5000FCCF8093C600319684918823B1F7029955
:10DD600003C0E9E2F3E009C0ECE2F3E006C0909101
:10DD7000C00095FFFCCF8093C60081918823B9F73E
:10DD8000E5EFFEE007C09091C00095FFFCCF8093C7
:10DD9000C600319684918823B1F7049903C0E9E263
:10DDA000F3E009C0ECE2F3E006C09091C00095FFFB
:10DDB000FCCF8093C60081918823B9F7ECEFFEE099
:10DDC00007C09091C00095FFFCCF8093C6003196AC
:10DDD00084918823B1F7069903C0E9E2F3E009C012
:10DDE000ECE2F3E006C09091C00095FFFCCF809379
:10DDF000C60081918823B9F7E3E0FFE007C0909166
:10DE0000C00095FFFCCF8093C60031968491882393
:10DE1000B1F7379903C0E9E2F3E009C0ECE2F3E0BF
:10DE200006C09091C00095FFFCCF8093C600819101
:10DE30008823B9F7EAE0FFE007C09091C00095FFA2
:10DE4000FCCF8093C600319684918823B1F7359931
:10DE500003C0E9E2F3E009C0ECE2F3E006C0909110
:10DE6000C00095FFFCCF8093C60081918823B9F74D
:10DE70008091C00085FFFCCFF2C235E4C32E34E0B0
:10DE8000D32E00E010E0F60181916F010E94A629D7
:10DE9000882359F10E948A29F3EFEF2EFFE0FF2E2D
:10DEA000E00EF11E0E94A7A7DC01CB01F7018083E1
:10DEB0009183A283B3830E948A2927ECE22E2FE06C
:10DEC000F22EE00EF11EF801ED5FFF4E2081318150
:10DED000428153810E9408AA0E94A7A7DC01CB01BE
:10DEE000F70180839183A283B3830C5F1F4F0031BE
:10DEF000110549F6B7C275E4C72E74E0D72E03E1C9
:10DF000010E1E4E0EE2EF60181916F010E94A62956
:10DF1000882349F00E948A29DC01CB01F801808323
:10DF20009183A283B383EA940C5F1F4FEE2059F7CD
:10DF300099C283E50E94A629882361F00E948A295C
:10DF4000DC01CB018093EB0F9093EC0FA093ED0FCE
:10DF5000B093EE0F84E50E94A629882309F482C2BB
:10DF60000E948A29DC01CB018093E70F9093E80F90
:10DF7000A093E90FB093EA0F75C283E50E94A6292A
:10DF8000882361F00E948A29DC01CB018093EF0F86
:10DF90009093F00FA093F10FB093F20F84E50E94DD
:10DFA000A629882361F00E948A29DC01CB01809395
:10DFB000D70F9093D80FA093D90FB093DA0F82E4C4
:10DFC0000E94A629882371F00E948A290E94A7A78F
:10DFD000DC01CB018093231090932410A093251093
:10DFE000B093261088E50E94A629882361F00E943C
:10DFF0008A29DC01CB018093E30F9093E40FA09377
:10E00000E50FB093E60F8AE50E94A629882361F008
:10E010000E948A29DC01CB018093DF0F9093E00FEF
:10E02000A093E10FB093E20F85E40E94A629882314
:10E0300009F418C20E948A29DC01CB018093DB0F0E
:10E040009093DC0FA093DD0FB093DE0F0BC255E46D
:10E05000C52E54E0D52E01E017E063E0E62EF60170
:10E0600081916F010E94A629882349F00E948A2984
:10E07000DC01CB01F80180839183A283B383EA940E
:10E080000C5F1F4FEE2059F7EDC183E50E94A629D2
:10E09000882309F4E7C10E948A290E94A2A7DC0113
:10E0A000CB0190930B0480930A0481E080931D07B9
:10E0B000D9C183E50E94A629882309F4D3C10E940F
:10E0C0008A290E94A2A7DC01CB01909309048093C6
:10E0D0000804C8C180E50E94A629882361F00E9437
:10E0E0008A29DC01CB018093360490933704A093F6
:10E0F0003804B093390489E40E94A629882391F05A
:10E100000E948A292FE632E143E05EE30E9408AADA
:10E11000DC01CB018093320490933304A093340448
:10E12000B093350484E40E94A629882391F00E94CC
:10E130008A292FE632E143E05EE30E943AA7DC0140
:10E14000CB0180932E0490932F04A0933004B093BE
:10E15000310483E40E94A629882361F00E948A2961
:10E16000DC01CB0180932A0490932B04A0932C0410
:10E17000B0932D040E940375E6E7F3E006C090918A
:10E18000C00095FFFCCF8093C60081918823B9F72A
:10E19000E9E7F3E006C09091C00095FFFCCF8093C3
:10E1A000C60081918823B9F7409136045091370415
:10E1B00060913804709139048FE59AE022E030E0F4
:10E1C0000E942B81EDE7F3E006C09091C00095FF1F
:10E1D000FCCF8093C60081918823B9F76091320407
:10E1E0007091330480913404909135042FE632E12C
:10E1F00043E05EE30E943AA7AB01BC018FE59AE0E1
:10E2000022E030E00E942B81E1E8F3E006C090912B
:10E21000C00095FFFCCF8093C60081918823B9F799
:10E2200060912E0470912F048091300490913104FC
:10E230002FE632E143E05EE30E9408AAAB01BC0195
:10E240008FE59AE022E030E00E942B81E5E8F3E0E0
:10E2500006C09091C00095FFFCCF8093C6008191CD
:10E260008823B9F760912A0470912B0480912C04C3
:10E2700090912D042FE632E143E05EE30E9408AA6C
:10E28000AB01BC018FE59AE022E030E00E942B81D7
:10E290008091C00085FFFCCFE2C081E00E94A89F72
:10E2A000E1C083E50E94A629882319F00E948A29EB
:10E2B00004C060E070E086E193E40E946A78D2C016
:10E2C0000E948B16CFC00E942B59CCC080E001C0A9
:10E2D00081E00E94395AC6C00E941825C3C010921E
:10E2E000FE068091C6099091C709A091C809B09116
:10E2F000C90980939C0990939D09A0939E09B093AE
:10E300009F090E94EF29AEC084E50E94A6298823B8
:10E3100009F461C00E948A290E94A7A76093C109DD
:10E32000EAE6F9E0662381F107C09091C00095FF0D
:10E33000FCCF8093C600319684918823B1F7E9E839
:10E34000F3E006C09091C00095FFFCCF8093C6001B
:10E3500081918823B9F78FE59AE06091C10940E087
:10E3600050E00E94F27FEBE8F3E006C09091C0001D
:10E3700095FFFCCF8093C60081918823B9F78091E7
:10E38000C00085FFFCCF6BC01092000707C09091C2
:10E39000C00095FFFCCF8093C600319684918823FE
:10E3A000B1F7ECE9F3E006C09091C00095FFFCCF17
:10E3B0008093C60081918823B9F7609100078FE5AB
:10E3C0009AE070E04AE050E00E942F808091C00007
:10E3D00085FFFCCF44C0EAE6F9E007C09091C00099
:10E3E00095FFFCCF8093C600319684918823B1F7C6
:10E3F000E1E1FFE007C09091C00095FFFCCF809362
:10E40000C600319684918823B1F72091900930910C
:10E41000910980E690E0289FF001299FF00D389F38
:10E42000F00D1124E45FF74F06C09091C00095FFF6
:10E43000FCCF8093C60081918823B9F7E3E2FFE027
:10E4400007C09091C00095FFFCCF8093C600319625
:10E4500084918823B1F78091C00085FFFCCF8AE0CA
:10E460008093C6000E94C52948C08BEE9DE00E94A3
:10E47000A42C0E9425A3DC01CB018093A4099093D6
:10E48000A509A093A609B093A7090E9425A3DC01C2
:10E49000CB018093A8099093A909A093AA09B093EE
:10E4A000AB09E0CF0E948B1688E50E94A62988233D
:10E4B00009F05CCA5CCA808191810E946D756B0114
:10E4C0007C016091C109E62FF0E0EE0FFF1FEE5DC9
:10E4D000F54F808191810E946D7520E030E040E829
:10E4E0005FE30E945AA69B01AC01C701B6010E94DE
:10E4F00033A718160CF0F2C8F5C8A2960FB6F89418
:10E50000DEBF0FBECDBFDF91CF911F910F91FF9066
:10E51000EF90DF90CF90BF90AF909F908F907F90C3
:10E520006F905F904F903F902F900895CF93DF931F
:10E5300080910808909109088330910514F40E9495
:10E54000882D84E297E060E00E946F88809108083F
:10E5500090910908009709F463C0809124078823EB
:10E5600009F446C0209190093091910980E690E02D
:10E57000289FE001299FD00D389FD00D1124C45F42
:10E58000D74FCE016EEA73E00E948BAE0097B9F4CC
:10E5900084E297E0BE010E940188EAE2FCE007C045
:10E5A0009091C00095FFFCCF8093C6003196849176
:10E5B0008823B1F78091C00085FFFCCF15C084E2AD
:10E5C00097E00E948489EDE2FCE007C09091C000D2
:10E5D00095FFFCCF8093C600319684918823B1F7D4
:10E5E0008091C00085FFFCCF8AE08093C60002C006
:10E5F0000E94385F809108089091090801979093D4
:10E6000009088093080880919009909191090196DA
:10E6100064E070E00E9401AB9093910980939009AF
:10E620000E94BE7581E00E942A2D0E945D0E0E940C
:10E63000DA5EDF91CF9108958F929F92AF92BF9251
:10E64000CF92DF92EF92FF920F931F93CF930E948E
:10E6500084298FE59AE040E052EC61E070E00E948E
:10E66000047FEDE7F9E007C09091C00095FFFCCF73
:10E670008093C600319684918823B1F78091C000C1
:10E6800085FFFCCF8AE08093C6008AE699E0FC0112
:10E6900007C03091C00035FFFCCF2093C6003196F3
:10E6A00024912223B1F724B720FF14C0E3E8F9E056
:10E6B00007C04091C00045FFFCCF3093C6003196A3
:10E6C00034913323B1F73091C00035FFFCCF3AE0ED
:10E6D0003093C60021FF14C0EBE8F9E007C0409179
:10E6E000C00045FFFCCF3093C600319634913323F0
:10E6F000B1F73091C00035FFFCCF3AE03093C6004F
:10E7000022FF14C0EBE9F9E007C04091C00045FFCB
:10E71000FCCF3093C600319634913323B1F730915A
:10E72000C00035FFFCCF3AE03093C60023FF14C091
:10E73000ECEAF9E007C04091C00045FFFCCF309300
:10E74000C600319634913323B1F73091C00035FFC4
:10E75000FCCF3AE03093C60025FF14C0ECEBF9E0A3
:10E7600007C03091C00035FFFCCF2093C600319622
:10E7700024912223B1F72091C00025FFFCCF2AE08D
:10E780002093C60014BEECECF9E007C03091C00045
:10E7900035FFFCCF2093C600319624912223B1F798
:10E7A000E4EDF9E007C03091C00035FFFCCF2093C5
:10E7B000C600319624912223B1F72091C00025FF95
:10E7C000FCCF2AE02093C600FC012491EAE6F9E0A0
:10E7D00008C03091C00035FFFCCF2093C6003196B1
:10E7E00024912223B1F7EEEDF9E007C03091C0008B
:10E7F00035FFFCCF2093C600319624912223B1F738
:10E80000EEEEF9E007C03091C00035FFFCCF209359
:10E81000C600319624912223B1F7E0E4FAE007C064
:10E820003091C00035FFFCCF2093C6003196249173
:10E830002223B1F7ECE4FAE007C03091C00035FFC5
:10E84000FCCF2093C600319624912223B1F720916A
:10E85000C00025FFFCCF2AE02093C600FC01849174
:10E86000EAE6F9E008C09091C00095FFFCCF8093E4
:10E87000C600319684918823B1F7ECE5FAE007C031
:10E880009091C00095FFFCCF8093C6003196849193
:10E890008823B1F70E94EF28BC018FE59AE04AE097
:10E8A00050E00E942F80EBE6FAE007C09091C00094
:10E8B00095FFFCCF8093C600319684918823B1F7F1
:10E8C0008FE59AE060ED74E04AE050E00E942F800E
:10E8D0008091C00085FFFCCF8AE08093C600109233
:10E8E0008C0910928D0910928E0910928F0980E088
:10E8F0000E94395A03EF1FE0A3E0AA2EA0E1BA2E2E
:10E90000B7EC8B2EBFE09B2EC0E0F80161917191B6
:10E91000819191918F01F501C190D190E190F19099
:10E920005F010E94D3A7A70196010E9408AA0E9436
:10E93000A7A7DC01CB01F40181939193A193B1933B
:10E940004F01CF5FC43009F70E94E2770E947D93A8
:10E950000E9420160E94B931CF911F910F91FF9014
:10E96000EF90DF90CF90BF90AF909F908F900895E1
:10E9700021E434E0FC01318320832781222319F034
:10E9800004960E94831B0895CF92EF920F938130DB
:10E990009105A9F484E297E00E942E8182EE96E030
:10E9A00064E141E120E105E135E0E32E56E0C52ECA
:10E9B0000E9426A687EF99E00E94A73216C0009712
:10E9C000A1F487ED97E00E94B87485E997E00E9472
:10E9D000B87486E797E00E94B87487E597E00E94D4
:10E9E000B87486E397E00E94B8740F91EF90CF90CF
:10E9F000089581E090E00E94C474089580E090E062
:10EA00000E94C474089560E070E08FE793E4209161
:10EA100032043091330440913404509135040E9403
:10EA20003AA7DC01CB018093250A9093260AA09394
:10EA3000270AB093280A0895FC01EC5DF54F808108
:10EA400090E00895CF93DF93EC01662351F1E3EB5F
:10EA5000F3E107C09091C00095FFFCCF8093C60002
:10EA6000319684918823B1F78FE59AE070E04AE00F
:10EA700050E00E942F80EAEBF3E107C09091C000C4
:10EA800095FFFCCF8093C600319684918823B1F71F
:10EA90008091C00085FFFCCF8AE08093C6000E9471
:10EAA000F72CBE01882777FD8095982F0E94D5A767
:10EAB0002FE632E143E050E40E9408AA20E030E073
:10EAC00040E851E40E9408AA0E94A2A7CB01DF916E
:10EAD000CF91089580E090E00895CF93DF93EC010B
:10EAE000662351F1E3EBF3E107C09091C00095FF7D
:10EAF000FCCF8093C600319684918823B1F78FE5CF
:10EB00009AE070E04AE050E00E942F80E6EDF3E1E9
:10EB100007C09091C00095FFFCCF8093C60031964E
:10EB200084918823B1F78091C00085FFFCCF8AE0F3
:10EB30008093C6000E94F72CBE01882777FD809540
:10EB4000982F0E94D5A720E030E04AEF5EE30E94B4
:10EB500008AA20E030E040E85DE30E9408AA20E037
:10EB600030E040E050E00E945AA6462F572F682F11
:10EB7000792FCB01BA01DF91CF9108952F923F9267
:10EB80004F925F926F927F928F929F92AF92BF92BD
:10EB9000CF92DF92EF92FF920F931F93CF93DF9369
:10EBA00000D00F92CDB7DEB78091170A882309F401
:10EBB000EDC18FB7F8941092170A8FBF80911E0A8B
:10EBC00090911F0A60E00E946D752B013C016091DD
:10EBD000180A7091190A80911A0A90911B0AA301D0
:10EBE00092010E9459A6C62EB72E182F092F980100
:10EBF000862F9B2DA32FB22F8093290A90932A0A48
:10EC0000A0932B0AB0932C0ABC01CD0120E030E088
:10EC100040E251E40E9436A918160CF450C1980144
:10EC20008C2D9B2DA32FB22FBC01CD0120E030E015
:10EC300040E251EC0E9433A787FD3DC180912D0A2F
:10EC4000882309F029C198018C2D9B2DA32FB02F6B
:10EC5000BC01CD0120913604309137044091380435
:10EC6000509139040E9408AA69837A831C01472FB6
:10EC7000862F942FA22DB32D8093320A9093330ABE
:10EC8000A093340AB093350A98018C2D9B2DA32FA5
:10EC9000B02FBC01CD0120912E0A30912F0A409156
:10ECA000300A5091310A0E945AA6B62EA72E982EED
:10ECB000892E0091360A1091370A2091380A2C8348
:10ECC0008091390A8B83A5019401852F942FA32F5E
:10ECD000B22FBC01CD013C812B81C02ED12EE32E61
:10ECE000F22EA70196010E9433A787FFB3C03C8193
:10ECF0002B81802F912FA32FB22F80932E0A9093D8
:10ED00002F0AA093300AB093310ABC01CD012091A3
:10ED100032043091330440913404509135040E9400
:10ED200008AA6B83872E182F092F9801862F982DFC
:10ED3000A32FB22F80933A0A90933B0AA0933C0AE8
:10ED4000B0933D0AC301B20120913E0A30913F0ABF
:10ED50004091400A5091410A0E9459A620912E04E8
:10ED600030912F0440913004509131040E9408AA40
:10ED700020ED3CEC4CE45DE30E9408AA6B017C01B1
:10ED80006091420A7091430A8091440A9091450A29
:10ED900023E333E343E75FE30E9408AA9B01AC014E
:10EDA000C701B6010E945AA6B62EC72EA82E992ECC
:10EDB000862F9C2DAA2DB92D8093420A9093430A49
:10EDC000A093440AB093450A40923E0A50923F0AEB
:10EDD0006092400A7092410A59814A81852F942F8E
:10EDE000A22DB32DBC01CD01FB81A8010F2F182D41
:10EDF000252F342FA90198010E945AA60B2D1C2DF6
:10EE00002A2D392DA90198010E9459A6C62EB72E88
:10EE1000182F092F9801862F9B2DA32FB22FBC01ED
:10EE2000CD0120E030E040E050E00E9433A787FDB4
:10EE30004EC098018C2D9B2DA32FB22FBC01CD016C
:10EE400020E030E04FE753E40E9436A918160CF09A
:10EE500042C038C00091250A1091260AE091270A85
:10EE6000EC83F091280AFB83A5019401852F942F50
:10EE7000A32FB22FBC01CD01C02ED12EEE2EFF2E1E
:10EE8000A70196010E9436A918160CF430CF0B2D5D
:10EE90001A2D9C828B822BCF80E090E0A0E0B0E026
:10EEA00080932E0A90932F0AA093300AB093310AD0
:10EEB00010922D0AC8CE81E080932D0A08C081E00F
:10EEC00080932D0ACC24BB241FE703E404C0CC2488
:10EED000BB2410E000E080911E0A90911F0A20914F
:10EEE000460A3091470A281739071CF01092240A65
:10EEF00014C020913A0430913B0482179307B4F771
:10EF000098018C2D9B2DA32FB02FBC01CD010E9409
:10EF1000A2A7759567956093240A0E9425A3DC013A
:10EF2000CB014091480A5091490A60914A0A709178
:10EF30004B0A841B950BA60BB70B883823E192076D
:10EF400020E0A20720E0B20708F10E9425A3DC011F
:10EF5000CB018093480A9093490AA0934A0AB09340
:10EF60004B0A80911C0A90911D0A181619066CF420
:10EF7000EFE38F3F9E074CF42091200A3091210A45
:10EF80008217930714F4A59A01C0A5980F900F90CB
:10EF90000F900F90DF91CF911F910F91FF90EF9005
:10EFA000DF90CF90BF90AF909F908F907F906F90A9
:10EFB0005F904F903F902F90089560E070E080E068
:10EFC00090E0089580E090E0A0E0B0E08093360A01
:10EFD0009093370AA093380AB093390A60E070E042
:10EFE0008FE793E42091320430913304409134044C
:10EFF000509135040E943AA7DC01CB018093250A89
:10F000009093260AA093270AB093280A6C9A6D9AC7
:10F010009D9AE1E0F1E080818061808387E061E09A
:10F0200070E00E94382C87ED80937A0010927E0069
:10F03000EDE7F0E0108280818160808380818260D2
:10F04000808380818460808380E888BDEEE6F0E084
:10F050008081846080836AEF70E080E090E00E94AD
:10F0600061A385E090E060E00E9422759093470ADA
:10F070008093460A83E191E060E00E9422759093BC
:10F080003B0480933A040895089580E090E060E0A6
:10F090000E94227580E090E0A0E0B0E08093180A22
:10F0A0009093190AA0931A0AB0931B0A1092210A8E
:10F0B0001092200A1092230A1092220A1092240A17
:10F0C00074981092250A1092240A1092250A7598B5
:10F0D000A59808952F923F924F925F926F927F92E0
:10F0E0008F929F92AF92BF92CF92DF92EF92FF9258
:10F0F0000F931F93CF93DF93CDB7DEB7AA970FB6C9
:10F10000F894DEBF0FBECDBF6B8B7C8B8D8B9E8B3F
:10F110000E9425A36F8B788F898F9A8FE2EBF3E0A3
:10F1200006C09091C00095FFFCCF8093C6008191EE
:10F130008823B9F78091C00085FFFCCF8AE08093D7
:10F14000C6000E9445788FE78093240A2F89388D66
:10F15000498D5A8D2F87388B498B5A8B2B873C874B
:10F160004D875E878FE790E0A0E0B0E089839A83C7
:10F17000AB83BC836FE7462E512C612C712C91E040
:10F180001A861986ECECF2E114911CA3E4EDF2E18D
:10F1900014911DA3E9EDF2E114911EA3E0EEF2E15A
:10F1A00014911FA3E7EEF2E1149118A7EDEEF2E13E
:10F1B000149119A7B92E0AA78091170A882309F478
:10F1C00028C38FB7F8941092170A8FBF80911E0A38
:10F1D00090911F0A60E00E946D756D837E838F831E
:10F1E00098875B8D4C8D3D8D2E8D852F942FA32F71
:10F1F000B22FBC01CD01FD81EE815F8148850F2FCB
:10F200001E2F252F342FA90198010E9436A9181608
:10F2100034F00B8F1C8F0F810D8F18851E8F5F8D23
:10F220002AA5852F922DA32DB22FBC01CD01FD81E2
:10F23000EE815F8148850F2F1E2F252F342FA901C6
:10F2400098010E9433A787FD05C00F8F212E3F80B4
:10F2500018851AA7BB2009F45AC05D814E813F81F1
:10F260002885852F942FA32FB22FBC01CD01FB89B8
:10F27000EC895D894E890F2F1E2F252F342FA90170
:10F2800098010E9436A918160CF0C3C20E9425A34B
:10F29000DC01CB010F85188929893A89801B910BE4
:10F2A000A20BB30B893813E1910710E0A10710E01E
:10F2B000B10708F4AEC2D301C20109811A812B81C2
:10F2C0003C81801B910BA20BB30BB595A79597952D
:10F2D00087958093240A0E9425A36B877C878D875E
:10F2E0009E878B019C018F859889A989BA89081B03
:10F2F000190B2A0B3B0B08A319A32AA33BA30B89C9
:10F300000B8F1C891C8F0D890D8F1E891E8F5D81AF
:10F310004E813F812885852F942FA32FB22FBC01CA
:10F32000CD01FB89EC895D894E890F2F1E2F252F7A
:10F33000342FA90198010E9433A787FF69C20E9458
:10F3400025A3DC01CB010B851C852D853E85801B0B
:10F35000910BA20BB30B893813E1910710E0A107C1
:10F3600010E0B10708F454C20E9425A36F87788B80
:10F37000898B9A8B09851A850115110509F42BC211
:10F38000DC01CB010B851C852D853E85801B910BF7
:10F39000A20BB30B88A099A0AAA0BBA0880E991EAF
:10F3A000AA1EBB1E28A139A14AA15BA1281B390BAB
:10F3B0004A0B5B0B69817A818B819C810E94CEAA6A
:10F3C000A50194010E9436AB89019A01040D151D17
:10F3D000261D371D0431110521053105E4F02801F2
:10F3E00039011CEE41165104610471042CF04BEEFE
:10F3F000442E512C612C712C20E8421651046104DA
:10F400007104BCF00EEF10E020E030E004191509A3
:10F410002609370909C034E1432E512C612C712C87
:10F4200004E110E020E030E009831A832B833C8361
:10F4300004C049825A826B827C828CA1ECECF2E19E
:10F440009AA50AC0292F9091C00095FFFCCF922F5A
:10F450008093C600319684918823A1F79AA78FE5FF
:10F460009AE0B301A2012AE030E00E94FA7F8DA168
:10F47000E4EDF2E19AA50AC0292F9091C00095FF12
:10F48000FCCF922F8093C600319684918823A1F7F8
:10F490009AA78FE59AE049815A816B817C812AE0A5
:10F4A00030E00E94FA7F8EA1E9EDF2E19AA50AC050
:10F4B000292F9091C00095FFFCCF922F8093C6001A
:10F4C000319684918823A1F79AA78FE59AE0FF8D62
:10F4D0002AA54F2F522D632D722F22E030E00E947B
:10F4E0002B818FA1E0EEF2E19AA50AC0292F90911D
:10F4F000C00095FFFCCF922F8093C6003196849177
:10F500008823A1F79AA78FE59AE0FB8DEC8D3D8DBE
:10F510002E8D4F2F5E2F632F722F22E030E00E943E
:10F520002B819AA58091C00085FFFCCF9AA78AE025
:10F530008093C60009851A85033011050CF44BC170
:10F5400069817A818B819C810E94D5A720E030E07F
:10F5500040E850E40E9408AA6B017C015B8D4C8D51
:10F560003D8D2E8D852F942FA32FB22FBC01CD0161
:10F57000FF8D4AA50F2F122D232D342FA90198019D
:10F580000E9459A620ED3FE049E450E40E9408AAF9
:10F5900020E030E040E05FE30E9408AA9B01AC015C
:10F5A000C701B6010E943AA7E62E372E082FF92E82
:10F5B000C501B4010E94D5A720E030E04AE754E439
:10F5C0000E943AA7D62EC72EB82EA92E88A5E7EE00
:10F5D000F2E108C09091C00095FFFCCF8093C60077
:10F5E000319684918823B1F78FE59AE04E2D532D03
:10F5F000602F7F2D22E030E00E942B8189A5EDEE67
:10F60000F2E108C09091C00095FFFCCF8093C60046
:10F61000319684918823B1F78FE59AE0F601950140
:10F620004F2F5C2D632F7A2D22E030E00E942B813A
:10F630008091C00085FFFCCF8AE08093C6008E2DAC
:10F64000932DA02FBF2DBC01CD012AE939E949E155
:10F650005FE30E9408AA6F8F7AA7F82EE92E562F33
:10F66000472F9701862F942FA32FB22FBC01CD01D6
:10F67000FA01A7010F2F1E2F252F342FA901980162
:10F680000E945AA6F601A5010F2F1C2D252F3A2DF9
:10F69000A90198010E943AA7962E872E382E292E6E
:10F6A0005F8D4AA59701852F942FA32FB22FBC0100
:10F6B000CD01A501252F3A2DA90198010E9408AA84
:10F6C00020E030E040E05EE30E9408AA062FD72E3B
:10F6D000C82EB92EE3EFF2E184919F8D3AA50AC0BE
:10F6E000292F9091C00095FFFCCF922F8093C600E8
:10F6F000319684918823A1F78091C00085FFFCCFCB
:10F700009F8F3AA78AE08093C600E0E0F3E18491FE
:10F710009F8D3AA50AC0292F9091C00095FFFCCF7C
:10F72000922F8093C600319684918823A1F79F8FF2
:10F730003AA78FE59AE0FF8DE32F97014F2F5E2FB9
:10F74000632F7E2D22E030E00E942B818091C0004B
:10F7500085FFFCCF8AE08093C600E6E0F3E107C0B6
:10F760009091C00095FFFCCF8093C60031968491A4
:10F770008823B1F78FE59AE0F40191014F2F582DBE
:10F78000632F722D22E030E00E942B818091C00017
:10F7900085FFFCCF8AE08093C600ECE0F3E107C070
:10F7A0009091C00095FFFCCF8093C6003196849164
:10F7B0008823B1F78FE59AE0402F5D2D6C2D7B2DCE
:10F7C00022E030E00E942B818091C00085FFFCCFB9
:10F7D0008AE08093C60089819A81AB81BC81840DC7
:10F7E000951DA61DB71DB595A795979587958093EF
:10F7F000240A09851A850F5F1F4F1A8709871B89FD
:10F800001F8F2C883D880E890AA7BB24B39401C0A2
:10F81000BB245B894C893D892E89852F942FA32F8A
:10F82000B22FBC01CD0120E030E040EA51E40E945B
:10F830005AA69B01AC01FD81EE817F8168858F2FE7
:10F840009E2FA72FB62FBC01CD010E9436A91816F6
:10F8500094F4E2E1F3E107C09091C00095FFFCCF82
:10F860008093C600319684918823B1F78091C000BF
:10F8700085FFFCCFADC00E9425A3DC01CB010F8921
:10F88000188D298D3A8D801B910BA20BB30B813DF6
:10F8900017E0910710E0A10710E0B10708F44BC092
:10F8A0000E9425A36F8B788F898F9A8FEBE3F3E10A
:10F8B00084919AA50AC0292F9091C00095FFFCCF92
:10F8C000922F8093C600319684918823A1F79AA73E
:10F8D00080911E0A90911F0A60E00E946D75AB0135
:10F8E000BC018FE59AE022E030E00E942B81E1E448
:10F8F000F3E184919AA50AC0292F9091C00095FF49
:10F90000FCCF922F8093C600319684918823A1F773
:10F910009AA76091240A8FE59AE070E04AE050E0EF
:10F920000E942F809AA58091C00085FFFCCF9AA7E6
:10F930008AE08093C6000E9425A36B017C010E948F
:10F9400025A3AB01BC018B859C85AD85BE850F854C
:10F95000188929893A89800F911FA21FB31FC81ADD
:10F96000D90AEA0AFB0AC40ED51EE61EF71E11E8E4
:10F97000C1161FE4D10612E1E10610E0F10690F095
:10F98000E5E4F3E107C09091C00095FFFCCF8093C0
:10F99000C600319684918823B1F78091C00085FF1D
:10F9A000FCCF16C009851A85063011056CF1E2E618
:10F9B000F3E107C09091C00095FFFCCF8093C60093
:10F9C000319684918823B1F78091C00085FFFCCFE8
:10F9D0008AE08093C600AA960FB6F894DEBF0FBEE9
:10F9E000CDBFDF91CF911F910F91FF90EF90DF90EE
:10F9F000CF90BF90AF909F908F907F906F905F90CF
:10FA00004F903F902F9008950E94DA5ED5CBCF9310
:10FA1000DF930F92CDB7DEB789830E9445780E94AD
:10FA2000352C6981882379F5E3EBF3E107C09091E8
:10FA3000C00095FFFCCF8093C60031968491882347
:10FA4000B1F78FE59AE070E04AE050E00E942F8025
:10FA50008091C00085FFFCCF8AE08093C600E3EF71
:10FA6000F3E107C09091C00095FFFCCF8093C600E2
:10FA7000319684918823B1F78091C00085FFFCCF37
:10FA80008AE08093C6000F90DF91CF910895CF93C5
:10FA9000DF930F92CDB7DEB789830E9445780E942D
:10FAA000352C6981882379F5E3EBF3E107C0909168
:10FAB000C00095FFFCCF8093C600319684918823C7
:10FAC000B1F78FE59AE070E04AE050E00E942F80A5
:10FAD0008091C00085FFFCCF8AE08093C600E0E201
:10FAE000F4E107C09091C00095FFFCCF8093C60061
:10FAF000319684918823B1F78091C00085FFFCCFB7
:10FB00008AE08093C6000F90DF91CF9108951F92F5
:10FB10000F920FB60F920BB60F9211242F933F93B3
:10FB20004F935F936F937F938F939F93AF93BF9305
:10FB3000EF93FF9380913C04882331F48091240A51
:10FB400080934C0A8111749A90914C0A80913C04E4
:10FB5000891708F074988F5F8F7780933C048091A9
:10FB60004D0A833009F450C0843028F48130F9F014
:10FB70008230D8F50DC0853009F471C0853008F4A5
:10FB80005FC0863009F487C0873009F08FC087C016
:10FB900088E080937B0080E480937C0080917A00F1
:10FBA000806480937A000E942E3281E01BC04091D5
:10FBB00078005091790060E070E080914E0A909159
:10FBC0004F0AA091500AB091510A840F951FA61FA9
:10FBD000B71F80934E0A90934F0AA093500AB09398
:10FBE000510A82E080934D0A61C088E080937B00D7
:10FBF00082E480937C0080917A00806480937A0014
:10FC00000E942E3283E0EECF40917800509179002F
:10FC100060E070E08091520A9091530AA091540ADA
:10FC2000B091550A840F951FA61FB71F8093520AE3
:10FC30009093530AA093540AB093550A84E0D2CF0C
:10FC400088E080937B0081E480937C0080917A003F
:10FC5000806480937A000E942E3285E0C3CF409169
:10FC600078005091790060E070E08091560A9091A0
:10FC7000570AA091580AB091590A840F951FA61FE0
:10FC8000B71F8093560A9093570AA093580AB093CF
:10FC9000590A86E0A7CF0E942E3287E0A3CF1092A8
:10FCA0004D0A80915A0A8F5F80935A0A80915A0AAE
:10FCB000803108F45DC020914E0A30914F0A309394
:10FCC0001F0A20931E0A8FEF9FE34091520A509122
:10FCD000530A841B950B90931D0A80931C0A81E0A4
:10FCE0008093170A10925A0A10924E0A10924F0AE5
:10FCF0001092500A1092510A1092560A1092570A06
:10FD00001092580A1092590A10925B0A10925C0ADB
:10FD100010925D0A10925E0A1092520A1092530AD3
:10FD20001092540A1092550A80913A0490913B0423
:10FD3000281739074CF01092230A1092220A80E00B
:10FD40000E94077D0E94B82C20911E0A30911F0A44
:10FD50008091460A9091470A821793074CF01092BF
:10FD6000230A1092220A80E00E94477D0E94B82C4C
:10FD7000FF91EF91BF91AF919F918F917F916F9183
:10FD80005F914F913F912F910F900BBE0F900FBE3F
:10FD90000F901F9018951F920F920FB60F920BB6EF
:10FDA0000F9211242F933F934F935F936F938F93F1
:10FDB0009F93EF93FF936091C6002091E00A3091EA
:10FDC000E10AC90101968F7790704091E20A509143
:10FDD000E30A8417950741F0205A354FF9016083F3
:10FDE0009093E10A8093E00AFF91EF919F918F91A8
:10FDF0006F915F914F913F912F910F900BBE0F909C
:10FE00000FBE0F901F9018950F931F939A01AB018F
:10FE1000203081EE380780E0480780E0580769F11C
:10FE200082E08093C00060E079E08DE390E00E9482
:10FE300036AB89019A010150104020403040C90181
:10FE4000B80122E030E040E050E00E9436AB309351
:10FE5000C5002093C4008091C10080618093C100DF
:10FE60008091C10088608093C1008091C10080684A
:10FE70008093C1001F910F9108951092C00020E15E
:10FE800030E0E5CF2091E20A3091E30A8091E00A68
:10FE90009091E10A8217930771F0F901E05AF54F4A
:10FEA00080812F5F3F4F2F7730703093E30A20938C
:10FEB000E20A90E008958FEF9FEF08958091E20AA3
:10FEC0009091E30A9093E10A8093E00A08956F927B
:10FED0007F928F929F92AF92BF92CF92DF92EF92DA
:10FEE000FF920F931F93CF93DF93CDB7DEB7A09709
:10FEF0000FB6F894DEBF0FBECDBF3C01DB01CA01D7
:10FF0000411551056105710551F4C30140E350E00D
:10FF100060E070E020E030E00E94FA7F41C08E0196
:10FF20000F5F1F4FCC24DD247601822E9924AA2452
:10FF3000BB24BC01CD01A50194010E9414ABF801C2
:10FF400061938F010894C11CD11CE11CF11CC901F3
:10FF5000DA010097A105B10561F714C0E1E0F0E016
:10FF6000EC0FFD1FEC0DFD1D40814A3010F4405D8B
:10FF700001C0495C50E060E070E0C30120E030E087
:10FF80000E94FA7F0894C108D108E108F108FFEF48
:10FF9000CF16FFEFDF06FFEFEF06FFEFFF06F1F6EC
:10FFA000A0960FB6F894DEBF0FBECDBFDF91CF9104
:10FFB0001F910F91FF90EF90DF90CF90BF90AF9087
:10FFC0009F908F907F906F9008952115310539F49F
:10FFD0008091C00085FFFCCF4093C60008950E9429
:10FFE000677F08959A01462F50E060E070E00E941C
:10FFF000E57F0895CF92DF92EF92FF92CF93DF9348
:020000021000EC
:10000000EC016A017B012115310539F48091C000B2
:1000100085FFFCCFC092C6001BC02A303105B1F469
:1000200077FF10C04DE250E060E070E020E030E08B
:100030000E94FA7FF094E094D094C094C11CD11C2B
:10004000E11CF11CCE01B701A6012AE00E94677FE6
:10005000DF91CF91FF90EF90DF90CF9008959A01BC
:10006000FB01AF01662757FD6095762F0E94FA7F4E
:100070000895CF93DF93EC014DE050E060E070E035
:1000800020E030E00E94FA7FCE014AE050E060E0DC
:1000900070E020E030E00E94FA7FDF91CF91089578
:1000A000CF93DF93EC019A01AB0160E070E00E9416
:1000B000E57FCE010E943980DF91CF9108958F9224
:1000C0009F92BF92CF92DF92EF92FF920F931F9376
:1000D000CF93DF934C016A017B01B22ECB01BA01B1
:1000E00020E030E040E050E00E9433A787FF0DC0E1
:1000F000C4014DE250E060E070E020E030E00E949A
:10010000FA7FF7FAF094F7F8F094C0E050E040E09E
:1001100030E02FE313C0FA01B9018F2F942FA72FDE
:10012000B22FBC01CD0120E030E040E251E40E945A
:100130003AA7562F472F382F292FCF5FCB1559F7C6
:10014000C701B601DA01F9010B2F142F2F2F3E2F13
:10015000A90198010E945AA66B01E82EC92F862F8B
:100160009D2DAE2DBC2FBC01CD010E94A7A7D62F7F
:10017000172F082FF92E0E94D3A79B01AC018C2DBD
:100180009D2DAE2DBC2FBC01CD010E9459A6D62EAF
:10019000E72EC82FC92EC4014D2F512F602F7F2D60
:1001A0002AE030E00E94E57FBB2009F446C0E5EC80
:1001B000F3E006C09091C00095FFFCCF8093C6008D
:1001C00081918823B9F739C08D2D9E2DAC2FBC2D80
:1001D000BC01CD0120E030E040E251E40E9408AAD9
:1001E000EB01182F092F9801862F9D2FA32FB22FD7
:1001F000BC01CD010E94A2A76B017C01EE24D7FCBB
:10020000E094FE2CC401B701A6012AE030E00E9470
:10021000FA7FC701B6010E94D5A79B01AC01B801C6
:100220008C2F9D2FA72FB62FBC01CD010E9459A660
:10023000D62EE72EC82FC92EBA94BB2029F6DF91FF
:10024000CF911F910F91FF90EF90DF90CF90BF90D3
:100250009F908F9008950E945F800895CF93DF93C1
:10026000FC01168A118E158A148A81E494E0938B1E
:10027000828B17AA12AE16AA15AA94AB83ABDF0124
:10028000AA5ABF4F1C9213961C92DF01AE5ABF4F61
:1002900013961C921E9212978D939C93DF01AB587C
:1002A000BF4F1C9213961C92DF01AF58BF4F13969D
:1002B0001C921E9212978D939C93DF01A057BF4F03
:1002C00029E111962C93119714961C92DF01A455E5
:1002D000BF4F1C92DF01A954BF4F1C9213961C9272
:1002E000DF01AD54BF4F13961C921E9212978D934F
:1002F0009C93DF01AE52BF4F1D921D921D921C9226
:100300001397DF01A652BF4F1D921D921D921C92A2
:100310001397118212821082EF01CA52DF4F1882A6
:1003200019821A821B82DF01A252BF4F81E08C9397
:10033000118A108A0E9425A3DC01CB0188579C4EAC
:10034000AF4FBF4F88839983AA83BB83DF91CF913F
:100350000895DB01FC0120E03EE24C91403229F09F
:10036000283009F431934C9141932F5F11962B3033
:10037000A1F7108208952F923F924F925F926F9251
:100380007F928F929F92AF92BF92CF92DF92EF9225
:10039000FF920F931F93CF93DF93CDB7DEB7C7586C
:1003A000D0400FB6F894DEBF0FBECDBF8C015B010D
:1003B0006A01FF2484E090E0C80ED91E23E0422E9B
:1003C000512C400E511E3FED832E912C800E911E1C
:1003D000E0EE6E2E712C600E711EF1E42F2EF4E013
:1003E0003F2EE7E4F0E0EC0FFD1F3496CA57DF4FD5
:1003F000F983E883C658D040E7E8F4E1E4900FC100
:10040000E2968FADE29790E09C0128713070203128
:10041000310509F00EC1F4014081413009F409C1F0
:10042000423009F406C1CE010196BE016A597F4FE0
:100430000E94A9811E86F5018081882331F4CE01B6
:100440000E9667EC73E00E9451AECE010E96B50198
:100450000E9451AECE010E96BE016F5F7F4F0E948B
:1004600051AECE010E9667EC73E00E9451AE2C9611
:100470001FAE2C972F961FAE2F972B961FAE1EAE3A
:100480002B9729963FAE2EAE2997CA57DF4F88810A
:100490009981C658D040B601AE014F5F5F4F21E051
:1004A0000E94B51D8823C1F5F40180818823A1F540
:1004B0008E2DE7E8F4E108C09091C00095FFFCCFD5
:1004C0008093C600319684918823B1F7E9ECF3E07C
:1004D00006C09091C00095FFFCCF8093C60081912B
:1004E0008823B9F78091C00085FFFCCF8AE0809314
:1004F000C600FE01319606C09091C00095FFFCCF6A
:100500008093C60081918823B9F78091C00085FF50
:10051000FCCF8AE08093C600FE01BC96CA57DF4F2D
:10052000A881B981C658D0408BE10D9001928150CD
:10053000E1F72B968EAD9FAD2B979BA78AA739A687
:1005400028A6C801BE01625F7F4FAE01485D5F4FC4
:100550000E94BB81CE0188960E94B874CE01895B4F
:100560009F4F0E94B8745BC0453E09F458C04E329C
:1005700009F455C04F3509F452C083FD50C081E0E5
:100580002031310509F080E0F8018787882359F48C
:10059000AF968FADAF97873409F041C0E0968FAD2D
:1005A000E0978E37E1F1C201BE016A597F4F0E9488
:1005B000A981F40180818823F1F4F50106C09091AE
:1005C000C00095FFFCCF8093C60081918823B9F7C6
:1005D000F20106C09091C00095FFFCCF8093C60049
:1005E00081918823B9F78091C00085FFFCCF8AE014
:1005F0008093C60014C0813039F4F3018081918169
:100600000196918380830BC0823049F48F2D90E056
:10061000F301208131818217930789F0F394C60199
:10062000BE016A597F4F0E94271A18160CF4E8CEB3
:1006300006C0A7964FADA797442309F095CFC95799
:10064000DF4F0FB6F894DEBF0FBECDBFDF91CF9165
:100650001F910F91FF90EF90DF90CF90BF90AF90E0
:100660009F908F907F906F905F904F903F902F90D2
:100670000895EF92FF920F931F93CF93DF93CDB71F
:10068000DEB76F970FB6F894DEBF0FBECDBF7C010B
:10069000FC01E152FF4F10828C010A5E1F4FC8011E
:1006A0000E94311BFE013596D8018BE10D9001921D
:1006B0008150E1F7F701848995899C838B8381E4DC
:1006C00094E09A838983C7016CED73E0AE014F5FBC
:1006D0005F4F0E94BB81CE0101960E94B8746F9655
:1006E0000FB6F894DEBF0FBECDBFDF91CF911F9143
:1006F0000F91FF90EF900895EF92FF920F931F9349
:10070000CF93DF937C01FC011282818D882321F03D
:10071000C70146960E94831BE701C057DF4FCE01F9
:1007200060E045E30E94130D8823F9F4E7E8F4E163
:1007300007C09091C00095FFFCCF8093C600319612
:1007400084918823B1F7EDE8F4E107C09091C000EF
:1007500095FFFCCF8093C600319684918823B1F732
:100760008091C00085FFFCCF77C087010B561F4FDB
:10077000C801BE0141E00E94AB23882331F5C801C6
:10078000BE0140E00E94AB238823F9F4EAE9F4E1DA
:1007900007C09091C00095FFFCCF8093C6003196B2
:1007A00084918823B1F7E1EAF4E107C09091C00099
:1007B00095FFFCCF8093C600319684918823B1F7D2
:1007C0008091C00085FFFCCF47C0C7014696B801A5
:1007D0000E9486188823F9F4EAE9F4E107C09091B1
:1007E000C00095FFFCCF8093C6003196849188238A
:1007F000B1F7E4EBF4E107C09091C00095FFFCCFA6
:100800008093C600319684918823B1F78091C0000F
:1008100085FFFCCF21C081E0F7018283E7E8F4E1A6
:1008200007C09091C00095FFFCCF8093C600319621
:1008300084918823B1F7E4ECF4E107C09091C00003
:1008400095FFFCCF8093C600319684918823B1F741
:100850008091C00085FFFCCF8AE08093C600D7015D
:10086000D796F70176968BE101900D928150E1F7D2
:10087000F7018489958996AB85ABC701429692AB07
:1008800081ABDF91CF911F910F91FF90EF90089571
:10089000CF93DF93FC01EC01E796DC0156968BE1E8
:1008A0000D9009928150E1F78489958996AB85ABCB
:1008B000CF01C39692AB81ABDF91CF910895FC013C
:1008C000118212820895FC018281882311F081E057
:1008D00081830895FC0181818111118208952F92F5
:1008E0003F924F925F926F927F928F929F92AF92C0
:1008F000BF92CF92DF92EF92FF920F931F93CF930D
:10090000DF93CDB7DEB7AC970FB6F894DEBF0FBE5E
:10091000CDBF6C014B01442EFC018281882309F478
:10092000BEC117EB612E712C6C0C7D1CC3010E94A3
:10093000831BF60111821A8A1D8A198A188A81E49A
:1009400094E09F878E87C601429692AB81ABF401FB
:1009500080818F3209F08EC0C4016FE270E00E9486
:100960005CAE7C010894E11CF11CAAE05A2EBEE0AA
:100970002B2E312C2C0E3D1E78C0C7016FE270E08B
:100980000E945CAE5C01009709F47CC0E816F90691
:1009900008F078C08C010E191F09CE010196B7012D
:1009A000A8010E947CAEE1E0F0E0EC0FFD1FE00F3B
:1009B000F11F10828E010F5F1F4FF80106C090914A
:1009C000C00095FFFCCF8093C60081918823B9F7C2
:1009D0008091C00085FFFCCF5092C600F60161A94E
:1009E00072A96115710519F06C5F7F4F02C060E05C
:1009F00070E0CE014296AE014F5F5F4F21E00E9452
:100A0000B51D882359F5EFECF4E107C09091C000C3
:100A100095FFFCCF8093C600319684918823B1F76F
:100A200006C09091C00095FFFCCF8093C600F801EE
:100A300081918F018823A9F7E3EEF4E107C090913B
:100A4000C00095FFFCCF8093C60031968491882327
:100A5000B1F78091C00085FFFCCFF3C0F60132AA48
:100A600021AA75010894E11CF11CE114F10409F0BC
:100A700084CF05C0C601C396F60192AB81ABE82CCA
:100A8000092D01C00F2DF60161A972A9442009F4B6
:100A90009EC06115710519F06C5F7F4F02C060E068
:100AA00070E0C3014E2D502F21E00E94B51D882318
:100AB00009F462C096012E523F4FF601E954FF4FF0
:100AC00081899289A389B489F90180839183A28362
:100AD000B383E5EEF4E107C09091C00095FFFCCF31
:100AE0008093C600319684918823B1F7EE2DF02FC4
:100AF00006C09091C00095FFFCCF8093C600819105
:100B00008823B9F7E2EFF4E107C09091C00095FFA8
:100B1000FCCF8093C600319684918823B1F7F6010B
:100B2000EE52FF4F40815181628173818FE59AE0DF
:100B30002AE030E00E94E57F8091C00085FFFCCF75
:100B40008AE08093C600F601E652FF4F10821182C0
:100B500012821382E9EFF4E107C09091C00095FF83
:100B6000FCCF8093C600319684918823B1F78091A1
:100B7000C00085FFFCCF88C0E7E0F5E107C0909199
:100B8000C00095FFFCCF8093C600319684918823E6
:100B9000B1F7EE2DF02F06C09091C00095FFFCCF6D
:100BA0008093C60081918823B9F7EBE1F5E107C096
:100BB0009091C00095FFFCCF8093C6003196849140
:100BC0008823B1F78091C00085FFFCCF3AC0611542
:100BD000710519F06C5F7F4F02C060E070E0C301E7
:100BE0004E2D502F26E50E94B51D882371F5EDE1AD
:100BF000F5E107C09091C00095FFFCCF8093C6003F
:100C0000319684918823B1F7EE2DF02F06C0909194
:100C1000C00095FFFCCF8093C60081918823B9F76F
:100C2000E1E3F5E107C09091C00095FFFCCF809310
:100C3000C600319684918823B1F78091C00085FF6A
:100C4000FCCF8AE08093C60026C081E0F601808355
:100C5000E3E3F5E107C09091C00095FFFCCF8093DE
:100C6000C600319684918823B1F7F40106C09091B3
:100C7000C00095FFFCCF8093C60081918823B9F70F
:100C80008091C00085FFFCCF8AE08093C6008E2D46
:100C9000902F0E94882CCE010E960E94B874AC96BC
:100CA0000FB6F894DEBF0FBECDBFDF91CF911F917D
:100CB0000F91FF90EF90DF90CF90BF90AF909F90FB
:100CC0008F907F906F905F904F903F902F900895FE
:100CD0004F925F927F928F929F92AF92BF92CF92EC
:100CE000DF92EF92FF920F931F93CF93DF93CDB7D5
:100CF000DEB7AC970FB6F894DEBF0FBECDBF6C0168
:100D00004B01FC018281882309F410C1C60189547A
:100D10009F4F0E94831BF60111821A8A1D8A198A2D
:100D2000188A81E494E09F878E87C601429692AB31
:100D300081ABF40180818F3209F08EC0C4016FE273
:100D400070E00E945CAE7C010894E11CF11C0AE09A
:100D5000702E2EE0422E512C4C0E5D1E78C0C70125
:100D60006FE270E00E945CAE5C01009709F47CC009
:100D7000E816F90608F078C08C010E191F09CE019B
:100D80000196B701A8010E947CAEE1E0F0E0EC0F13
:100D9000FD1FE00FF11F10828E010F5F1F4FF80142
:100DA00006C09091C00095FFFCCF8093C600819152
:100DB0008823B9F78091C00085FFFCCF7092C600F0
:100DC000F60161A972A96115710519F06C5F7F4F79
:100DD00002C060E070E0CE014296AE014F5F5F4F0F
:100DE00021E00E94B51D882359F5E5E4F5E107C02F
:100DF0009091C00095FFFCCF8093C60031968491FE
:100E00008823B1F706C09091C00095FFFCCF809376
:100E1000C600F80181918F018823A9F7E9E5F5E182
:100E200007C09091C00095FFFCCF8093C60031961B
:100E300084918823B1F78091C00085FFFCCF6FC0FB
:100E4000F60152AA41AA75010894E11CF11CE114B3
:100E5000F10409F084CF05C0C601C396F60192AB38
:100E600081ABE82C092D01C00F2DF60181A992A9B3
:100E7000009711F0049602C080E090E06E2D702F74
:100E80000E94771E882309F1EBE5F5E107C09091F8
:100E9000C00095FFFCCF8093C600319684918823D3
:100EA000B1F7EE2DF02F06C09091C00095FFFCCF5A
:100EB0008093C60081918823B9F7F601E652FF4F6F
:100EC00010821182128213822DC0E9E6F5E107C07B
:100ED0009091C00095FFFCCF8093C600319684911D
:100EE0008823B1F7EE2DF02F06C09091C00095FF3A
:100EF000FCCF8093C60081918823B9F7E1E8F5E142
:100F000007C09091C00095FFFCCF8093C60031963A
:100F100084918823B1F78091C00085FFFCCF8AE0DF
:100F20008093C600CE010E960E94B874AC960FB6A0
:100F3000F894DEBF0FBECDBFDF91CF911F910F910F
:100F4000FF90EF90DF90CF90BF90AF909F908F90E9
:100F50007F905F904F900895CF93DF93EC018A814B
:100F60008823C1F1E3E8F5E107C09091C00095FF47
:100F7000FCCF8093C600319684918823B1F7FE019F
:100F8000E652FF4F40815181628173818FE59AE083
:100F90002AE030E00E94E57FE5E9F5E107C09091A5
:100FA000C00095FFFCCF8093C600319684918823C2
:100FB000B1F7CE52DF4F488159816A817B818FE53D
:100FC0009AE02AE030E00E94E57F8091C00085FF32
:100FD000FCCF11C0E7E9F5E107C09091C00095FF93
:100FE000FCCF8093C600319684918823B1F780911D
:100FF000C00085FFFCCF8AE08093C600DF91CF91CF
:101000000895CF92DF92EF92FF920F931F93CF93A9
:10101000DF936C017B01DB010D900020E9F78D016E
:1010200001501040061B170BFC01E954FF4F1082C2
:10103000CB016EE470E00E945CAEEC01009729F4F5
:10104000F8013197EE0DFF1D0FC060E270E00E94C5
:101050005CAE7C010894E11CF11CCE016AE270E0F8
:101060000E945CAEFC0131978DE081838AE082832F
:101070001382C6018D549F4FB7010E940B25F601C4
:10108000E954FF4F8081882309F1EAE9F4E107C0C0
:101090009091C00095FFFCCF8093C600319684915B
:1010A0008823B1F7E7EAF5E107C09091C00095FF0A
:1010B000FCCF8093C600319684918823B1F780914C
:1010C000C00085FFFCCF8AE08093C600DF91CF91FE
:1010D0001F910F91FF90EF90DF90CF9008952F9286
:1010E0003F924F925F926F927F929F92AF92BF9288
:1010F000CF92DF92EF92FF920F931F93CF93DF93E4
:10110000CDB7DEB7CC55D0400FB6F894DEBF0FBEDA
:10111000CDBF5C016623C1F4FC01E252FF4F808128
:10112000882309F4D8C0F501EA52FF4FC080D1806E
:10113000E280F3800E9425A3DC01CB01C816D9060A
:10114000EA06FB0608F4C7C0F501E252FF4F108221
:10115000D50112968C911297882341F4C5010E9403
:101160007C83F5018281882309F4B5C000D000D0CA
:10117000EDB7FEB731965FE1C52ED12CCC0EDD1E4A
:10118000ADB7BEB71296DC92CE9211978DED93E07B
:1011900093838283D50150968D919C91519795832D
:1011A00084830E94A5AEEDB7FEB736960FB6F894CD
:1011B000FEBF0FBEEDBF860108C0D6018C9190E046
:1011C0000E941BAEF60181936F01F801019000208F
:1011D000E9F73197E01BF10BC601801B910B8E17CD
:1011E0009F075CF336E1432E512C4A0C5B1CC20175
:1011F0000E94311B99248E01035C1F4F4FE1242E66
:10120000312C2C0E3D1E3E010894611C711C47C000
:10121000D6018C9190E00E941BAEF60181936F0184
:10122000C701F80101900020E9F73197E01BF10BAD
:101230000894E11CF11C8E179F0754F327968FAD7D
:1012400027978E3761F1C801B10145E050E00E9457
:101250006EAE009721F500D000D0EDB7FEB7319605
:10126000ADB7BEB712967C926E92119786EE93E060
:1012700093838283358224820E94A5AEADB7BEB728
:1012800016960FB6F894BEBF0FBEADBFC3010E9445
:101290000C298DEE93E00E940C2999249394C201AD
:1012A000B8010E94271A181624F46801EE24FF24BE
:1012B000B7CF992031F48FEF9FEFF501918B808BA1
:1012C0000AC0D50150968D919C91519701965196E7
:1012D0009C938E935097C45ADF4F0FB6F894DEBF9D
:1012E0000FBECDBFDF91CF911F910F91FF90EF9077
:1012F000DF90CF90BF90AF909F907F906F905F9066
:101300004F903F902F9008950F931F93CF93DF93AB
:101310008C01EC01C954DF4FCE010E94381BCE0175
:101320000E94831BF8011082DF91CF911F910F91D2
:1013300008950F931F93CF93DF93CDB7DEB76F97C9
:101340000FB6F894DEBF0FBECDBF8C01C396F80177
:1013500092AB81ABE152FF4F82E08083F801E05213
:10136000FF4F60831182C801C7960E94311BF801AC
:1013700081A992A9DE011596FC0134962BE101901A
:101380000D922150E1F7FC01828193819C838B8334
:1013900081E494E09A838983C8016CED73E0AE0127
:1013A0004F5F5F4F0E94BB81CE0101960E94B874CF
:1013B0006F960FB6F894DEBF0FBECDBFDF91CF9111
:1013C0001F910F9108950F931F93CF93DF93CDB784
:1013D000DEB76F970FB6F894DEBF0FBECDBF8C019E
:1013E000C396F80192AB81ABE152FF4F81E080835D
:1013F000F801E052FF4F11821082C801C7960E9487
:10140000311BF80181A992A9DE011596FC013496E1
:101410002BE101900D922150E1F7FC018281938133
:101420009C838B8381E494E09A838983C8016CED6B
:1014300073E0AE014F5F5F4F0E94BB81CE0101960A
:101440000E94B874F801E052FF4F808191816F963D
:101450000FB6F894DEBF0FBECDBFDF91CF911F91C5
:101460000F910895CF92DF92EF92FF920F931F9307
:10147000CF93DF93CDB7DEB76F970FB6F894DEBF8B
:101480000FBECDBF8C01F62EE72E1D8218861C8262
:101490001B8281E494E09A838983F80182AD8823DA
:1014A00021F472E1C72ED12C03C063E3C62ED12CE8
:1014B000C00ED11EB6016C5F7F4FCE0105964F2D39
:1014C0005E2D21E00E94B51D882371F5E7E8F4E167
:1014D00007C09091C00095FFFCCF8093C600319665
:1014E00084918823B1F7EDEBF5E107C09091C0003E
:1014F00095FFFCCF8093C600319684918823B1F785
:10150000EF2DFE2D06C09091C00095FFFCCF80937B
:10151000C60081918823B9F78091C00085FFFCCF78
:101520008AE08093C60035C098012F583F4FF901DB
:101530003496D801AA5ABF4F8BE10D900192815089
:10154000E1F7F801EC5AFF4F80819181F901938313
:101550008283D801AA5ABF4FF60134968BE10190DD
:101560000D928150E1F7F60182819381F801EE5AE4
:10157000FF4F93838283D801D796FE0135968BE186
:1015800001900D928150E1F78B819C81F80196AB1F
:1015900085ABCE0101960E94B8746F960FB6F89491
:1015A000DEBF0FBECDBFDF91CF911F910F91FF9096
:1015B000EF90DF90CF900895CF93DF93EC018AAD49
:1015C0008250823028F1DE01D796FE01EA5AFF4FA1
:1015D0008BE101900D928150E1F7FE01EC5AFF4F33
:1015E000808191819EAB8DABCE018E5A9F4FDC01E5
:1015F0001496FE01EB58FF4F2BE101900D92215004
:10160000E1F7CD58DF4F28813981FC0133832283F4
:10161000DF91CF910895CF93DF93EC010E948B1659
:101620000E940817198281EF93E00E940C29DF9134
:10163000CF9108952F923F924F925F926F927F9237
:101640008F929F92AF92BF92CF92DF92EF92FF92D2
:101650000F931F93CF93DF93CDB7DEB7C055D04024
:101660000FB6F894DEBF0FBECDBF2C017A8F698F05
:101670004A012CA708AFE9AEAAAEBBAECCAEDDAE38
:10168000022F10E0000F111F000F111F9A01200FF1
:10169000311F3DAB2CABD9018D919D910D90BC912B
:1016A000A02D898B9A8BAB8BBC8BF201E00FF11FC5
:1016B000BC01CD0120813181428153810E945AA613
:1016C0006EAF7FAF21968FAF219722969FAF229763
:1016D000B8ADEB2EFF24EE0CFF1CEE0CFF1CF4014A
:1016E000EE0DFF1DFFABEEAB80809180A280B3803A
:1016F000F201EE0DFF1DC501B4012081318142814F
:1017000053810E945AA623966FAF239724967FAFEA
:10171000249725968FAF259726969FAF2697F9ADEC
:101720008F2F90E0880F991F880F991FF201E80F03
:10173000F91F20813181428153812B8F3C8F4D8F46
:101740005E8FE98DFA8DE80FF91F608171818281CA
:1017500093810E9459A6462F572F682F792F4F8FBC
:1017600058A369A37AA3A98DBA8D1C968D919D91DA
:101770000D90BC91A02D88AB99ABAAABBBABD201AD
:101780001C962D913D914D915C911F972FA338A7E9
:1017900049A75AA729893A894B895C895058298BCE
:1017A0003A8B4B8B5C8BD501C401B0588D8B9E8BD3
:1017B000AF8BB88FE98DFA8DE00FF11F60817181D9
:1017C00082819381FEADEFAD21965FAD2197229688
:1017D0004FAD22970F2F1E2F252F342FA9019801CF
:1017E0000E9459A66B01482E792EE98DFA8DEE0DD7
:1017F000FF1D60817181828193812396FFAD2397C4
:101800002496EFAD249725965FAD259726964FAD8C
:1018100026970F2F1E2F252F342FA90198010E94E4
:1018200059A6F62EE72E682E592E69897A898B895A
:101830009C89F7010F2F1E2F262D352DA901980108
:101840000E9408AA4B015C016D897E898F89988D61
:101850000C2D1D2D242D372DA90198010E9408AAB9
:101860009B01AC01C501B4010E9459A66BA37CA3E6
:101870008DA39EA369897A898B899C89242D372D14
:10188000A90198010E9408AA4B015C016D897E891B
:101890008F89988DF7010F2F1E2F262D352DA90129
:1018A00098010E9408AA9B01AC01C501B4010E94E5
:1018B0005AA69B01AC016BA17CA18DA19EA10E94A7
:1018C000CDA6162F072FF82EE92EA8019701852FF8
:1018D000942FA32FB22FBC01CD0120E030E040E0D7
:1018E00050E00E9433A787FF12C0A8019701852FFF
:1018F000942FA32FB22FBC01CD012BED3FE049EC7B
:1019000050E40E945AA6162F072FF82EE92EAB9608
:101910008FADAB97882391F0A8019701852F902F69
:10192000A32FBE2DBC01CD012BED3FE049EC50E4CF
:101930000E9459A6162F072FF82EE92EA80197010D
:10194000852F902FA32FBE2DBC01CD01AA962CADC3
:101950003DAD4EAD5FADAA970E9408AA2F8D38A16C
:1019600049A15AA15F770E9443A94B015C012FE670
:1019700032E143E85AE30E9433A787FD6AC2C501FA
:10198000B4010E9410A80E94A7A7DC01CB019FA769
:101990008EA7009721F4A1E0B0E0BFA7AEA7EEA507
:1019A000FFA5BF0180E090E00E94D3A74B015C013E
:1019B000A8019701852F902FA32FBE2DBC01CD012B
:1019C000A50194010E943AA7362E272E8BA39BA730
:1019D0006F8D78A189A19AA1A50194010E943AA7CF
:1019E0002A966FAF2A972B967FAF2B972C968FAFA7
:1019F0002C972D969FAF2D9768A979A98AA99BA9A5
:101A00002FA138A549A55AA50E9459A6A501940160
:101A10000E943AA72E966FAF2E972F967FAF2F97E3
:101A200060968FAF609761969FAF6197A1013BA1D0
:101A30002BA5852F942FA32FB22FBC01CD0120E021
:101A400030E040E05FE30E9408AAF1015BA14BA5F2
:101A50000F2F1E2F252F342FA90198010E9408AAAD
:101A60009B01AC0160E070E080E89FE30E9459A612
:101A700068AB27967FAF279728968FAF2897299630
:101A80009FAF299729ADE22FF0E0EE0FFF1FEE0F79
:101A9000FF1FCE010196E80FF91F2B8D3C8D4D8D58
:101AA0005E8D20833183428353832FA138A549A5BE
:101AB0005AA52D873E874F87588B882441E050E0F8
:101AC00058A74FA3BCA5AB2FB0E0AA0FBB1FAA0F0E
:101AD000BB1F9C012A0F3B1F3C8F2B8F58AD452FFE
:101AE00050E0440F551F440F551F81E090E08C0FCC
:101AF0009D1F840F951F98A38F8FFDA7ECA788C10A
:101B000098E198150CF46FC069897A898B899C8952
:101B1000432D522DEBA1FBA58A019F01A90198013C
:101B20000E9408AA6B017C016D897E898F89988D3E
:101B300048A927965FAD27972896EFAD2897299655
:101B4000FFAD29978A019F01A90198010E9408AA67
:101B50009B01AC01C701B6010E945AA6762E672EE2
:101B6000582E492E69897A898B899C892896EFADF0
:101B700028972996FFAD29979F01A90198010E94F6
:101B800008AAF62EE72ED82EC92E6D897E898F8958
:101B9000988D432D522DEBA1FBA58A019F01A90130
:101BA00098010E9408AA9B01AC01F701B6018F2F92
:101BB0009E2FA72FB62FBC01CD010E9459A6462FFC
:101BC000572F682F792F498B5A8B6B8B7C8B839483
:101BD000A3019201852F942FA32FB22F8D8B9E8B63
:101BE000AF8BB88F81C0AFA1B8A5BD0180E090E0F8
:101BF0000E94D3A7432D522DEBA1FBA58A019F0183
:101C0000A90198010E9408AA162F072FF82EE92E85
